:109C6A00414952434F544543004256332E33342020
:109C7A00455350004558414300532F4E2146414910
:109C8A004C555245005245454E54455221532F4E8C
:109C9A0000434F4E5441435420414952434F544587
:109CAA004300475053004032444000403344400090
:109CBA00415047214E564F404D454E55000A160019
:109CCA000180000300007E0000FE00001E00003636
:109CDA000003E60001C4000000000FFFE0425553F4
:109CEA0043415240534154200043414C40414C545B
:109CFA0049202300494D4147454E20200052414EFC
:109D0A004B494E47004D41504120202020004345F9
:109D1A004E54524F202000564152494F20202000D5
:109D2A004241524F4752202000525554415320205D
:109D3A00200043455243412020200042414C495AC9
:109D4A00412020004D4152434153202000504F52A0
:109D5A0021444546454300202020214449532120DF
:109D6A002020204D454400545241434B21454E4347
:109D7A002000545241434B2141504720004D41524B
:109D8A004B00545241434B2D4152524942004E4FCF
:109D9A005254452D4152524942002153414C495295
:109DAA0020200153454C40525554412001434F4E07
:109DBA0046494720414C54015655454C4F532020A3
:109DCA006869015655454C4F5320544F440142414E
:109DDA004C495A4153206869015255544153202035
:109DEA002068690145535021414552454F68690130
:109DFA00434F4E4649472020686900434F4E464923
:109E0A004720414C5400414C54404241524F20207B
:109E1A0000414C542047505320202000514E4820E6
:109E2A00202020402148504100464C0052454749D5
:109E3A00535420564143494F20003E2153414C4937
:109E4A005220200053414C495220200156455220AD
:109E5A00202001454E5649415201424F5252415229
:109E6A00002153414C4952202001434F4D3A2020B2
:109E7A002020202001544E432031232035374B0126
:109E8A00544E4320312320392E3601015057434086
:109E9A003130234035374B0150574340313023404E
:109EAA0031394B01014D5850403130234035374B41
:109EBA00014D58502034232035374B014D5850203E
:109ECA0031232035374B014D585040313023403132
:109EDA00394B014D58502031232031394B00215341
:109EEA00414C49522020014E56412042414C4920C2
:109EFA00200145444954412042414C4901424F52B4
:109F0A0052412042414C490101434F4D3A015245C9
:109F1A004349422042414C4901454E56494120425B
:109F2A00414C4901454E56405444534042414C012C
:109F3A0001444953542142414C2142414C01424F70
:109F4A005252215444532142414C00444952202147
:109F5A004449535400475241422000504F53494309
:109F6A004041435455414C004D454D4F52494120C3
:109F7A0020002053544F5245215750542000204668
:109F8A00554C4C20002140424F52524152005345F9
:109F9A005220004952444100555342200055534231
:109FAA0020004C49535400454E5620002045525239
:109FBA004F52205452414E534D49432000215341A0
:109FCA004C495220200153454C20525554412001FE
:0D9FDA004E5641205020525554410145443F
:109FE700495441205255544101494E564552542037
:109FF70052555401424F525241205020525401426F
:10A007004F52524120525554410143594C2052411D
:10A017004449555301434F4D3A0152454349422064
:10A027005255544101454E5649412052555441011C
:10A03700434845434B2052550053454C21525554F4
:10A047004120004E5545564F00204E564140504F37
:10A057005340210021494E56455254495200494E1A
:10A06700564552540021424F52405040525420000E
:10A0770021424F52205255544100564143494120F5
:10A087004E4F2020002140454E5640525554410026
:10A097002020524144495553002153414C49520114
:10A0A70043415247415220435452015645522020C2
:10A0B700202043545201424F5240544453214354A9
:10A0C700520101434F4D3A015245434942495221FA
:10A0D70043545201454E564941522043545200566B
:10A0E7004552204354522020202020202020004D7C
:10A0F7004F5645522020004D4F5645522148414367
:10A10700494100455343202020582F5920205341CF
:10A117004C495200424F5220444953540041555430
:10A127004F2E454E43004155544F2E415047002076
:10A137002020455343414C0044495354204B4D0084
:10A1470044495354204E4D002153414C495220203D
:10A1570001564152494F20202068690158432D4339
:10A167004F4E4649686901434F4E46215255544167
:10A1770068690147454E4552414C20686901494D80
:10A187004147454E202068690101014D4F44214652
:10A197004143494C0156414C2146414252494341B2
:10A1A700015655454C4F21505255455601424F5285
:10A1B70021544F4421565545002153414C495220C3
:10A1C7002001544F4E2044455343014445534321F6
:10A1D7002D0144455343404D4F44014445534340AB
:10A1E700494E5601564152205443402020402301F6
:10A1F700564F4C554D454E01564152494F204E55ED
:10A207004C4F01534F4E49444F0146524543554524
:10A217004E4301564152214D4544212030402301F0
:10A22700544543202020403030402501534F4E20D5
:10A23700434845434B2000544F4E4F214445534319
:10A2470000444553432141504720004455414C2188
:10A257004E4F202000564152494F204E554C4F003B
:10A2670051554945544F203130204D494E2020202B
:10A2770000414E54455320444520414E554C4152D0
:10A28700002153414C495220200154524159454322
:10A29700544F014155544F43454E54010150524FBD
:10A2A7002F4449535401504C414E454F2020014CF7
:10A2B7002F44010157494E4421542D415001434534
:10A2C7004E5421542D415001574159505421425267
:10A2D70047002153414C4952202001484F524140E9
:10A2E7005350202020015052494D450144454C54BC
:10A2F700413A20014D554C5449504C452001554C8D
:10A3070054494D0143594C534947402020402301AC
:10A3170053454C4052555441200101010143594CCA
:10A32700520143494C20542D4152002153414C497D
:10A337005220200101554E494401434C49434B40AB
:10A34700302C40202301434F4E5452415354014E69
:0DA357004D45412131383301494D502F4112
:10A364004750530101432D564152494F014D454D2C
:10A374004F525944554D50004D454D4F5259445537
:10A384004D50004042414C495A2045584953544588
:10A394004E5445400042414C495A4120200020532C
:10A3A400414C495220202100524543494249520020
:10A3B4004C49425240003C2D204C495354202D3EE0
:10A3C4002020455849540053454C004E45585400EC
:10A3D40050524F582042414C0042414C20414E546F
:10A3E4002000424F5252215452414D00424F52528A
:10A3F4002153554D41004F46462020202020202047
:10A404002000204F4646004552524F524750532099
:10A4140020004755415244414E444F005255544147
:10A424002000434552434120004C495354410045C8
:10A43400544500414C54403000525554412056413B
:10A44400434941004D5543484F20202020002140DE
:10A4540053454C404C495354002053454C404241D1
:10A464004C4021002140524543494249524000207A
:10A4740020404F204B40202021004F4B005641529A
:10A48400004649580047415445215800535441520D
:10A49400544C494E452000535443594C2000404FDE
:10A4A40046460054502000406A40494E2000406710
:10A4B400404F555400204552524F52202021002035
:10A4C40053414C49004544495400405340490045D8
:10A4D40044495420204E564F204755415244410090
:10A4E40053494720202053454C202053414C495286
:10A4F400005843542D464C49474854200055534571
:10A504004400454E54455220004D4D2E4D4D4D2096
:10A51400004D4D2753532E530057475321383400D1
:10A524002040554054404D402000554054404D007B
:10A534002055544320004C4F43414C00535749533A
:10A5440053474400414C5400535549405800415628
:10A55400474020304023003530300031363430005D
:10A56400205D203130404B632F70005D202020316E
:10A5740040632F2300205D202035404B5453005D61
:10A58400203230304046504D00406340204B630041
:10A594004654204B6300406340204E4D00465420F7
:10A5A4004E4D004D2F53003230305E003530305E5A
:10A5B40000312200322200332200352200382200EA
:10A5C400464C3700464C313600464C333300464C3B
:10A5D40036350046313030004631363000463236AA
:10A5E40030005E252640534F47005E2526405441E7
:10A5F4005300414C540056415200225E2F24004B1C
:10A60400545300532F4E002224004B5400225E006A
:10A614004E4D00302C3500312C3000322C300030BF
:10A624002C3600312C3200322C3500332C380037D4
:10A634002C35004031350040333000403630005472
:10A6440041534B00464C2D44415445005450005452
:10A654004F46005354410046494E004C414E00536E
:10A664004554204F464653455400495341204845DC
:10A6740049474854004155544F2D474F20005354E7
:10A684004152540020434845434B40414C4C0052F6
:10A6940041442044495354004053454C40484549A3
:10A6A4004748543A00475053404241524F40414C6E
:0FA6B4004C0053494E4B40312D3221632F230070
:1064F400304D2475A7049005C2E0F51CE0F51DE0BD
:10650400F51EE0F51FE0F56DE0F56EE0F56FE0F5E2
:10651400541270B6126AF42275C70375C6E475B9CD
:1065240001E5BCB481431270B61256DC8E628F63EF
:106534007568F97569001265CA203C2D203B2B1241
:1065440066FF1266D3856D1C856E1D856F1E85548E
:106554001F126636203C12203243201D231266FF90
:10656400126AF4E532242850DC22126636203CF903
:10657400203DF6203205201DBD80EF301DB880EA95
:106584001266FF126AF4856D1C856E1D856F1E856B
:10659400541F1266E9126AF4203DCE8099126922D2
:1065A400201D0D7553107400126885203DBB808634
:1065B400E553540FC553C4540F20350512679A8010
:1065C40003126885808BC23CD23B126686FD12663C
:1065D40086FC126686C39573F565EC9574F564EDD7
:1065E4009575600504600A800EE56424E05011800E
:1065F40006E56424204009126686126686026686D1
:10660400126686FD126686FC126686C39576F56769
:10661400EC9577F566ED9578600904600122E566EE
:10662400F48002E5668562F0A474E025F04002C2BD
:0D6634003B22C23C126686A2E7923DA2E620
:10664100921DA2E592324026A2E492E592E692E7FB
:10665100FC1266862565F565EC3564F5641266867F
:10666100FC1266862567F567EC3566F56622A2E4BD
:106671009235540F79C6F712668609F7301D051257
:106681006686F55322E5697023E56860302404408D
:106691002CE56875F004A485F0C7F5C675B901E568
:1066A100BCB4811985BD68756902801E54037010E0
:1066B10005C675B901E5BC056953690F22D23C22B3
:1066C100147004E5BD80F0147004E5BE80E9E5BFF7
:1066D10080E575A7009006F6E56DF0A3E56EF0A3E1
:1066E100E56FF0A3E554F02275A7009006F6E0F5FA
:1066F1006DA3E0F56EA3E0F56FA3E0F55422E56428
:10670100B2E7F56D85656EAB67E566FC30E707C3FB
:10671100E49BFBE49CFCAA62A9631253DCE56630AE
:10672100E707C3E49DFDE49EFEEEB2E7F56F8D54ED
:106731002275380C12698B1269D6D553012275382E
:106741000C12695C1269CCD55301227538001269AB
:0E6751007412699BD553012275380012695CE1
:10675F0012699BD553012275380312698B126A0790
:10676F00D553012275380312695C1269FDD55301A7
:10677F002275380F126974126A2CD553012275389D
:10678F000F12695C126A2CD553262290679F2373D0
:10679F008091807780688059804A803B802C801D53
:1067AF00800E80DA80CB80BC80AD809E808F808011
:1067BF0075381512698B126A4ED55301227538152B
:1067CF0012695C126A43D553012275380912697434
:1067DF00126A14D553012275380912695C126A14B2
:1067EF00D553012275380612698B1269BED5530134
:1067FF002275380612695C1269B3D55301227538B8
:10680F00121269741269E4D5530122753812126994
:10681F005C1269E4D553012202673275381512698B
:10682F008B126A4ED553012275380F12695C126AAA
:10683F002CD553012275380F126974126A2CD55357
:10684F00012275380312695C1269FDD55301227557
:10685F00380312698B126A07D5530122753800125B
:10686F00695C12699BD55301227538001269741245
:10687F00699BD553262290688A2373809E80A980B6
:10688F00B480BF80CA80D580E08010801B802680B6
:10689F0031803C80478052805D806875380C12696A
:1068AF005C1269CCD553012275380C12698B1269B1
:0E68BF00D6D553012275381212695C1269E4B5
:1068CD00D55301227538121269741269E4D553013A
:1068DD002275380612695C1269B3D55301227538D9
:1068ED000612698B1269BED55301227538091269DA
:1068FD005C126A14D5530122753809126974126A33
:10690D0014D553012275381512695C126A43D5539B
:10691D00012202682A78C686040886037AED12538E
:10692D009A78CAA60408A60378C686040886037A50
:10693D006212539A78CCA60408A60378C68604087A
:10694D0086037AB512539A78C8A60408A603227551
:10695D001A6A751B0A78CA8618088619126B9F78F1
:10696D00CC86060886072278C88618088619E4F5AD
:10697D001AF51B126B9F78C886060886072278C603
:10698D008618088619751A00751B01026B9FE51D87
:10699D002519F51DE51C3518F51CC3E51F9FF51FC1
:1069AD00E51E9EF51E22C3E51F9FF51FE51E9EF5F4
:1069BD001EC3E51D9519F51DE51C9518F51C22E561
:1069CD001D2FF51DE51C3EF51CC3E51F9519F51F83
:1069DD00E51E9518F51E22C3E51D9FF51DE51C9EB0
:0969ED00F51CC3E51F9519F51F07
:1069F600E51E9518F51E22E51F2FF51FE51E3EF52F
:106A06001EE51D2519F51DE51C3518F51C22C3E5E7
:106A16001D9519F51DE51C9518F51CE51F2FF51F8D
:106A2600E51E3EF51E22E51D2FF51DE51C3EF51C57
:106A3600E51F2519F51FE51E3518F51E22C3E51DB0
:106A46009FF51DE51C9EF51CE51F2519F51FE51E86
:106A56003518F51E22E51A7009E51B70058C068DA2
:106A66000722ED851BF0A4A2F792D5ED851AF0A4B6
:106A7600AEF0FFEC851BF0A4A2D53FEE35F0FF92F9
:106A8600D5EC851AF0A42FFFE435F030D50104FECD
:106A960022E4F51AF51BEF4E7003051B22EF65196C
:106AA6007006EE65187001227808C3EF33FFEE33E7
:106AB600FEEF9519F5F0EE95184003FEAFF0E51AD6
:106AC60033F51AD8E5F4F51A751BFF7805C3EF33CD
:106AD600FFEE33FEEF9519F5F0EE95184003FEAF85
:036AE600F0E51BBD
:106AE90033F51BD8E5F4C403F51B22E51D9511E523
:106AF9001C9510500BE56E9511E56D95105001220E
:106B0900E51F9511E51E9510500BE5549511E56F9C
:106B19009510500122E51D9513E51C9512400BE5D2
:106B29006E9513E56D9512400122E51F9513E51E3B
:106B39009512400BE5549513E56F951240012253C8
:106B49002CF8C3E51F9554FFE51E956FFE92605022
:106B590007C3E49FFFE49EFEC3E56E951DF519E5A5
:106B69006D951CF5189261500BC3E49519F519E45C
:106B79009518F518C3E5199FE5189E9262500AE524
:106B890018CEF518E519CFF519126A97E52C5407AF
:106B990075F003A4F538E538906BA573026BBD0257
:106BA9006BD1026BDF026BF7026C0A026C1D026C7F
:106BB9002B026C43851C16851D17C3E4951FF5151B
:106BC900E4951EF514026C56851C16851D17851E45
:106BD90014851F158077C3E4951DF517E4951CF5F9
:106BE90016C3E4951FF515E4951EF514805FC3E4FB
:056BF900951DF517E4F5
:106BFE00951CF516851E14851F15804CC3E4951F34
:106C0E00F517E4951EF516851C14851D158039851E
:106C1E001E16851F17851C14851D15802BC3E49524
:106C2E001FF517E4951EF516C3E4951DF515E495AD
:106C3E001CF5148013851E16851F17C3E4951DF5CC
:106C4E0015E4951CF5148000C3E5179513E516950C
:106C5E001210D70122E5159513E514951210D701E0
:106C6E0022E519F92517FFE518F83516FED3EF952D
:106C7E0011EE9510500122E5119517FDE5109516B0
:106C8E00FC402A4D6027126A5BE5152FF515E514B9
:106C9E003EF514E5159513E514951210D70122E56E
:106CAE00199DF9E5189CF8851016851117E5172919
:106CBE00FFE51638FEE5139FE5129E500BC3E51354
:106CCE009517F9E5129516F8E51A700AE51B700688
:106CDE00AA00AB018013E9851AF0A4E5F0FBE88564
:106CEE001AF0A42BFBE435F0FAE5152BFBE5143A6C
:066CFE00FAE5119BE51010
:106D04009A10D70122EB9515FDEA9514FCC3E515FD
:106D14009511E514951010D717E5139BE5129A50B9
:106D240036E5139515FFE5129514FE126FD38027EF
:106D3400EB9511FFEA9510FEAA00C001126FD3D0A3
:106D440003E5172BFBE5163AFAEB99F517EA98F5E4
:106D540016851115851014C2D5E5466002D2D5AA50
:106D640056E98AF0A4ABF0E88AF0A42B30D5047578
:106D7400F00384F8700122E5172513FDE51635129A
:106D8400FCED8AF0A4ABF0EC8AF0A42B30D50475AA
:106D9400F00384FEE5152513FDE5143512FCED8A98
:106DA400F0A4ABF0EC8AF0A42B30D50475F0038486
:106DB400F9E538906DBB73026DD3026DDF026DE8A7
:106DC400026DF1026DF7026E03026E0A026E0FC3CA
:106DD400743E9EFFC3743E99FE8032C3743E9EFF90
:106DE400AE018029AF06C3743E99FE8020AF06AE83
:0D6DF40001801AC3743E9EFEC3743E99FFD9
:106E0100800EC3743E99FF8007C3743E9EFEAF019E
:106E110008EF2437FFE51B7007E51A700CE8800EB8
:106E2100A2E7E51A50030460F488F0A4E5F06001DC
:106E310004F923FA98FBC3E998C333F9906E43E54B
:106E41003873026E5B026E88026EBD026EEA026FDB
:106E510017026F44026F71026F9E05A7800BEB3022
:106E6100E7032A8002291E1FFBEEC45403F583EEBB
:106E71005408C42FF582EE5407243883F5F0E04519
:106E8100F0F0D8DA05A72205A7800BEB30E7032A3B
:106E91008002290E1FFBEEC45403F583EE5408C48F
:106EA1002FF582EE5407240B83F5F0E045F0F0D87E
:106EB100DA05A722804020100804020105A7800BF3
:106EC100EB30E7032A8002291E0FFBEEC45403F5C1
:106ED10083EE5408C42FF582EE540724EC83F5F0B9
:106EE100E045F0F0D8DA05A72205A7800BEB30E7E3
:056EF100032A800229C4
:106EF6000E0FFBEEC45403F583EE5408C42FF5823F
:106F0600EE540724BF83F5F0E045F0F0D8DA05A784
:106F16002205A7800BEB30E7032A8002291F1EFB00
:106F2600EEC45403F583EE5408C42FF582EE5407DD
:106F3600249283F5F0E045F0F0D8DA05A72205A7FC
:106F4600800BEB30E7032A8002291F0EFBEEC454A8
:106F560003F583EE5408C42FF582EE5407246583A7
:106F6600F5F0E045F0F0D8DA05A72205A7800BEB8F
:106F760030E7032A8002290F1EFBEEC45403F58373
:106F8600EE5408C42FF582EE5407243883F5F0E05A
:106F960045F0F0D8DA05A72205A7800BEB30E7030A
:106FA6002A8002290F0EFBEEC45403F583EE540823
:106FB600C42FF582EE5407240B83F5F0E045F0F07C
:106FC600D8DA05A7228040201008040201EC701FC1
:086FD600ED20E740D2E023CFDB
:106FDE0023CF30E7F980357B08801A7B1080167B33
:106FEE002080127B40800E20E4ED20E3EE20E2EFC5
:106FFE0020E1F07B80EE8BF0A4CF8BF0A4E5F02F98
:10700E00FFEC8BF0A4CD8BF0A4E5F02D2499838FAB
:10701E00F0A433E5F033FBE98BF0A4E5F0C88BF078
:10702E00A428F9E435F0F822FFFEFCFAF8F6F4F2A3
:10703E00F0EFEDEBEAE8E6E5E3E1E0DEDDDBDAD901
:10704E00D7D6D4D3D2D0CFCECCCBCAC9C7C6C5C45F
:10705E00C3C1C0BFBEBDBCBBBAB9B8B7B6B5B4B379
:10706E00B2B1B0AFAEADACABAAA9A8A8A7A6A5A465
:10707E00A3A3A2A1A09F9F9E9D9C9C9B9A99999829
:10708E009797969594949392929190908F8F8E8DD0
:10709E008D8C8C8B8A8A898988878786868585845C
:1070AE00848383828281818075A7009070DCE5469F
:1070BE00FA24FA50027A05EA2323F978107F049312
:1070CE00F60809E9DFF99070F4EA93F556227FC2CB
:1070DE00803E7F4680BA7E8C81747D1882E87A303D
:1070EE0085D074608BA08080402010081271000241
:1070FE007356D215D274D273C219C23A1256DC8E9E
:10710E0047757D0075460575520212914612022191
:10711E00E53524EB500E1291467F1990A11B127685
:10712E00F012DD59E55275F016A4F57012730C7558
:10713E007E151271D77F237E0990A0F61277021268
:10714E00DD5910000810010D10021280E212727F3C
:10715E0075330180DA1272C475330180D2757E00E8
:10716E001271D77E0090A10A1277357F237E05908B
:10717E00A0FE12770212722812DD59E55210000F8E
:10718E0010010510028780D5045403F55280CE12EB
:10719E0071D77F237E0B90A138127702E5466007E8
:1071AE001460041412411A12DD59E546100008103D
:1071BE00010B10021180D860D6154680D2B405029C
:1071CE0080CD054680C902711B75320012DF2F7FFC
:1071DE00017E1190A0E61277357E0012D5F0E57E85
:1071EE00D26612D64775170812DA7A12415975719E
:1071FE0000C20612D797741BFFF5177E0F90A13FA2
:10720E00305D0390A147127735129189125D0D12F0
:10721E0046BFC20612651C021E03E55260141460BE
:10722E001E1460297F647E2D791C1272721E1FD966
:10723E00F9227F6A7E1F79281272721FD9FA227F75
:10724E00487E2D791C1272720F1ED9F9227F567E3E
:10725E003379281F12DE740F0F12DE741F12DE74C4
:10726E001ED9F0221E12DE740E0E12DE741E02DE07
:10727E0074E552605514606814606D800075709EE0
:10728E001272F98003757000E5732540F573E435CD
:10729E0074F574E43575F575227570161272968054
:1072AE000375702DE5762542F576E5773541F57750
:1072BE00E43578F57822E55260CB1460DC1460E199
:1072CE0080007570441272B2800375705AE5739522
:0972DE0040F573E5749400F574A9
:1072E700E5759400F575227570711272DB80037570
:1072F7007088E5769542F576E5779541F577E578F7
:107307009400F57822E54690732293F540FEAD4749
:10731700E4FFFC12546F8E418F4222020C1830603A
:10732700C07F40120E9E121E1912DD591275D1EB45
:107337007005909E3D800B1273DF90A473500390ED
:10734700A4B97F3F7E0412770212DD5912DE3A128A
:10735700DE6A75370990A0A0121CFF90736673024E
:1073670002930275260270FA0276020273560273BE
:107377007E0273970273287F2E12168680D17F367E
:107387007E0490A44812770212DD5912DE3A80BFBC
:107397007F37120E9E121E1912DD591275B512484B
:1073A7004FD2AC1000A9306DFA12748F203BCF403A
:1073B700ED7568F97516001274DC40FB1276787F5C
:1073C700367E29E51612D3D012DD5905161277A895
:1073D70078C6B6F7E20275AF7C0512484F12DC7328
:1073E700744112DC84745312DC41EB12DC621277B5
:1073F700BA5003DCE5227515F975160010000EE585
:1074070015602512743140051274585002D3227F3B
:107417003F7E29E51612D3D012DD597F1412DE51B3
:107427000516E51664F870D4C322127D7075B9018C
:10743700E5BCB4811AE5BDF51570037516F778C676
:0B744700A616127EB9127EB1127EB1B3
:10745200C3027EB1D3227F0575F019D5E0FDD5F0C8
:10746200FA12484F12DC73744112DC84744212DC4B
:10747200417E0F78C6E60812DC41DEF912DC6512A5
:1074820077BA400122DF012275F00080CEC23B12A2
:10749200484FD2AC12DBCC204C3CB440F712DBD1CB
:1074A200B4400312DBD1B4412DF53812DBD1B45311
:1074B2002512DBD1FA12DBD1E538701A12DBD1B416
:1074C2000D1412DBD1B40A0EC3E5169A40030277FB
:1074D2009FC2ACD23B22C2ACD3221277FE12484FDB
:1074E200D2AC1000F112DBCC204CEBB440F412DB36
:1074F200D1B4400312DBD1B441DCF53812DBD1B494
:1075020042D47E1078C612DBD1F608DEF9E5387077
:10751200C512DBD1B40DBF12DBD1B40AB9C2ACC300
:10752200220273567F0A120E9E121E1912DD591282
:1075320075B5124868D2AC1000E712DBD1B440F541
:10754200F53812DBD1B46EED12DBD1E538600A12E8
:107552004868744F12DC4D80DC124868744012DCBB
:1075620084E51612DC4D12DC577568F975160012A7
:107572004868D2AC10003912DBD1B440F7F53812AA
:10758200DBD1B44EC07E1078C612DBD1F608DEF92C
:10759200124868E5386007744F12DC4D80D11276CC
:1075A200780516745112DC4D78C6B6F7C2127615FC
:0C75B200027356751500751603127D67F4
:1075BE0075B901E5BC30E70205160515E515242061
:1075CE0050EB227B007515F9127D7075B901E5BC83
:1075DE00B481010B0515E515240450EC7515011247
:1075EE007D6775B901E5BCB481010B0515E5152460
:1075FE002050EC227F1C120E9E121E5C400675154A
:10760E00F9127615027356E51560372404401A24D4
:10761E001E5019E515240740028027127D70127640
:10762E00510515E515240450F2751501127D677587
:10763E00B901E5BC30E7031276510515E515242096
:10764E0050EA22127666124EE605C6124EE605C6C0
:10765E00124EE605C6024EE674FF800574048001E4
:10766E00E4F5BCF5BDF5BEF5BF22E568606AF5151B
:10767E000515E5152404501D751501127D6775B9A4
:10768E0001E5BC30E70280190515E515242050EB05
:10769E00751500800C241C60F750E0E5152406508B
:1076AE0037E56875F004A485F0C7F5C675BC81E5AD
:1076BE0015F5BDF56878C6B6F70375BD00081276E8
:1076CE00DB1276D51276D586BC0886BD0886BE0836
:0976DE0086BF08124EE605C62223
:10C0A20012AEDE12C1A112828112C126128289123F
:10C0B200C13302AEE212AEDE12C1A11282817F5AF8
:10C0C200C23C12816312835F783F79437F607EEACC
:10C0D20012C1951282897F6512816312835F783D56
:10C0E20079417F207E4E12C195303C2012C35712F7
:10C0F200C1B2783F794312C111783D794112C11121
:10C1020012C35778D7E65480F675370002935BC3A3
:10C11200E796FF1819E796FE0809C3E69FF7181974
:10C12200E69EF7227F5B7E0690A54C1277351F8034
:10C132000A7F667E14745912D4E91F127FEC7E398D
:10C14200E402D5087866E620E73418C3E69472085C
:10C15200E694045029C318E6941F08E69404401E8E
:10C162007869E620E71818C3E6940E08E6940150B1
:10C172000DC318E6947508E694004002D322C32248
:10C18200E67D0030E7011D08E62BFB18E63CFCE4E7
:0EC192003DFD22C3EB9FF6F71819EC9EF6F761
:10C1A0002212C146400CE47842F608F67840F608C0
:10C1B000F6227864C3E6946AF55708E6944CF5567F
:10C1C0000808C3E69458F55B08E694AEF55A75394D
:10C1D00000AC56AD57EC12B28B784C12B319AC5A76
:10C1E000AD5BEC12B28B785012B3197F2B7E867D3B
:10C1F000777C1812B250785012B30D12B15C12B2A3
:10C2000050785012B30D12B15C12B250785012B384
:10C210000D12B15C12B2507F367E847D257C641293
:10C22000B250785012B30D12B15C12B250784C1269
:10C23000B30D12B15C12B2507F3F7EA27D607C8B49
:10C2400012B250785012B30D12B15C12AF4A12AF55
:10C250004A12B3257F3F7E807D057CE6053912B109
:10C260005C784812B3197F2C7E937D477C7F12B295
:10C2700050785012B30D12B15C12B250785012B314
:10C280000D12B15C12B250784C12B30D12B15C12A7
:10C29000B2507F357EB47DF87CDF12B250785012F8
:10C2A000B30D12B15C12B250785012B30D12B15CE2
:10C2B00012B2507F3F7EED7D227CCD12B250784C81
:10C2C00012B30D12B15C12AF4E12AF4A784412B3E2
:10C2D000197F317E397D9D7CE712B250784C12B3C4
:10C2E0000D12B15C12B250784C12B30D12B15C1247
:04C2F000B25078448C
:10C2F40012B30D12AF4E12B2507F2C7E377D0C7CE0
:10C30400A312B250784C12B30D12B15C12B2507831
:10C314004C12B30D12B15C12B250784C12B30D1220
:10C32400B15C12AF4E12B3257F3F7E807D027C9FAD
:10C33400053912B15C784412B319784812B30D125E
:10C34400B2C28E428F43784412B30D12B2C28E40F1
:10C354008F4122753900AC42AD43EC12B28B784860
:10C3640012B319AC40AD41EC12B28B784412B3193C
:10C374007F2B7E537D507C0912B250784812B30D46
:10C3840012B15C12B250784812B30D12B15C12B201
:10C3940050784412B30D12B15C12B2507F347EF265
:10C3A4007DCD7CA312B250784812B30D12B15C1249
:10C3B400B250784812B30D12B15C12B2507F3F7E76
:10C3C4000A7D2E7CAE12B250784412B30D12B15CC9
:10C3D40012AF4A12AF4A784C12B3197F2B7E4F7DAD
:10C3E400AF7CB212B250784812B30D12B15C12B2E3
:10C3F40050784812B30D12B15C12B250784812B39F
:10C404000D12B15C12B2507F357EB17D4B7C95121A
:10C41400B250784812B30D12B15C12B25078441283
:10C42400B30D12B15C12B2507F3F7E497DCD7C4585
:10C4340012B250784812B30D12B15C12AF4E12AF63
:10C444004A785012B319784C12B30D12B2C28D55FA
:10C454008E568F57785012B30D12B2C28D598E5A20
:04C464008F5B78640E
:10C46800E557246AF608E556344CF608E5553404D1
:10C47800F608E55B2458F608E55A34AEF608E435C4
:03C4880059F62240
:1091A90012AEDE12983A12AEE27F6690A52E1277C1
:1091B900331292177F5A78C41291F31291FB78C631
:1091C9001291F31291DE7F6578C81291F31291FB27
:1091D90078CA1291F37E2DE51B12D5087E33E51A64
:1091E90012D5087E39E51902D508860408860302D6
:1091F90053397E15E51C12D5087E1BE51B12D508CF
:109209007E21E51A12D5087E27E51902D5087F5A6D
:109219007E01E53A12D41E7E0B909C2EE53B93020B
:10922900D51BE6FF08E6FE08E6FD339217E4500178
:10923900F4FC12B33675130A75390112B53478D7AF
:10924900E6C2E775F00A84F9303D02A9F012B33697
:109259008913053912B50D30170A053912B52005DC
:109269003912B520A80302B31912AEDE12983AC218
:109279003C7F5A7E0312851012921712DD59100095
:109289000810011510022080EFE53A146004153A20
:109299008003753A3CD23C80DFE53AB43C05753A27
:1092A9000180F2053A80EE7E0312850B7E0B128552
:1092B9001012921712DD5910000810011510022022
:1092C90080EFE53BB40205753B158002153BD23CA6
:1092D90080DFE53BB41505753B0280F2053B80EE66
:1092E9007E0B12850B7F5A78C41291F31291FB12EF
:0792F900936412836F78C437
:109300001293BC78C61291F31291DE129396751CDB
:109310000012836F78C61293BC7F6578C81291F3F0
:109320001291FB12936412836F78C81293BC78CAAF
:109330001291F31291DE129396751C0012836F78CE
:10934000CA1293BC303C14E53B24F4500B78C9E6B8
:109350002410F618E63427F61293C212AEE2127EFB
:10936000F102DD59C2247E15E51C128460F51CD281
:10937000247E1BE51B128460F51B1023E77E21E58C
:109380001A128460F51A1023E67E27E5191284600C
:10939000F5191023E822C2247E2DE51B128460F506
:1093A0001BD2247E33E51A128460F51A1023E77E5F
:1093B00039E519128460F5191023E622ECF608EB62
:1093C000F622129C4678C8E6FE0886073395E0FD33
:1093D000FC12B2507FE87E037D007C0012B534128F
:1093E000B25078CAE6FE0886073395E0FDFC12B558
:1093F0000D12B2507F807E697D677CFF12B50DEC47
:1094000012B28712B2507F3F7E807D0D7C1D12B15B
:109410005C12B2507F3D7E407D007C0012B25078DD
:10942000BC12B30D12B15C12B2507F3E7E807D0043
:109430007C0012AF4E12B25078BC12B30D12B15C68
:0994400012B2507F3F7E807D00D6
:109449007C0012AF4A12B25078B412B30D12B15C5B
:1094590012B1D4783C12B3197F407E807D007C0024
:1094690012B250783C12B30D12B15C12B3B312B2FE
:10947900507F3F7EA87D007C0012B25078B812B3AD
:109489000D12B15C12B15C12B2507F407E007D00BA
:109499007C0012B250783C12B30D12B15C12B3B316
:1094A90012B2507F3F7EC07D007C0012B15C12AFCA
:1094B9004E12B25078B812B30D12B15C12B2507894
:1094C9003C12B30D12AF4E785412B31912B39D78F2
:1094D9005812B31912B25012B15C12B25078C012BC
:1094E900B30D12B15C784412B319785412B30D124A
:1094F900B3B3783C12B31912B25012B15C12B25024
:1095090078BC12B30D12B15C783C12B3197F3E7E60
:10951900C07D007C0012B250783C12B30D12B15CD0
:1095290012B2507F3F7E007D007C0012AF4E12B216
:1095390050783C12B30D12B15C12B2507F3F7E805D
:109549007D007C0012AF4E12B25078B412B30D12E6
:10955900B15C787012B31978C4E6FE0886073395B2
:10956900E0FDFC12B2507FE87E037D007C0012B55D
:109579003412B25078C6E6FE0886073395E0FDFC42
:1095890012B50D12B2507FE07E5E7DF87CFF12B5F8
:109599000DEC12B28712B2507F3F7E7F7DE57CC908
:0595A90012B2507870C1
:1095AE0012B30D12B15C12B1D4785012B3197F3FC1
:1095BE007EF07D007C0012B250783C12B30D12B1D9
:1095CE005C12B2507F3F7EC07D007C0012AF4E1207
:1095DE00B250783C12B30D12B15C12B2507F3F7E86
:1095EE00807D007C0012AF4E783C12B31978BC120D
:1095FE00B30D12B2507F3F7E807D007C0012AF4AC9
:10960E0012B250783C12B30D12B25078B412B30DA0
:10961E0012B15C12B15C784012B319785412B30DCA
:10962E0012B3EB783C12B31912B25012B15C7874CB
:10963E0012B3197F417E107D007C0012B25078C0AB
:10964E0012B30D12B15C12B2507F407E807D007C51
:10965E000012B250784412B30D12B15C12B2507FA8
:10966E00417E207D007C0012AF4A12B25078441227
:10967E00B30D12B15C12B2507F407E407D007C0073
:10968E0012B250787412B30D12B15C12B2507F4008
:10969E007EA07D007C0012AF4E12AF4E12AF4A126A
:1096AE00B250785012B30D12B15C12B25078501203
:1096BE00B30D12B15C12B2507F3D7E2A7DAA7CABF7
:1096CE0012B15C12B2507F3F7E007D007C0012AF63
:1096DE004A12B250783C12B30D12B250787012B3D7
:1096EE000D12B15C12B250784012B30D12B1D412F9
:1096FE00B250785012B30D12B15C12B250785012B3
:10970E00B30D12B15C12B15C12B250785412B30D9B
:0C971E0012AF4A12B2507F4A7E517DD239
:10972A007CCB12B15C12B2C278AC12B3197F407E04
:10973A00007D007C0012B250787412B30D12B15C35
:10974A0012B2507F3F7E807D007C0012AF4E12B273
:10975A0050784412B30D12AF4E12B250785012B371
:10976A000D12B15C12B250785012B30D12B15C12E4
:10977A00B250785012B30D12B15C12B2507F3E7ED5
:10978A002A7DAA7CAB12B15C12B250785012B30D8A
:10979A0012AF4A12B250785812B30D12B1D412B2A3
:1097AA00507F4A7E517DD27CCB12B15C12B2C2127A
:1097BA00B250AF3AEF3395E0FEFDFC12B2507F4053
:1097CA007E7E7D057C0012B53412B2507F607E75B4
:1097DA007D587CFF12B50D12B50D78B012B3197809
:1097EA00AC751B641298118F1C78B0751B671298A0
:1097FA0011E51C75F00AA42FFF249C50027F007803
:10980A00D7E654802FF62275390012B30D12B250E2
:10981A007F0A7E007D007C0012B5E0A81BE513F6E6
:10982A0008E512F608E511F6335004EFF404FF22B6
:10983A00C23D78647BAC12922BD23D78677BB01222
:10984A00922B129C467F007EE47D577C0012B25018
:10985A0078AC12B30D12B50D12B2507F007E537D53
:0E986A00077C0012B5E012B26F85133B7F80C1
:109878007ECB7DA47C0012B25078B012B30D12B525
:109888000D12B2507F407E7E7D057C0012B5E0123D
:10989800B26FE513F56F04F53A85126E85116D8583
:1098A800106C7F407E7E7D057C0012B250786C1271
:1098B800B30D12B53412B2507F607E0C7DA27C00CD
:1098C80012B25078B012B30D12B50D12B520786CE3
:1098D80012B31978AC12B30DEC12B28712B2507FE2
:1098E800347E9C7D2B7C5F12B15C785412B31912C4
:1098F800B39D785012B319786C12B30DEC12B2877D
:1099080012B2507F347E9C7D2B7C5F12B15C12B208
:1099180050785012B30D12B15C784012B3197F40E1
:109928007E007D007C0012B250785412B30D12B143
:109938005C12B3B312B2507F3D7EC07D007C001232
:10994800B25078BC12B30D12B15C12B2507F3E7E99
:10995800C07D007C0012AF4E12B25078BC12B30D1D
:1099680012B15C12B15C12B2507F3D7E407D007C2A
:109978000012B25078BC12B30D12B15C12B2507F13
:109988003E7E807D007C0012AF4E12B25078BC1231
:10999800B30D12B15C12B2507F3F7E807D007C0017
:1099A80012AF4A12B250785412B30D12B15C12AF12
:1099B8004A12B2507F407E807D007C0012B25078FF
:1099C8005412B30D12B15C12B3B312B2507F3D7E84
:1099D800707D007C0012B25078BC12B30D12B15CDD
:1099E80012B25078BC12B30D12B15C12B15C12AF56
:1099F8004E12B25078B412B30D12B15C785812B34B
:109A080019785412B30D12B3B3783C12B3197854C1
:109A180012B30D12B3EB785412B319783C12B30D8C
:109A280012B25012B15C12B25078BC12B30D12B11E
:109A38005C783C12B3197F3E7EC07D007C0012B278
:109A480050783C12B30D12B15C12B2507F3F7E00C9
:109A58007D007C0012AF4E12B250783C12B30D124A
:109A6800B15C12B2507F3F7E807D007C0012AF4E09
:109A780012B25078B412B30D12B15C787012B319E7
:109A8800785012B30D12B25012B15C12B25078C0B5
:109A980012B30D12B15C784412B319785412B30D95
:109AA80012B25012B15C787412B319784012B30D27
:109AB80012B25012B15C783C12B3197F407E807D9F
:109AC800007C0012B250784412B30D12B15C12B28D
:109AD800507F417E107D007C0012AF4E12B250784C
:109AE8004412B30D12B15C12B250787412B30D1255
:109AF800B2507F407EA07D007C0012AF4A12AF4E6C
:109B080012B250783C12B30D12B15C12B2507F3DC4
:109B18007E2A7DAA7CAB12B15C12B2507F3F7E00D8
:109B28007D007C0012AF4E12B250785412B30D1261
:109B3800B250787012B30D12B15C12B250783C1268
:109B4800B30D12B15C12B15C12B250785812B30D59
:109B580012AF4E12B2507F3F7E7F7DE57CC912B1B5
:019B68005CA0
:109B690012B2507F4B7E187D967C8012AF4E12B296
:109B7900C212B2507FE87E037D007C0012B5E0126C
:109B8900B26F78C8A61208A61308A60608A6077811
:109B99007412B30D12B2507F3F7E807D007C00129B
:109BA900AF4A12B250784412B30D12AF4E12B250EE
:109BB9007F3E7E2A7DAA7CAB12B15C12B2507840FE
:109BC90012B30D12B15C12B250783C12B30D12B13E
:109BD9005C12B250784012B30D12AF4E12B2507FE0
:109BE9003F7E7F7DE57CC912B250787012B30D12A9
:109BF900B15C12B15C12B2507F487EF47D247C00C6
:109C090012AF4E12B2C212B2507FE87E037D007CC1
:109C19000012B5E012B26F78C4A61208A61308A6FE
:109C29000608A607223F3F4344454647484A4B4C4E
:109C39004D4E5051525354555657583F3FE4F539FC
:109C4900F5A7909C5A791078B4E493F6A308D9F94A
:109C59002232A5C24A4A19DC3A885CDB3BFFD6DCD2
:019C69003BBF
:10AEDE00D2D58002C2D575A70490040078107F0BDE
:10AEEE0012AF0A78267F0512AF0A783C7F2212AF86
:10AEFE000A786A7F0F12AF0A75A7002230D506E6D0
:10AF0E00F008DFFB22E0F608DFFB22D2D58002C27A
:10AF1E00D575A7049006FA78737F0612AF0A75A747
:10AF2E000022DA0CD902800BD906303701B3500556
:10AF3E0002B0BD923702B0A9D9F680F9D23680029E
:10AF4E00C23612B0EE303606C86002B237C892363C
:10AF5E00DAD0D9E4B8000A12B135A236923702B06F
:10AF6E009260FBB51300400F12B135A23692F7A2D4
:10AF7E00379236A2F79237C398F40424E740DF24C1
:10AF8E0019AD29AC28AB277A00C394084008CDCC64
:10AF9E00CBCAE4CD80F424086010F9C3ED13FDECA8
:10AFAE0013FCEB13FBEA13FAD9F1A236303701B3D7
:10AFBE0040308A17E5102BF518E5113CF519E5120E
:10AFCE003DF51A501A13F51AE51913F519E518136C
:10AFDE00F518E51713F5170513E51370020514029E
:03AFEE00B048E484
:10AFF100C39AF517E5109BF518E5119CF519E512B3
:10B001009DF51A500DB237C378177F04E496F60800
:10B01100DFFA7A047019E513C39408F51350021589
:10B0210014E4C517C518C519F51ADAE802B0E92004
:10B03100E7BAE5137002151415137817C37F04E6F8
:10B0410033F608DFFA80E8E51A20E7137817C37FA3
:10B0510004E633F608DFFAE513700215141513E55B
:10B06100173378187F03E63400F6500E08DFF775C2
:10B071001A800513E51370020514E51420E75470D6
:10B0810027E513604E046020851A12851911851871
:10B09100105326F0AC10AD11A237E51313FFE512E2
:10B0A10092E7FEA81302B26FE4F512F511F510F55F
:10B0B100147513FF5326F043260580D8E5FFF512DA
:10B0C100F511F510751400F513D2375326F0432608
:10B0D1000980C15326F0432603E4F512F511F5105A
:10B0E100F514F513C23780AC5326F080EC79017A60
:10B0F100018512F0E513A2F7339237751400F513A9
:10B101006002D2F785F012A813B8FF0809E512C250
:01B11100E756
:10B112006001098C278D288EF0A2F7EF3304700AA4
:10B122000AC2F705F00AD5F0011A146002D2F785B7
:10B13200F02922C88813C512C529C512C511C52810
:10B14200C511C510C527C51022DA03B8000302B025
:10B15200BDD9028002D9F702B0A912B0EE30370190
:10B16200B392377004D9E78005DADEB8000302B083
:10B17200E9D9E2C3947E500215142513F513500247
:10B1820005147815760008B81BFA78277915E608B1
:10B19200FAE8FC78108AF0E608A427F709E5F03708
:10B1A200F7500989F00907E760FBA9F0B813E6191F
:10B1B20019ECF8B82AD802B04802B0D4B8FFFA02A3
:10B1C200B0BDD9FB02B0A9DAF6B800F002B0E912BC
:10B1D200B32512B0EE303701B392377007D9E3B816
:10B1E20000E280DBDAE1B8000280E1D9D5C8C39879
:10B1F20050021514247F50020514F513781A7600B4
:10B202007A1A7B80C3E5109527E5119528E51295FA
:10B21200294016C3E5109527F510E5119528F5117B
:09B22200E5129529F512E64BF640
:10B22B00DA0302B048EB03FB30E703187600C3E503
:10B23B001033F510E51133F511E51233F51240CA51
:10B24B0030E7DD80B6E53905396010D0F0D0E0C0CD
:10B25B0010C011C012C013C0E0C0F08F138E128D3E
:10B26B00118C1022E539146010D0F0D0E0D013D03F
:10B27B0012D011D010C0E0C0F01539227920800C0B
:10B28B007910800479087D007E007F003392D550C1
:10B29B000312B2FFEC33400FEF33FFEE33FEED330F
:10B2AB00FDEC33FCD9EE22EECCF5F0747E29A2D561
:10B2BB0013FF92F7AEF022EF8EF0A2F7D2F7339294
:10B2CB00D5C3947F5006E4FFFEFDFC22942040047E
:10B2DB0074FF80F304CCFEE4FFFAE5F0CC6012C3FC
:10B2EB00CC13CCCD13CDCE13CECF13CF0450EEDA7F
:10B2FB00EC30D5D7C3E49FFFE49EFEE49DFDE49CB8
:03B30B00FC22E63B
:10B30E00FC08E6FD08E6FE08E6FF22ECF608EDF680
:10B31E0008EEF608EFF622CFC513CFCEC512CECD6E
:10B32E00C511CDCCC510CC22E4F513F512F511F5EF
:10B33E001022E493FCA3E493FDA3E493FEA3E49311
:10B34E00FFA322C0E012B25012B15C12B38412B34A
:10B35E0040D0E0C0E012B25012B37B12B15C12B218
:10B36E005012B34012AF4ED0E0D5E0E722AC48AD5C
:10B37E0049AE4AAF4B228C488D498E4A8F4B227470
:10B38E00FF7809FFFEFDFCE52654F048F526221253
:10B39E00B44404A2E1927F1420E01590B4C5740465
:10B3AE0012B351802912B44430E102B27F20E0EB97
:10B3BE008C4C8D4D8E4E8F4F90B4D9740412B35168
:10B3CE0012B250AC4CAD4DAE4EAF4F12B15C307FA1
:10B3DE0004EF6480FFEE33EF337001FF2212B444AA
:10B3EE00C0E08C4C8D4D8E4E8F4F90B4FD74031279
:10B3FE00B35112B250AC4CAD4DAE4EAF4F12B15C1C
:01B40E00EC51
:10B40F00C54CFCEDC54DFDEEC54EFEEFC54FFF9093
:10B41F00B4ED740312B351D08212B250AC4CAD4D97
:10B42F00AE4EAF4FE58230E00712B1D4B27F809DB0
:10B43F0012B1D18098EE33EF3324605007D0E0D0B3
:10B44F00E002B38DEFA2E7547F927FFF12B2507CE0
:10B45F00837DF97E227F3E12B15CEE33EF33248180
:10B46F00501012B25012B2C212B287EFB2E7FF12EF
:10B47F00AF4EEE33EF33602A2403F8C313FFEE927F
:10B48F00E7FEE82481E4501A12B25012B2C2EF0460
:10B49F00C2E0FCF58212B28FEFB2E7FF12AF4EE5BA
:10B4AF008203FAEE33EF33600B148FF0A2F713FF22
:10B4BF00EE92E7FEEA2283FA703AE4E9AABCF8E0DA
:10B4CF00813EE6E99DBF0000803F1A3C283966693E
:10B4DF0099BBE335A33DE75D25BFDB0FC93FCCDB50
:10B4EF008D41EE3649C43F91C9453DF8B0C50000C6
:10B4FF00803F34F517C373FA2F45DDFD0AC6EF25DC
:10B50F0013FFEE3512FEED3511FDEC3510FC02B2D6
:10B51F006FC3EF9513FFEE9512FEED9511FDEC95B0
:10B52F0010FC02B26FEFF88513F0A4FFE513C5F01E
:0AB53F00CEF9A42EFEE435F0CDFA9B
:10B5490088F0E512A42EFEED35F0FDE433CC851329
:10B55900F0A42CFCE5128AF0A42CFCE51189F0A4D6
:10B569002CFCE51088F0A42CFC89F0E512A42DFD33
:10B57900EC35F0FCE51188F0A42DFDEC35F0FC8AE2
:10B58900F0E513A42DFDEC35F0FC02B26FE4CCF824
:10B59900E4CDF9E4CEFAE4CFFB75F020C3E513332B
:10B5A900F513E51233F512E51133F511E51033F50D
:10B5B90010EF33FFEE33FEED33FDEC33FCEF9BEE82
:10B5C9009AED99EC98400CFCEF9BFFEE9AFEED99F1
:10B5D900FD0513D5F0C622C2D5EC30E705B2D51268
:10B5E900B2FFE51030E70DB2D512B60312B59612C7
:10B5F900B2FF800312B59630D515C3E49513F51340
:10B60900E49512F512E49511F511E49510F510225F
:10A6C300E57124885002D2191256DC8E4712D22E1D
:10A6D300129189125A98305E0F125A3612887812E4
:10A6E300596712C03412425412393A1247FB1036DA
:10A6F30029201F1C301219E412A84912A85E12A9BE
:10A703005E12A98030510302AA0A12ACDB20510960
:10A71300C251E4F552F545F5442275A70075830748
:10A72300E559C454F0F582E0F538A3E0F518A3A386
:10A73300A3E0F51E74FF12A8491256DC8E1C8F1B72
:10A743007510DF751100E51164B4700612A8147555
:10A75300111012A7E14028AE1CAF1B125764203220
:10A763001EAC03AB027A0C125371ED701275A70085
:10A77300758304851182ECF00583E510F00511D58E
:10A7830010C412A81475C70375C6E075A704900515
:10A79300007F0412A7CFDFFB75A700122B83125A89
:10A7A30036E4F5A7F8F559758307E8C4F582E06543
:10A7B300387011A3E06518700BA3A3A3E0651E70A6
:10A7C3000388592208C3E5589850DC22E0F5BCE021
:10A7D300F5BDE0F5BEE0F5BF124EE605C622E51075
:10A7E30075F004A4F5C685F0C775B901E5BC33401F
:0BA7F3001F05C605C675B90185BE64D0
:10A7FE0085BF6505C675B90185BC6685BD6785BE15
:10A80E006885BF69C322E51124FE502E75A7007F0F
:10A81E0010AE111E7583048E82E0FD1582E0CDB55B
:10A82E0005005012F00582CDF00583E0FD1582E0A3
:10A83E00CDF00582CDF0DEDCDFD72275A754900473
:10A84E000005A79005007FB4F0F0DFFC75A700228D
:10A85E0012BE88C2517B077AFFE4FFF5A790040071
:10A86E0012A944ED244C4035EC603075A7008D8262
:10A87E0005A712A90A7583058D82E02410401CF0ED
:10A88E0005A7E02CF0500505A7E004F0BA000CBBBC
:10A89E000009D251EF24DC50027F23DFC3EA6005AA
:10A8AE0012A8BD8006EB600312A8F575A700223032
:10A8BE00E0047553082230E1047553182230E20487
:10A8CE007553282230E3047553382230E40475534F
:10A8DE00482230E5047553582230E6047553682239
:10A8EE0030E7037553782230E0047553882230E147
:10A8FE00047553982230E2037553AA22ED54F0C426
:10A90E00232390A914735302FE225302FD225302F5
:06A91E00FB225302F722A8
:10A924005302EF225302DF225302BF2253027F223B
:10A934005303FE225303FD225303FB225303FB2242
:10A9440012BDC012BC4EE4F5F7C2B2C2B2ADF7F507
:10A95400F7C2B2C2B2ACF7D2B22290050078B4E02A
:10A964006015FD54F0C4CD7C00540FFE1583E0FF48
:10A9740012546FEFF005830582D8E42275830478BE
:10A98400FF088882E060FAF5D38812E512244C505F
:10A99400012285D3D288D4881279FF0512E512608A
:10A9A400F00908E875F0B484A8F08882E060ECF55A
:10A9B400D3B9000280D5B9230050D0C395D292D127
:10A9C4005002F40409FEE4FFFCAD0112547C74014E
:10A9D400FA25D475F0B484A8F0AC06AB071253631F
:10A9E400EB30E7010CE5D22C30D1029C9C8882F03C
:10A9F4000AEAB501DCE512244C50012285D3D28544
:10AA040012D4A812809390040012AAC98C068B0554
:10AA140012AAC9E4FFF512F5118C148B13C3ED9B34
:0EAA2400F9EE9CFA4012E51199E5129A500ADB
:10AA32008C148B138A1289118F528F82E0F9C3ED25
:10AA420099FDEE9400FEE582245A5002244C75F0E2
:10AA5200B48485F082E0FA2DFDEE3400FEEB9AFB21
:10AA6200EC9400FCE92BFBEC3400FC0FBFB4B0E526
:10AA72005224D3400224B4F552C3E51333FBE51448
:10AA820033FCE511FE2BFBE512FF3CFC1254D1E92D
:10AA9200F890AADB93F511FDEBF513FFECF514FE2C
:10AAA2007C0012546F8F44E890ABDB93FAAB13AC8B
:10AAB2001412539AAF03AE04AD117C0012546FEF1F
:10AAC2007002F552F545227C007B007F5AE02BFB99
:10AAD200EC3400FC0582DFF522B4B4B4B4B4B4B4EF
:10AAE200B4B4B4B4B4B4B4B4B4B4B4B3B3B3B3B329
:10AAF200B3B3B3B3B3B3B3B3B2B2B2B2B2B2B2B22C
:10AB0200B2B1B1B1B1B1B1B1B0B0B0B0B0B0B0AF3B
:10AB1200AFAFAFAFAEAEAEAEAEAEADADADADADAC56
:10AB2200ACACACACABABABABAAAAAAAAA9A9A9A97B
:10AB3200A9A8A8A8A8A7A7A7A7A6A6A6A5A5A5A5A8
:10AB4200A4A4A4A4A3A3A3A2A2A2A2A1A1A1A0A0DF
:10AB5200A0A09F9F9F9E9E9E9D9D9D9D9C9C9C9B19
:10AB62009B9B9A9A9A999999999898989797979658
:10AB7200969695959594949493939392929291919B
:10AB820091919090908F8F8F8E8E8E8D8D8D8C8CDB
:10AB92008C8B8B8B8A8A8A89898988888887878720
:10ABA2008686868585858484848383838282828166
:10ABB20081818080807F7F7F7E7E7E7E7D7D7D7CA9
:10ABC2007C7C7B7B7B7A7A7A7979797878787777EB
:10ABD2007776767675757574740002030506080932
:10ABE2000B0C0E101113141617191A1C1D1F2122FB
:10ABF200242527282A2B2D2E303133343637393A63
:10AC02003C3D3F404243454648494B4C4E4F5052D3
:10AC120053555658595A5C5D5F6061636466676854
:10AC22006A6B6C6E6F707273747677787A7B7C7EE7
:10AC32007F80818384858688898A8B8D8E8F90918F
:10AC4200929495969798999B9C9D9E9FA0A1A2A451
:10AC5200A5A6A7A8A9AAABACADAEAFB0B1B2B3B42A
:10AC6200B5B6B7B8B9BABBBCBDBEBFC0C0C1C2C31E
:10AC7200C4C5C6C7C7C8C9CACBCCCCCDCECFD0D02D
:10AC8200D1D2D3D4D4D5D6D7D7D8D9DADADBDCDC53
:10AC9200DDDEDEDFE0E0E1E2E2E3E4E4E5E5E6E793
:10ACA200E7E8E8E9EAEAEBEBECECEDEEEEEFEFF0E9
:10ACB200F0F1F1F2F2F3F3F4F4F4F5F5F6F6F7F756
:10ACC200F8F8F8F9F9FAFAFAFBFBFBFCFCFDFDFDDA
:10ACD200FEFEFEFEFFFFFFFFFFC251E4F544F81443
:10ACE200FB900400A9007C0FC2D112ADF6E8240546
:10ACF200F8B8B4F08B13E5122403FA244C5001FA8D
:10AD0200BBFF012275112C8A1912AE2D8F16203D20
:10AD120012AA1975112312AE2D8F15751600303D2A
:10AD2200E2801175112312ADD5751500303D05E88D
:01AD32002FF1
:10AD330013F51575111212ADD5751400303D05E8E4
:10AD43002F13F514EA2404F552244C5002F552E46F
:10AD5300F51AF51BF51CE516600AFB7A00AF137EA6
:10AD6300FF12AD9BE515600AFB7A4FAF137EFF120E
:10AD7300AD9BE516600DFB7A00E5146006FF7ECF00
:10AD830012AD9BAE1CAF1B7C00AD1A12546F8F45E6
:10AD9300EF2513F544D25122EFF5F0A4FCADF0EB0F
:10ADA300F5F0A49CFCE5F09DFDEB8AF0A4FAABF072
:10ADB300EF8EF0A49AF8E5F09BF9E833F8E933F95C
:10ADC3007B00125515051AE51B2BF51BE4351CF505
:10ADD3001C22EA2511F9244C5001F9C2D112ADF419
:10ADE300303D428F00C3EA9511F9500324B4F9D2E0
:10ADF300D17C09E4FDFEFF8982E060062FFFE43E7B
:10AE0300FE0D09B9B4027900DCEDED20D118F51E71
:10AE130024FE923D500F12547CEFB503005006857B
:10AE23001E1FFB881222F51D80E612ADD5203D437F
:10AE3300740212AECC12ADD5203D38740412AED4D8
:10AE430012ADD5203D2D740612AECC12ADD5203DEA
:10AE530022740812AED412ADD5203D17740A12AE77
:10AE6300CC12ADD5203D0C740C12AED412ADD5204E
:10AE73003D0122C3E89F605088148F158A1640084D
:10AE83001ABAFF0A7AB380060ABAB4027A0012AD7C
:10AE9300D5303D34C3E89FF9602EC3E5149515FB07
:10AEA3006930E7D4E930E703F404F9EB30E702F45F
:10AEB30004C3995002AA16E5142515C82F28FFE4E8
:10AEC300FC33FE7D0412546F222AFA244C5001FAFB
:0BAED30022C3CA9AFA500324B4FA22EA
:10BC1500758000C2B212DE4FD2B275F8302275803F
:10BC250000C2B2F5F7C2B2C2B2D2B222758000C26A
:10BC3500B2F5F7C2B2C2B2856CF7C2B2C2B2856BB9
:10BC4500F7C2B2C2B2856AF722758000C2B275F733
:10BC550003C2B2C2B2856FF7C2B2C2B2856EF7C275
:10BC6500B2C2B2856DF72212BCA5740612BC23744C
:10BC75000212BC318FF7C2B2C2B2D2B222909F7209
:10BC85007F631276F012DD59D214120E9412766E7D
:10BC9500124EE612BCA5740612BC2374C712BC234F
:10BCA50012BCAB40FB22758000C2B275F705C2B26B
:10BCB500C2B2C2B2C2B275F705C2B2C2B2C2B2C294
:10BCC500B2E5F7D2B2A2E022120E9485BF6C85BE12
:10BCD5006B756A00E56B7015E56A701112BCA57489
:10BCE5000612BC2374D812BC31D2B2D21F22E54B46
:10BCF5000475F03C8485F04B12BFB0852E72E55F6C
:10BD0500030354C0F8E55E543F28F57C3055012205
:10BD150012BD4A12BCAB40F7E54C60F312BCA5124C
:10BD2500BD6112BD2F80F112BCA5C21F740612BCE5
:10BD350023740212BC31787086F708B880FAD2B243
:10BD450012BD7E808F787075A704758304E54CC499
:0CBD5500F5827F10E6F0DFFC054C801941
:10BD6100787075A704758304154CE54C30E701E440
:10BD7100C4F5827F10E0F6DFFC75A7002274102560
:10BD81006A54F0F56AE4356BF56BE4356C540FF5E4
:10BD91006C22E54B75F010A4256A54F0F56AE5F0C4
:10BDA10080E4E56A24F054F0F56AE56B34FFF56B45
:10BDB100E56C34FF80D7E56A24FF80ECC380EBE5B6
:10BDC1006D24F054F0F56DE56E34FFF56EE56F34DA
:10BDD100FF540FF56F2212BE2F12BE57C22DC2544F
:10BDE100C255E57F7002D255147002D254E54A3033
:10BDF100E00122B4061C20540D12BDA312BEFF1295
:10BE0100BF8F12BFC72212852F7E0412DE47754AEB
:10BE1100012220550D12BD7E12BF6E12BFB012BE9F
:10BE2100D82212852F7E0412DE47754A052274033B
:10BE310012BC317870E4F5F7C2B2C2B2A6F708B805
:10BE410080F3D2B222740312BC31E4F5F7C2B2C25C
:10BE5100B2E5F7D2B222E575F8541F30E40244E0AE
:10BE6100F57585722EA2779226E57C543F30E50266
:10BE710044C0F55EE57C54C02323F55FE57FC2E74E
:10BE810079BCF709A77E22856C6F856B6E856A6D1B
:01BE9100228E
:10BE9200856F6C856E6B856D6A22E4FEFF74077593
:10BEA200A704F5838E8274FFF0DFFD75A70022746C
:10BEB200067E007FB012BEA1E4F55AF55B2275A79B
:10BEC20004758306E55A600A75F00A84E5F070028B
:10BED200740AC4F58222307720E55A240240020512
:10BEE2005A12BEC0E55AF0E573F0E574F0E575F05C
:10BEF200E576F0E577F0E578F075A700223077F97E
:10BF020012BEC07F1074FFF0DFFDE55A24F5500326
:10BF120012BF2A155AE55AB4FF02055AC3E55A95CB
:10BF22005B50D6755B0080D112BE887F0A056D0515
:10BF32006D12BC4EE4F5F7C2B2C2B2E5F7D2B2302E
:10BF4200E704DF02800512BDC080E2056D12BC4E1F
:10BF520012BEC0E55A24F6F07F06E4F5F7C2B2C27B
:10BF6200B2E5F7F0DFF4D2B275A70022053FE53F54
:10BF7200B43C17753F00053EE53EB43C0D753E00EE
:10BF8200053DE53DB41803753D00024ABB153FE58A
:10BF92003FB4FF17753F3B153EE53EB4FF0D753EBE
:10BFA2003B153DE53DB4FF03753D17024ABB054213
:10BFB200E542B43C0F7542000541E541B43C0575CC
:0CBFC20041000540221542E542B4FF0F8B
:10BFCE0075423B1541E541B4FF0575413B154022D5
:10BFDE00AC40AB41A842EC75F03CA42BFBE435F031
:10BFEE00FC7A3C125363EB28FBE43CFC22AC3DABE9
:10BFFE003EA83F80E178AE8604AB3EE53FC313F822
:10C00E00800C7800120E5DE5BE75F005A4FBE5BF51
:10C01E0075F03CA42BFBE435F0FC7A1E125363EB57
:10C02E0028FBE43CFC2212C010AE04AD0312C00388
:10C03E008C148B13120E67E5BFFF24F650027F019E
:10C04E00E5BE75F096A4AAF0F9C3ED9513FBEE9537
:10C05E0014FC924E4B701120110E30480B75364B5E
:10C06E003003037536FFD22E304E02DF1F7A0212D6
:10C07E00536375A7009004EEECF0A3EBF0C3E5BF9D
:10C08E009F04BF0102D2E79005CBF022ED29FDEE11
:04C09E003AFE80B531
:10DE340012DE3D12DE3D12DE3D7E0480067E02804F
:10DE4400027E017F0080087F6480027F017E00EFF4
:10DE54004E6012E4FD0D1D0DEDC394AD40F7EF1FB0
:10DE640070ED1E80EA22753500C200C201C2022292
:10DF1B00F5D8D2DCE5F520E7FBE5DA540FFEAFD9F7
:04DF2B0075D8002283
:10DB22007F767E06909C7E127702740412DF1B7C45
:10DB3200007D5212546FEFF875F00A84C0F07F76C0
:10DB42007E2312D5087E29742E12D51B7E2ED0E09C
:10DB520012D5087E35745612D51B7F6B7E1190DB71
:10DB62008B12D547E824E04001220423F824E75031
:10DB720002781812DB7BD8FB227F6CE82411FE7935
:10DB82000512DE740E0FD9F922071DFFFFFFE08098
:10DB9200000020C0000038E0000008F0000038F863
:07DBA200000020FFFFFFE07F
:10DBA90012DBD130E6022409540F75F00AA4F515E9
:10DBB90012DBD130E6022409540F25152212DBD1DC
:10DBC900540F2275F000800875F044800375F00742
:10DBD900E4206D09D5E0FAD5F0F7D24C229247C27C
:10DBE900ACE54F623885504FA26E926D859950C24F
:10DBF9006FD2ACC24CA2472212DC0BC4FA12DC0B66
:10DC09002A2212DBD120E603540F225407240922C9
:10DC1900E612DC2018E608FAC412DC26EA540F449E
:10DC290030F924C6E950112407800D75F00A84C023
:10DC3900F012DC3FD0E0443030530975F00085E044
:10DC4900E0D5F0FA3099FDC299F599623822E538A4
:10DC590080F2E53812DC20800812DC41E53812DC5C
:10DC690041740D12DC41740A80CE744012DC417497
:10DC79004080C5742C80C1742E80BD75380080B871
:10DF410085A0835383FE438380858384F075840099
:01DF510022AD
:10D9D00074A212DF4174A112DF4174A612DF4174F8
:10D9E000A412DF4174C012DF41742512DF4112DA44
:10D9F0006075C70375C6FC75B90112B619740812B3
:10DA0000DF1BEE75F020A4FEEF54F80303032E2471
:10DA100092C313FE24EA50027E16EE90DA49932553
:10DA2000BCFE24E6501F24E8401B748112DF41EE47
:10DA300012DF4112DA6D744012DF41742F12DF41A0
:10DA400074AF02DF417E2680E1F7F7F8F8F9FAFBC0
:10DA5000FCFDFEFF000000000101020202030303BF
:10DA6000A8BCA9BDAABEABBFACC7ADC62288BC8945
:0ADA7000BD8ABE8BBF8CC78DC62295
:10DD5900C006C007C5F075A7019000007EB7E58C25
:10DD6900240340FA12DD7B1EBEAFF3C5F0D007D005
:10DD7900062275A700EE12DF41741012DF41740408
:10DD890012DF4185A08343838185838475A7517FF1
:10DD990020E0F0E0F0E0F0E0F0DFF6E4F5A7F5844C
:01DDA9002257
:10DF2F0075A711900000E4C583F0C58330E2F8F5C2
:02DF3F00A72217
:10DE7400EF20E723EE20E71F20E61C05A7C4540388
:10DE8400F583EE5408C42FF582EE5407240983F574
:10DE9400F0E045F0F005A7228040201008040201BC
:10DEA400EF20E723EE20E71F20E61C05A7C4540358
:10DEB400F583EE5408C42FF582EE5407240983F544
:10DEC400F0E055F0F005A7227FBFDFEFF7FBFDFE82
:10D4C800FDA42582F582E5F03583F583ED22906091
:10D4D800AC7A0475F00512D4C87D05805E7A0580A3
:10D4E800027A04547FC0E0C083C082C394205001F4
:10D4F800E490605C12D4DB802E9061BA7A058005D6
:10D508009062777A0675F00712D4C87D07802C7A66
:10D518000580027A06C0E0C083C082C3942050010F
:10D52800E490620712D50DD082D083D0E022905FBC
:10D53800D075F00A12D4C87D0A7A07C2D18002D207
:10D54800D1C0A7C082C083C007C006C0E030D109DF
:10D5580075A704E493FDE493FAEEFB75A704EBFECC
:10D56800EAFC7901D9067908E493F5D4E5D423F5E2
:10D57800D420E01612DEA40EDCEA0FDDE1D0E0D004
:10D5880006D007D083D082D0A72212DE7480E8901C
:10D598005F1075F00E12D4C87D0E7A0812D543902C
:10D5A8005FB875F00212D4C8E493FDE4A393FACEF1
:10D5B8002408CE7C0812D5C47C06AD02ED23FD20DC
:0ED5C800E00712DEA40FDCF42212DE7480F7FE
:10D3B300F5D2C2D58036F5D2D2D58030F5D224F657
:10D3C30050090E0E24A650030E0E0EE5D2F5D275AB
:10D3D300F0648485F0D3C2D57009D2D5742012D5F8
:10D3E3001B800312D508CE2406CEE5D375F00A843C
:10D3F30085F0D3700A30D507742012D51B80031231
:10D40300D508CE2406CEE5D312D508E5D222F5D22F
:10D4130075F0648485F0D3C2D58022F5D2C2D5805D
:10D4230025F5D2D2D5801FF5D275F0648485F0D36B
:10D43300C2D57009D2D5742012D51B800312D50131
:10D44300CE2405CEE5D375F00A8485F0D3700A3077
:10D45300D507742012D51B800312D501CE2405CE27
:10D46300E5D312D501E5D222F5D2C2D58035F5D266
:10D47300D2D5802F30E70DF404C0E0742D12D4E927
:10D483000E0ED0E0F5D275F0648485F0D3C2D5706A
:10D4930009D2D5742012D4E9800312D4D6CE240441
:10D4A300CEE5D375F00A8485F0D3700A30D50774BE
:10D4B3002012D4E9800312D4D6CE2404CEE5D312AD
:05D4C300D4D6E5D222E1
:1076E700909F721276F002DD597E00800E7405FEBF
:1076F700F51EE4FFF51DF51F203C3375A700E49345
:10770700700122A3B40204051D8003B4010A051FFA
:10771700EF2409FFAE1E80E612D51B7D06B440029A
:107727007D03B421027D02EE2DFE80D27E0075A777
:1077370000E493700122A3B40204051D8003B40181
:107747000F051FEF2407FFAE1E80E612D4E5800861
:10775700B45B0050F612D4E90EB4210280D30EB404
:10776700400280CDB42C0280C80E0EB45F0280C1E7
:10777700B45B0040BC0E0E80B8E60812D51BEE24A1
:1077870006FED513F422909CAC307409909CB0305F
:107797007303909CB502770275F019D5E0FDD5F01B
:1077A700FA12484F12DC73744F12DC84744B12DCEC
:1077B70062C322C2501277FE12484FD2AC12DBCC02
:1077C700304C1212DBCC304C0C12DBCC304C06D2D6
:1077D70050C2ACD322B440E512DBD1B4400312DB74
:1077E700D1B44FED12DBD1B44BE712DBD112DBD1B1
:1077F70012DBD1C2ACC32230530975F008D5E0FDC6
:10780700D5F0FA227F0575F019D5E0FDD5F0FA120B
:10781700484F12DC73745712DC84745012DC4174C5
:097827008112DC41E56312DC4131
:10783000E56212DC4178D0E612DC4108B8D7F8E600
:10784000F8795F30E702792FE912DC4112DC41124E
:10785000DC4112DC41745812DC41744312DC41E417
:1078600012DC41E8C2E775F00A84C425F012DC415D
:107870007864E612DC4108B869F8E612DC62127737
:10788000BA400122DF02800A20508B75F000808010
:10789000D250C2ACD3221277FEC25012484FD2ACA3
:1078A0002002EF12DBCC204CE7B440F412DBD1B461
:1078B000400312DBD1B457DAF53812DBD1B450D221
:1078C00012DBD112DBD1F56312DBD1F56278D01275
:1078D000DBD1F924A0500353015FE924E040027991
:1078E0005FA60108B8D8E8780612DBD1D8FB12DB16
:1078F000D1FC53040FC4540F75F00AA42CFC249C33
:1079000050027C0078D78601E4B92F02D2E72CF62A
:10791000786412DBD1F608B86AF812DBD1E538607A
:107920000302789212DBD112DBD1C2ACC32290A346
:10793000878003909FB67F2012773312DD5902DED5
:1079400045753400C26B1279FD12DE45127DADE53E
:1079500016600312795902025912800F121E461244
:10796000DD5910002010010280F8127E1850131209
:107970001E5112792E10000D10010280F8121DF315
:0579800080D7127B9D81
:1079850022C26BD22775480A122B77753400127EF6
:10799500E5C26A1233CF106A0512024A80ED12025F
:1079A5004A127D3F127E97127EF178D0E6642660FA
:1079B5004412800F121E4612DD59100038100102C4
:1079C50080F8127E18501BE965156018121E5112B9
:1079D500792E12DE3D10001D10010280F8121DF3F4
:1079E50080BCD26B127EC3751607855917122BF012
:1079F5007535008096020259127DAD127A1F127EEE
:107A0500F17F19127A3990A3B47E121277357E234D
:107A1500E51602D48790A50180EF7862E4127A30EA
:107A250078D0745F127A3018E4F6227F08F608DF02
:107A3500FC227F7B7E007810742012D4E9CE2404CA
:107A4500FED8F5227F197E081277357E28909F98FB
:107A5500305303909F9D027735C26B127A1F127ABD
:107A650069020259C251127EF190A3AC127A4912F1
:107A75001E19127DAD7F20127A0812DD59E51670A8
:107A85000512DE3A803675A6FF3051031277A8122B
:107A9500484FD2AC200025306DFA127899400C126F
:107AA5007E184011127B9DD25180BB105003127974
:107AB50033C25180D1D25112792E80CAC2AC22D2A2
:107AC5002775480A122B77753400C26B127EE5C202
:107AD5006A1233CF106A0512024A80EB12024A126B
:0D7AE5007D3F127E97127EF1127AF550DA85
:107AF200020259909FB1127A49121E2B12DD59C30C
:107B020010001310010510020E80F412780B4001D0
:107B12002212793380DDD3C2AC22D227C26B7548E0
:107B22000A122B77753400127EE5C26A1233CF1027
:107B32006A0512024A80EDD26B127D3F127E9712C5
:107B42007D6775B901E5BCB2E7F5BC124EE6751664
:107B520007855917122BF080CB127DADE516601FF9
:107B620078D0E53D127B8EE53E127B8EE53F127B9F
:107B72008E765A08765F12C84C127EC3027D7E7FD3
:107B82003E7E11909F8812770202DD5975F00A84B9
:107B92004430F608E5F04430F60822D26B127EC378
:107BA200127D7EE51775F01084240AF54824E8500A
:107BB2000375480A122B838558592275320012BE6A
:107BC2009C75A704900700751500127D6775B901B1
:107BD200E5BC20E705E515F0801004600D648260C5
:107BE2000975BCFF75B90575B9020515E51524209F
:107BF20050D8E58224FE4003027C96A882187F00BA
:107C020075A7007583078882E0FE75F004A4127DD3
:107C120012A9BCAABDABBEACBF1582E0FD75F004D3
:107C2200A4127D12C3E995BC404C7052EA95BD4046
:0D7C320045704BEB95BE403E7044EC95BF95
:107C3F004037703DEE75F004A404127D12A9BCAA62
:107C4F00BDABBEACBFED75F004A404127D12C3E949
:107C5F0095BC4015701BEA95BD400E7014EB95BE98
:107C6F004007700DEC95BF5008EEF00582EDF01552
:107C7F0082E5826009C3EF95825003027C0A0FC32D
:107C8F00E89F4003027C0275A70490070075C703A5
:107C9F0075C6A8E0F5BCE0F5BDE0F5BEE0F5BF7533
:107CAF00B90575B90205C6E58224204006E5C6244C
:107CBF002050E00875C70375C68075B901E5BC1281
:107CCF007CFCF5BCE5BD127CFCF5BDE5BE127CFC71
:107CDF00F5BEE5BF127CFCF5BF75B90205C6E5C65A
:107CEF00245850D6E5320470FB75A70022B4FF016B
:107CFF0022F975A704900700E582686005E06970B6
:107D0F00F7E922F5C685F0C775B901E5BC645F7068
:107D1F000375BC27E5BD645F700375BD27E5BE64C1
:107D2F005F700375BE27E5BF645F700375BF2722C1
:107D3F0075C703E54875F004A42480F5C6E55975A9
:107D4F00F00484A8F00825C6F5C675B901A9BCAA28
:077D5F00BDABBEACBF8615F1
:107D660022E515242050037515DFE51575F004A4EA
:107D760054FCF5C685F0C722E51724204028E517F0
:107D860075F00484A8F00824A8F5C675C70375B96C
:107D960001A9BCAABDABBEACBFA61589BC8ABD8B6A
:107DA600BE8CBF124EE622E4F516F51579FF127D5C
:107DB6006775B901E5BCB4FF040516A9150515E5F7
:107DC60015242050E9891579FF75C70375C6A8756E
:107DD600B90109E5BC04601B09E5BD04601509E5A8
:107DE600BE04600F09E5BF04600905C6E5C6242088
:107DF60050DD09891722751600751501127D677504
:107E0600B901E5BC20E70205160515E51524205045
:107E1600EB227900E975F004A454FCF5C685F0C799
:107E260075B901E5BC20E73078D066702B08E5BD52
:107E360066702508E5BE66701F08E5BF6670190501
:107E4600C675B90108E5BC66700E08E5BD66700822
:107E560008E5BE667002D32209E9242050B6C32283
:107E6600127E86127E6EA8017F08E0F608DFFB22EE
:0B7E7600127E86127E7EA8017F08E6C7
:107E8100F008DFFB2278D0796275A704758307EBD0
:107E9100C454F0F58222127D6778D0127EB1E5BC20
:107EA100F9C23C20E702D23C127EB17862127EB167
:107EB10075B901A6BC08A6BD08A6BE08A6BF0805DF
:107EC100C622127D6778D0127ED3127ED3786212D9
:107ED1007ED386BC0886BD0886BE0886BF08124EC2
:107EE100E605C622125A3612DF2F12866E02DD59BE
:107EF10012DF2F7F007E0990A3991277027F0A7EFD
:107F010012E5150412D3BF7F1412CA36121DF37F76
:107F1100277E0875130778D0127780E6793E30E71F
:107F210002792F7E34E912D51B7F3D7E0190A51D7C
:107F310012773520311B3030031291A9C23B1281D7
:107F4100A1127F57D23B1281A1127F691281E88071
:107F51007C12C0A280E6C23B7F4474532017027496
:107F61004E7E0012D51B8017D23B7F4F74572017CE
:107F71000274457E0012D51B7E06E51E12D5087ED1
:107F81000CE51D12D5087E12E51C12D5087E17746A
:107F91008112D51B7E1CE51B12D5087E22E51A1223
:107FA100D5087E28742E302602742712D51B7E2D0B
:107FB100E51912D5087E33E51812D5087E39302629
:0F7FC10007742C12D5177E3BE53702D508742DB7
:107FD000201702742B7F707E1512D51B127FEC7E4A
:107FE0003A12D3687E0190A5480277027E1BE51CF9
:107FF00012D5087E21E51B12D5087E27E51A12D579
:10800000087E2DE51912D5087E33E51802D5081231
:10801000808D1280B812838F127EF11283E72017B1
:108020001E10021B1248F012C84C128075121DFE61
:108030007F347E2F12778D127F2A12DD5980E21253
:108040001DF3203026203128C23B1281A11280CDA1
:1080500078661282A1D23B1281A11280E278691265
:1080600082A11281E812815C02834412927280F232
:1080700012C0B780EDE57D75F01084AAF075F00AA6
:10808000A42A547FFA78D7E654802AF6227F277EE6
:108090000879D08700C001D224B9D002C22412844A
:1080A0006ED001A70010230909EE2406FEB9D7E31C
:1080B0002219EE24FAFE80DB7E3479D7E7A2E7921C
:1080C0001712841B79D7E7A21792E7F722C224C2BE
:1080D0003B751E007F447E0012842B801E1023ED12
:1080E000802AD23BC2247F4F7E00128433D2247E6A
:1080F00006E51E128460F51E1023E7D2247E0CE5EF
:108100001D128460F51D303BD41023E1D2247E1271
:10811000E51C128460F51C1023E17E1CE51B128413
:0381200060F51BEC
:108123001023E67E22E51A128460F51A1023E87EF6
:108133002DE519128460F5191023E87E33E5181232
:108143008460F5181023E87E393026027E3BE5373C
:10815300128460F5371023E3227F707E1512842387
:10816300C2247E1BE51C128460F51CD2247E21E50B
:108173001B128460F51B1023E77E27E51A12846027
:10818300F51A1023E67E2DE519128460F5191023E4
:10819300E87E33E518128460F5181023E82278D7B7
:1081A300E6C2E775F00A847866F537303B057869EF
:1081B30085F03712821130262BE53775F003A404BE
:1081C3000475F00584FBE51975F00AA4251875F00C
:1081D30006A42BFBE435F0FC125585F537125585C3
:1081E300F5188B1922E563FC339217AB6250031227
:1081F30055F6305C0A7AD21253717840125513AE99
:1082030004AF037C277D1012547C8F1C8037E6FD5E
:1082130033921718860418860350031255FE7A0901
:10822300792778C01255108B1EADD3ACD2AB06792B
:10823300EA786012550E8B1DAF06AED27C177D70A7
:1082430012547C8F1CAF05AE047C037DE812547C72
:0F8253008F1BAF05AE047C007D6412547C8F1A24
:10826200ED75F00A84F51985F01822EC3392175057
:10827200031255F6751D30301786751D2D808178D5
:10828200427B607CEA800678407B207C4E12C18271
:108292007927781012550E8B1CAF06AED280AB3008
:1082A200262AE51975F00AA4251875F00AA42537BF
:1082B200FBE435F0FC7A051253638C068B077C00D5
:1082C2007D0312546F8E048F031281DBE51E75F05D
:1082D2000AA4251D75F00AA4251C75F006A4251B09
:1082E200FBE435F0FC7A0A125363EB251AFBE43CFB
:1082F200FC7A0A125371EB2519FBE43CFCE43DFDC8
:108302007A0A125383EB2518FBE43CFCE43DFD3072
:1083120017031255FEA60518A60418A60378D7E679
:10832200A2E7923DC2E775F00A84FCABF0303B0E47
:10833200AB37EC75F00AA42BA23D92E7F622AC37DC
:1083420080F012835F305C0A7A4012537178D21245
:1083520055133017031255F68C638B622212836F0A
:108362007A0A125363EB2518FBE43CFC22E51C75E8
:08837200F00AA4251B75F00AB6
:10837A00A4251AFBE435F0FC7A0A125363EB25199B
:10838A00FBE43CFC221283C112DE41C202C2231268
:10839A0083C110000810010510021B80F51031ED91
:1083AA0010300D102604D22680E3D230C23180DD8F
:1083BA00D231C23080D7227F3590A506127733900A
:1083CA00A52420300F90A54020310990A51520261C
:1083DA000390A50D1F7E1712770202DD597F357EA5
:1083EA0001909F651277357F347E3A128510744E5C
:1083FA0012D51B12DD5912DE41C2027F347E3AD2F7
:10840A001775115975124E802675112E751227800F
:10841A001E75113E75122F801675112B75122D803F
:10842A000E75114E75125380067511457512571245
:10843A008510E511301702E51212D51B12DD59100D
:10844A00000810010510020B80F5D23C1017E3D288
:10845A001780DF02850B4430F812846AE8540F2231
:10846A00C2218002D221A22492229223128510E8EC
:10847A0030E709D23C7430302102745FF812D51B00
:10848A0012DD5910003410010510025D80F5D23C4E
:10849A00102266102367B43909745F2021DF743013
:1084AA0080DBB45F04742D80D4B42D04744180CD74
:1084BA00B45A04743080C60480C3D23C30240610F7
:0F84CA002237102338B44104742D80B1B42D042F
:1084D900745F80AAB45F04743980A3B43009745AF4
:1084E90020219B74398097148094B48908D223E899
:1084F90012D51B800DF8C223800874898001E80217
:1085090084879085258003908521C007EF2408FF83
:1085190012D547D00702DD590205F8F80205000017
:10DCF90075A70090DD2B75F02D84C2D5C2D16017B0
:10DD0900D2D1146007D2D514600DC2D1E5F093FCCD
:10DD1900742D95F093FB22E5F093FB742D95F09308
:10DD2900FC220009121B242C353E474F58606870AD
:10DD39007880888F969DA4ABB2B8BEC4CACFD4D917
:10DD4900DEE2E6EAEDF0F3F6F8FAFCFDFEFFFFFF8E
:10DDF300D23D8002C23DED8BF0A430E70205F0C3B3
:10DE0300E895F020D50425F025F0FEED8CF0A43044
:10DE1300E70205F0C3E995F030D10425F025F0FFC2
:10DE2300203D0B2487500122EF24CC40012202DE47
:01DE3300747A
:10D79700203A7A7E1C7F5312DE747F5912DE741E84
:10D7A7007F5712DE747F5512DE747E2312DE747F7C
:10D7B7005712DE741E7F5912DE747F5312DE741FF8
:10D7C7007E2012DE747F5A12DE747E1E12DE747F94
:10D7D7005212DE74120E67E5BD20E0143006117F89
:10D7E700357E1C90D853E571700390D85D02D547FC
:10D7F700E5716018E57012DCF9781F79567D09121A
:10D80700DDF7303A0312D8260DBD16F3227E1C7FB2
:10D817005390D83C12D547200CD612CA9280C0C06C
:10D82700060E30D5021E1E12DE74D0061F30D1023E
:10D837000F0F02DE74070700386C446C38000505CB
:10D847002070D8702005057088A8887008071038E0
:10D857007CFE383838000807102844C628283800C6
:10C8710090A5527F717E23127735120E67E5BC7E3B
:10C881003112D4D630121AC23C120E67E5BCFB75C8
:10C89100F00AA4F904FAC23D12BE8812CB0F303D52
:10C8A1000122DAF712CA167C00EBF4042E4019AD0E
:10C8B1000312546FEFA2D1203C077E237F6502D182
:10C8C10035AE16AF1702C9B7AD0112546FEF12D2D0
:10C8D10023203C077E237F6502D159AE16AF170294
:10C8E100C9DB7F567E0512CA427F3D12CA557F6F52
:10C8F10012CA5512CA927E0A7F4112CAC57E227F90
:10C901005912CAC52012012212BE88857A1D855E80
:10C911001C857B1B855F1A7AC0C23D12CB0B203D63
:10C921005212CA167C007D1412546F74562F20D1F6
:10C93100029F9FFF24CB40028037EF248850028062
:10C9410030EA1475F00384FE12DE74C3E51B957B97
:10C95100FEE51A955F92D55004EEF404FEEEC31382
:10C96100FE24E0400C741F2E30D5029E9EFE12DE86
:10C9710074DAA8227F5212C9877F5A12C9877517A4
:10C9810053751600802B7E0012DEA40EBE12F92212
:10C991007F157E28742012D51B7F1C7E2812DEA4F1
:04C9A1000EBE40F98D
:10C9A500223012E712C99175171575162DD23C0262
:10C9B500C88AC23D6002D23D92D175F080305C04D8
:10C9C500F5F08001A4A2E792D5E5F075F03284F880
:10C9D500E5F075F00584C0E0E5F0A2D533C0E0E8E8
:10C9E500601E12D508EE2406FED0E0F8D0E012D580
:10C9F50008EE2406FE742C12D51B0E0EE802D5088F
:10CA05007420303D07742B20D102742D12D51B8064
:10CA1500D4C3ED957AFFEC955EFE92D15003125585
:10CA2500E6227F1512CA2E7F327E3E12DE74DEFBB1
:10CA3500227E0912DE740EBE36F9227E0112DE74E4
:10CA45000E0EBE3FF8227E3312DE740EBE40F92272
:10CA55007E047D1112DE740E0E0EDDF81F1F7E356D
:10CA650090A55B305C057E3190A55F027735740536
:10CA7500305C097E32740112D4D674067E3612D427
:10CA8500D67E3A740012D4D67E3D02D4D67F417E3E
:10CA95001F7D0F12DE740F0F0FDDF8227F687D03F7
:10CAA50080047F677D0512DE740FDDFA227F667DC7
:10CAB5000780F37E1F7F5012DE741F1FBF3EF822D2
:07CAC5007D0A12DE740E0E63
:10CACC000F0FDDF722203D07123C767003D23D227A
:10CADC00056D12BC4EE4F5F7C2B2C2B2ABF7F5F776
:10CAEC00C2B2C2B2E5F7FA30E411EB251DF51DE434
:10CAFC00351CF51C0519EA30E3010ED2B28015780D
:10CB0C000380027801203D07123C767003D23D224F
:10CB1C00D8F3056DE56D2409F56D12BC4EE4F5F7FF
:10CB2C00C2B2C2B2ADF7F5F7C2B2C2B285F71BF50D
:10CB3C00F7C2B2C2B2E5F7FCD2B2543F30E50244C0
:0FCB4C00C0CC54C02323F51AE56D24F6F56D22F5
:10D6BE007E017F0990D73C12D5472051097E037F0A
:10D6CE0000743F02D51BE4FEFFC3E54512CF8DFD6E
:10D6DE00940AED403D9464ED4002746312D3B97E1A
:10D6EE00017F09E552240575F02D84AAF075F00529
:10D6FE00A4CA75F00B842A90D7279312DCF9BCB814
:10D70E00027BB87D04EE2DF8EF2DF90D12DDF3DD61
:10D71E00FB227E0312D50880C6000C1622222D395C
:10D72E00444F4F5A66707C7C87939EA9A9000909C5
:10D73E000800410000000000888000000000410049
:10D74E000800120E7BE5BCB4F8339004C3E0602CE5
:10D75E00FA24F340277F137E0012DE740F0F12DEC1
:10D76E00740E12DEA41F1F12DEA40EDAEC7F147EDE
:10D77E000012DE740E12DEA40EBE12F5229005CC3F
:09D78E00E0C3941240F60480C7C8
:10CF8D00305D0A75F08AA42480E5F0340022207407
:10CF9D00157F017E1190D01512D5477F0A7E0AE5C7
:10CFAD002E540702D3D07F087E1190D02512D5477D
:10CFBD0020730C7F0A7E1712DEA40E0E12DEA47FE4
:10CFCD00007E0BE57112CF8D12D3BF7F0C7E11E564
:10CFDD0071602F0EE57064B4602864B475F032840E
:10CFED00C0F012D501CE2405CED0E075F00584C079
:10CFFD00F012D501CE2405CED0E023302D01040250
:10D00D00D50190886A027702070FFFFFC473BDAF89
:10D01D00A463B5FBCDE7FFFF030F0100FFFE038007
:10D02D00306701227F357E00748812D51BE5516073
:10D03D001712CF8D75F06484F87E06E5F012D41EBC
:10D04D00E860E07E0002D5087E003074D63073169D
:10D05D0079BCE7FC09E7FB12530B781D201704E69A
:10D06D0070011802D2E9909CB0027702202C0122A7
:10D07D0090D08302D547050EFFF0E01CF004F81C9C
:10D08D00FFF0301201227F637E00909CC712D547BE
:10D09D007F1512CA2E7F1F12CA2E7F2912CA2E7F0C
:10D0AD00177E06E53F30E00B90A56F305C0390A531
:10D0BD008380132074077E01909CE7800990A564FE
:10D0CD00305D0390A579127702307306E54E60024C
:10D0DD00154E205718E54EB40113120E8AC3E55CA8
:0DD0ED009560F5BCE55D9561F5BD124EE660
:10D0FA007F217E01E53F30E021305705909E108068
:10D10A0016E54E7005909E1B800D909CF3127702D7
:0BD11A007E30E54E02D4241277022282
:10D28B0012530B7F207E05751900781DC2D5E63031
:10D29B00D51712D501EE2405FE18B818F17E1F74B0
:10D2AB0063305C02748202D51B7005B8191880E2DA
:10D2BB00D2D5CE24FACE7484301702742D12D51B1E
:10D2CB00EE2406FE80C8742012D51780C8781C8007
:10D2DB000D7F007E23AC5EAB7A12530B781DC2D54B
:10D2EB00E630D50C12D508EE2406FE18B818F1223C
:10D2FB007005B8191680EDD2D53017E4CE24FACECE
:10D30B00742D12D51BEE2406FE80D5742012D51B6E
:10D31B0080D512530B781DC2D5E630D51612D4D654
:10D32B00EE2404FE18B818F10E745E305C027427FC
:10D33B0002D4E57005B8191680E3D2D53017DACED2
:10D34B0024FCCE742D12D4E9EE2404FE80CB742081
:10D35B0012D4E980CBC23D12D3730F0F0E0E746340
:10D36B00305C02748202D51B12530B781DC2D5E6BA
:10D37B0030D50C12D536EE2408FE18B818F12270F1
:10D38B0005B8191680EDD2D5301716740BCE24F8CC
:10D39B00CE12D536EE2408FE80D5740C12D536800D
:08D3AB00D5303DCB740A80E58A
:10D867007F797E24E55F30E70122AC5F1CAB7B123A
:10D877005339E51B700E742012D51BEE2405FE12DA
:10D88700D8B5800C12D8B5E51B12D501EE2405FEDC
:10D89700E51A12D501EE2405FE742C12D51B0E0EC7
:10D8A700E51912D501EE2405FE745E02D51B742D11
:10D8B700201702742B12D51BEE2406FE22E55F30DB
:10D8C700E70122AC5F1CAB7B125339E51B700E746A
:10D8D7002012D4E9EE2404FE12D90E800C12D90EC0
:10D8E700E51B12D4D6EE2404FEE51A12D4D6EE2494
:10D8F70004FE742C12D4E90E0EE51912D4D6EE24C8
:10D9070004FE742A02D4E9742D201702742B12D452
:06D91700E9EE2404FE22EB
:10D125007F097E2530040512D21F8028A275E57976
:10D13500C23D6002D23D92D175F080305C04F5F0BD
:10D145008001A4A2E792D5E5F075F03284F8E5F008
:10D1550075F00584C0E0E5F0A2D533C0E0E8602AAB
:10D1650012D536EE2408FED0E0F8D0E012D536EE22
:10D175002408FE0F0FE52B5403701F746012D51B96
:10D185001F1FEE2404FEE802D536740C303D0674EC
:10D195000A20D1010412D53680C9205904742E8085
:10D1A500DC205804747F80D5748080D1300405124A
:10D1B500D21F8028A275E579C23D6002D23D92D189
:10D1C50075F080305C04F5F08001A4A2E792D5E506
:10D1D500F075F03284F8E5F075F00584C0E0E5F00F
:10D1E500A2D533C0E07F3E7E1CE8602012D597D0E3
:10D1F500E0F8D0E07F3E7E2812D5977F447E3274DA
:10D205002E12D51B7F3E7E37E802D597303DE07460
:10D215000A20D1010412D59780D59005CAE075F092
:10D225000A84F8E4C5F0C2D522301105E54AB402F6
:10D2350050C39006E9E0957AFB9006E8E0955EFC20
:06D2450050031255F6EC47
:10D24B00C31360047B63800FEB13FB249C40F5241A
:10D25B004F4004C20480079005CAEBF0D20490063D
:10D26B00E6E09006E8F09006E7E09006E9F0E55E70
:10D27B009006E6F0E57A9006E7F02212D26980DE9E
:10CB5B00E54424F64001227800E552206607C39590
:10CB6B0070500224B40475F00384F9E928FE24C440
:10CB7B005001FE12CB9D12CBA91E12DE74C3E99895
:10CB8B00FE5003243CFE12CB9D1E12DE7408B81F10
:10CB9B00DA22EE2420FE24C250032402FE22E824D3
:10CBAB00F1E8C2D55006D2D5E8F4241F23FF90CC70
:10CBBB002B93CF0493FAE545F5F0A4ACF0FB12539D
:10CBCB009AE544F5F0A49BFBE5F09CFCEB2420FBE1
:10CBDB00EC3400FC12CC0CFAE5458FF0A430E702E4
:10CBEB0005F0E5F020D502F4042A75F005201903B1
:10CBFB0075F00384FF24DF50027F20C374329FFF44
:10CC0B0022EC24F0500BEB2460EC340090CC7B93A3
:10CC1B0022EB33FBEC33FCEB33EC3390CC4B93221A
:10CC2B00FF00FF03FA0BF318EA2ADE40CF58BE735E
:10CC3B00AB8D96A880C068D64FE835F51BFD00FF7D
:10CC4B0000080B0E101214151718191B1C1D1E1F94
:10CC5B0020212223242526262728292A2A2B2C2D5E
:10CC6B002D2E2F2F30313132333334343536363796
:10CC7B00373839393A3A3B3B3C3C3D3D3E3E3F3FF2
:10CC8B004042444648494B4D4E50525355565859C5
:10CC9B005B5C5D5F60616364656668696A6B6D6E42
:10CCAB006F7071727374767778797A7B7C7D7E7F07
:10CCBB00808182838485868788898A8B8B8C8D8EF5
:10CCCB008F9091929394949596979899999A9B9CFF
:10CCDB009D9E9E9FA0A1A2A2A3A4A5A6A6A7A8A91C
:10CCEB00A9AAABACACADAEAFAFB0B1B1B2B3B4B44B
:10CCFB00B5B6B6B7B8B9B9BABBBBBCBDBDBEBFBF85
:10CD0B00C0C1C1C2C3C3C4C5C5C6C7C7C8C8C9CAC9
:10CD1B00CACBCCCCCDCECECFCFD0D1D1D2D2D3D417
:10CD2B00D4D5D5D6D7D7D8D8D9DADADBDBDCDDDD6D
:10CD3B00DEDEDFDFE0E1E1E2E2E3E3E4E5E5E6E6C8
:10CD4B00E7E7E8E8E9EAEAEBEBECECEDEDEEEEEF2A
:10CD5B00EFF0F1F1F2F2F3F3F4F4F5F5F6F6F7F791
:10CD6B00F8F8F9F9FAFAFBFBFCFCFDFDFEFEFFFF00
:10CD7B00E54524FD400122E552206607C39570501E
:10CD8B000224B40475F00384241FFE24C250032430
:01CD9B000295
:10CD9C00FE12CDD6EEFD241EFE24C250032402FE4C
:10CDAC0012CDD6E544240275F00520190375F00365
:10CDBC0084F4042432FF24EE500F12CDCBAE051EAA
:10CDCC001E7C0512DE740EDCFA227F1512DE740F47
:05CDDC000FBF2DF8223D
:10D5D6007E00206615E5700475F0B484E5F075F0FC
:10D5E6000384FE6004C3743C9EFE745312D6017419
:10D5F6005712D601744E12D60174457F2F12D4E904
:10D60600BE00077E3C12D4E97E00EE240875F03C8D
:10D6160084AEF00F0F0F12DE740E12DE740F12DEE0
:10D62600741E12DE74EE240775F03C84AEF02230D0
:10D63600745C301259E54AB4040122B4060122E5AD
:10D646007112CBF58F057C037E1E30662AE57004C9
:10D6560075F00384241EFE24C6501C24FB500424AB
:10D66600038013C00612D67DD0E024C67C01600676
:10D676000C1460020C14FE12D6890EEE24C1400270
:10D68600DCF5228D0712DE740FEF24CE50F722E56B
:10D6960053206607C39570500224B40475F00384C2
:10D6A600241FFE24C250032402FE12D6B40E7F238A
:08D6B60012DE740FBF2DF922F2
:10DDAA00AF177E00E53C12D3B37E0C742E12D51B3E
:10DDBA007E12E53B12D3B37E1E742E12D51B7E242F
:10DDCA00E53A02D3B37E0E78ADE612D41E7E1874FD
:10DDDA002C12D51B7E1B18E612D41E7E25742C121B
:09DDEA00D51B7E2818E602D41EA8
:10CDE1007F797E00E54012D41E7E0A743B12D5176E
:10CDF1007E0CE54102D41E7F797E16743B12D51755
:10CE01007E18E53F12D41E7F797E0078AEE612D4FB
:10CE11001E7E0A743B12D5177E0CE53E02D41E30ED
:10CE21005EE52043E27F6D7E0078AEE612D41E7E81
:10CE31000A743B12D5177E0CE53E12D41E7F757E17
:10CE41000075F00A84E5F012D5360F0F7E08743AAA
:10CE510012D5171F1F7E0DE53F75F00A84C0F01231
:10CE6100D536EE2408FED0E002D536851C1E851B82
:10CE71001FAB1BAC1C305D0A7A1B12537178321246
:10CE81005513C3EB33FBEC33FC923D125342303D5F
:10CE9100087409F51DF51CF51B7F75E51D60157EF0
:10CEA1002412D5367E2CE51C12D5367E34E51B12B4
:10CEB100D536803D7E22E51C601912D5367E2AE5E5
:10CEC1001B12D5367F787E31742E12D5177F75E50A
:10CED1001A8019E51B12D5367F787E29742E12D55A
:10CEE100177F757E2DE51A12D536E5197E3512D5D7
:10CEF100367F777E3C125CCC851E1C851F1B227FF2
:10CF0100397E1F12DE740FBF40F9781F79567A00FF
:10CF11007D1A12DCF912DDF7EA2406FABAAEF378CB
:01CF21001BF4
:10CF2200C3E5119570500224B4FA604214603E14B5
:10CF3200603A2450603A146036EA24A540278A1EDB
:10CF4200751D007D1912CF520D30740312CF520D90
:10CF5200781F7956AA1DEA12DCF912DDF70AD3EA24
:10CF6200951E40F2228A1D751EB380D70808080854
:10CF72007F367E1C90D853E571700390D85D12D530
:0BCF8200477F3CAE0090852102D547A0
:10DA7A00787512DACA7453201702744E207406E5B8
:10DA8A002E54074430AF1712DAF47E3BE57DC454B6
:10DA9A000F12D5082074077E07742012D51B7878D8
:10DAAA0012DACAE5172409FF7457201702744520B1
:10DABA007402742012DAF47E3BE57D540F02D50815
:10DACA00E6FD339217188604188603301703125599
:10DADA00FE7917787012550E8B13AF06AED27C0002
:10DAEA007D6412547C8F148D15227E0012D51B7E04
:10DAFA0007E51312D3D07E19748112D51B7E20E557
:10DB0A001412D3B37E2B742E2073030E742C12D5E9
:08DB1A001B7E2FE51502D3B3B9
:10DC8900E54A602E7A2420E00E7A26141460087A78
:10DC990028141460027A297F667E01EA12D51B20B6
:10DCA9005505205406800B745B8002745C7E00125B
:10DCB900D51B20110778A9B60007802130261EC27E
:10DCC90026909D877F681276F07F66A85AE54AB448
:10DCD900060108E875F06484E5F012CE5A20080FB1
:10DCE900E537640260097F367E2E744112D4E92239
:10D91D0020144F740512DF1BEF33EE33F9EF0303C1
:10D92D00541FF5F090D970E993A4C5F013C5F01309
:10D93D00C5F013C5F013C5F0135403FCE5F013FB4C
:10D94D00E9242093C9244093C39BC4540FFBE99C45
:10D95D00C4FC540FF9EC54F02B2446F57BE934F656
:10D96D00F55F22FFFFFFFFFFE6C5AD9C8F857D773D
:10D97D00726E6C6A696A6A6C6F747A828D9DB4D9A5
:10D98D00FFFFFFFAE9DCD3CEC9C6C3C0BEBBB9B732
:10D99D00B5B4B2B0AFADABAAA8A6A4A2A09E9C99F7
:10D9AD0096918C00381CE735D137246F00C5B3C173
:10D9BD00E61F66B60E68C21867AADBF4EDB94675A8
:03D9CD0010A200A5
:10DEFB00D2A27408D2A1D2A300C2A3C2A1D2A30002
:10DF0B00C2A3D5E0EF7405D2A300C2A3D5E0F822DB
:10DED400C2A3D2A2D2A1D2A300C2A375F0083392E6
:10DEE400A1D2A300C2A3D5F0F5C2A175F003D2A3B9
:07DEF40000C2A3D5F0F822E3
:10C48B0012DED4D2A300C2A3C2A175F008E4D2A3DA
:10C49B0000C2A3A2A233D5F0F5FE75F008E4D2A337
:10C4AB0000C2A3A2A233D5F0F5FFD2A300C2A322F0
:10C4BB00E478806608B88BFB70012274D512C48BAC
:10C4CB007881C3EE13FEEF13F692D118EE2460F6CB
:10C4DB0074D612C48B7888EF33CE33CE33CE33CEB3
:10C4EB0033A2D192E25407FCEEFB7A08125363ECB1
:10C4FB00244FF608EBF674D912C48BEF543F7882B5
:10C50B00F67886EF33CE33CE33CE33CE335403F6B9
:10C51B0008EEF618161608E6C4FF54F0F618E6C433
:10C52B00CF540F2FF674DA12C48BEF232354FC78FD
:10C53B0083F67884EEF608EF54C0F67880E466084C
:10C54B00B88AFBF62212C4937889C3EF96FF18EED4
:08C55B0096FEA2E792165010B3
:10C563001255E6740FF8F91253B0EF2CFFEE3DFEAF
:10C57300788BEEF608EFF622E6182016072CF7E67E
:10C583003D19F722C39CF7E69D80F66A405E80560C
:10C59300E050F04B0044803DC0384031D02BA02503
:10C5A300601F2018D014000F000AA0014401580195
:10C5B300680178018801A001B401D001EC021002E6
:10C5C30038026802A002DA030C034D78BE8020858E
:10C5D3008E8A9D8F4D95BA9A97A0BEA631AC53B261
:10C5E3002AB801BD6AC1EDC4D1C78812C493788D3E
:10C5F300EEF608EFF67887798C1253B0788379904A
:10C6030012C57B7885798C1253B07881799212C5E3
:10C613007B788DE624E4FE08E63392D13392D55439
:10C62300FCFFEEA2D133A2D533FE780F79921253D9
:10C63300B078947990C3EC97F61819ED97F679943E
:10C6430090C58E7F1F7D11EF93C3971F19EF9397AB
:10C653001F091DED600240EF0F90C5AE798DEF937A
:10C66300F7090FEF93F7788E79941253B090C5CEF4
:10C67300EF93C39BFB1FEF939C2420FC7897E62B3F
:10C68300F618E63CF618E436F6740612DF1BD237CA
:09C69300EE24F7400624025002D7
:10C69C00C237EEFCEFFD740712DF1BC3ED9FFFECFE
:10C6AC009EFE78B7E6FD337C0050011CEF2DFFEEAB
:10C6BC003CFE789CEF26F618EE36F622201412205B
:10C6CC00370F789DE6B4050912C78012C7B512C79B
:10C6DC00FE2220145E7897799A12C82F12556EC3D9
:10C6EC00EE9420FE924550031255E67C007D051217
:10C6FC00547C3045031255E6E531B40C3612DA6041
:10C70C00120E80E5BC2FF560E5BD3EF56120E7110A
:10C71C0024F8500DFAC3E5609AF560E5619400F5D4
:10C72C0061120E8AE5BC2560F57AE5BD3561F55ED2
:10C73C0012DA6D7897799AC3E697FB1819E697FC8D
:10C74C007A0212536330370B7A02125363ECFEEB0E
:10C75C00FF800312C78012C7B520140312C7FE78DE
:10C76C00957998E6F776000809E6F776000809E669
:10C77C00F7760022799CE77700FB19E77700FC78C5
:0CC78C009DE6B40506EB33FBEC33FCEC3F
:10C79800A2E792D550031255F67A32125371ECFB88
:10C7A800EDFC30D5031255F6ECFEEBFF22EE240823
:10C7B800FE74042037167406307511789DE6B405AA
:10C7C80004740C8007F42406C323540FFD7C001264
:10C7D800534F789FE6FC08E6FBC374109DFA12538A
:10C7E80071EFF8EEF912556EE878A02FF6FF18EE03
:10C7F80039F62480FE22927540031255E678BBE68E
:10C80800F5F02438400375F0E1EF33EE3378A8F6FD
:10C81800A485F07930E7020579C276307508E579A4
:10C8280024F15002D27622E627FB1819E637FC18C5
:10C8380019E637FD2212BE2F7F087871793A12C89F
:10C8480058024ABB855E63857A62787379647F068D
:10C85800E6F70809DFFA227864797380F17873794A
:09C86800AF80EB78AF797380E535
:1052E900E4FEFFFC7D0A791DE7540F2FFFE43EFE23
:1052F900B9190280061912534F80ED301703125560
:10530900E622305C2BEC33921750031255F6EC244D
:10531900D950047C277B007AD2125371EB33CC33FA
:10532900CD33CC33ED33FBEC33FC3017031255F698
:10533900EC33921750031255F67919125585F7096E
:10534900B91DF8A70322EFF88DF0A4FFEDC5F0CE43
:10535900A42EFEEC88F0A42EFE22EB8AF0A4FBE535
:10536900F0CC8AF0A42CFC22EB8AF0A4FBE5F0CC6B
:105379008AF0A42CFCE435F0FD22EB8AF0A4FBE5CD
:10538900F0CC8AF0A42CFCE435F0CD8AF0A42DFDF4
:1053990022EB8AF0A430E70205F0E5F0CC8AF0A40C
:1053A9002CFBE435F0FC2286F0E7FDA4FAABF019FA
:0653B900E786F0A42BFBC7
:1053BF00E435F0FC18E68DF0A42BFBEC35F0FCE4A3
:1053CF0033FDE687F0A42CFCED35F0FD22EB89F0E0
:1053DF00A4CBAEF08AF0A42EFEE5F03400FDEC89EC
:1053EF00F0A42EFEE5F03DFDE433CC8AF0A42DFDB4
:1053FF00E5F03CCEFC22EB89F0A4CBAFF08AF0A411
:10540F002FFFE5F03400FEEC89F0A42FFFE5F03E0E
:10541F00FEE433CC8AF0A42EFEE5F03CFCED89F0DF
:10542F00A42EFEE5F03CFCE433CD8AF0A42CFCE581
:10543F00F03D8E058C068F04FF22C2D5EC30E705B8
:10544F00B2D51255EEEE30E70DB2D51255E6125425
:10545F007C1255EE800312547C30D5031255E62290
:10546F00C3EC13C0E0ED132FFFD0E03EFEBC000BEA
:10547F00BE0029EF8DF084FFADF022E4CCF975F07A
:04548F0008EF2FFFF4
:10549300EE33FEEC33FCEE9DEC994005FCEE9DFEF5
:1054A3000FD5F0E9E4CEFD22EDF9F5F0EE8420D23C
:1054B3001CFEADF075F008EF2FFFED33FD400799AB
:1054C3005006D5F0F222C399FD0FD5F0EA22EC3352
:1054D300EE3400FEEF3400FF7D007A007900780996
:1054E300C3ED9AFDEE9BFEEF9CFFB392D54009ED11
:1054F3002AFDEE3BFEEF3CFFA2D5E933F9ED33FD88
:10550300EE33FEEF33FFD8D92279007A00C380153A
:1055130079007A00C3EA13FFE913FEE8132BFBEECD
:105523003CFCEF3DFDE4F5D2F5D333FE7F19C3EE2A
:1055330098FEE5D299F5D2E5D39AF5D3B392D54047
:105543000DEE28FEE5D239F5D2E5D33AF5D3A2D54F
:02555300EB3338
:10555500FBEC33FCED33FDDF0122EE33FEE5D23308
:10556500F5D2E5D333F5D380C3EDC454F0FEECC4D6
:10557500FF540F2EFEEF54F0FFEBC4540F2FFF2204
:10558500EC75F00A84FCEB54F025F0C475F00A8440
:10559500C4CBC454F025F0C475F00A842BFBE5F0A8
:1055A50022AC10AB11125585A904AD03FA7C197B09
:1055B50099125363AE04AF03EA75F006A4F8AC1272
:1055C500AB131255852875F00A8485F014F8EF2B76
:1055D500FFEE3CFEEF28FFE43EFEE43DFDE439FC32
:1055E50022C3E49FFFE49EFE22E4C39DFDE49CFCF0
:1055F50022C3E49BFBE49CFC22C3E49BFBE49CFCF0
:10560500E49DFD2275D4107B807A0079807800EACC
:0A561500F5F0A4FCADF0EBF5F0A4F5
:10561F00FEAFF0EB8AF0A4C333C5F033C5F092D5DB
:10562F002DFDC5F03EFEE430D501043FFFB5150D4D
:10563F00EEB51409EDB51305ECB51201224006EADB
:10564F0098FAEB99FBD5D40ABB0001220ABA0001E4
:10565F000B22C3E913F9E813F8EA28FAEB39FB80B8
:10566F00A478087B807D807C00EDF5F0A4FAE5F04E
:10567F008EF0B5F007EA8FF0B5F001224003ED9BF5
:10568F00FDD827BDFF0122EDF5F0A4F9A8F0ED0438
:10569F00F5F0A4C399FAE5F09813CA1329F9E83A7B
:1056AF00F8C3E99FE89E50010D22C3EB13FBED2BCE
:1056BF00FD80B6C374689511FB74019510FC8004CE
:1056CF00AC10AB117A0B79B81253DC80177473F8E6
:1056DF00F9E627FB0809E637FC0809E637FD30E74E
:0556EF00031255FEEB63
:1056F40033FBEC33FCED3323FD242083F8ED241C31
:1057040083FFED241883FAED241483F9EF99F9E863
:105714009AFA1253DCEF9DFFE89EFE22FFFFFFB6CC
:10572400FED7FD63FB5DF8C4F59BF1E3ED9EE8CF86
:10573400E379DD9ED743D06BC919C153B91CB07945
:10574400A7709E06943F8A237FB674FF6A045ECBDB
:10575400535B47BB3BF1300423FB17DE0BB2FF80E6
:10576400C21DC232532CF8C3E5679576FBE56895F4
:1057740077FCE5699578FD30E705D2611255FE2482
:10578400F05003125838AA06A907125405EC2480D5
:10579400E43DFBF9F51AE43EFCFAF519E43F600236
:1057A400D2321253DC8B128C138D148E15C3E56424
:1057B4009573FBE5659574FCE5669575FD30E70525
:1057C400D2621255FEEBF9F51FECFAF51DED6002FD
:1057D400D232303201221253DCEB2512F512EC35B1
:1057E40013F513ED3514F514EE3515F51540E102F6
:1057F400560912576420323BEB242E40D3EA24018D
:10580400CB3400FC7A07793D1253DCC010C0118EF2
:10581400108D118C128B13E4FCFD7E077FD012B522
:0E58240096851203851302D011D010BB00052B
:10583200BA0002D21D22B261C374809BFB74F59C34
:10584200FC74209DFD22204D69204866303F637F15
:10585200697E0112CA427E1F12CAB275A700900465
:10586200EDE0A2E792171392E7FC1582E013FB30FA
:1058720017031255F6BC003AEB603720E73420E6F6
:105882003110E513201707C3741F9BFE80027E1F91
:1058920012CAA70EDBFA22FB2017097E00C374206E
:1058A2009BFB8008EB241FFE74209BFB12CAA10EF7
:1058B200DBFA2275A700758307E559C4440FF58208
:1058C200E0A2E792522212C8651258B5C2E775F0FB
:1058D2000A84FEAFF075A7045382F1786412593E30
:1058E200AE07786712593E75A700E57DC4540FFED6
:1058F200E57D540FFF7873125932AE07787612594C
:105902003274AF1256DE1257F68B148A1312092024
:10591200ACCCAB017A0A125363E5139B9004ECF012
:10592200FBA3E5149CF0FCA2E7923DD23F02C86BB8
:10593200860308860408860518188006E0FBE0FC4A
:0A594200E0FD7A0A12538320E70CFF
:10594C00EB2EF608E43CF608E43DF622C3EB9EF69B
:10595C0008EC9400F608ED9400F622204D0920483E
:10596C0006C23F302A0522C23380F6E54824F640B1
:10597C00F5E5580460F075A700758307E559C42454
:10598C0008F582E0FEA3E0FF1209207437125A2AB0
:10599C00500B30381BC23878C586468013743212CF
:1059AC005A2A400C203809D23878C5A646754600CC
:1059BC00740D125A2A404A1258C8303D3820112210
:1059CC00204D1F20481C204019BCFF16EB243250E0
:1059DC0011D240120E62E5BF75F019A4F536D22E25
:1059EC00D22F205238E55965586032204D2F20486F
:1059FC002CD2338028201109204D062048037536FF
:105A0C0000303319204D1220480F1291460559C30E
:105A1C00E55895595003855859C233C2402229FB89
:105A2C00E435CCFCC3EB9FEC9E22E558B4FF01227D
:105A3C0085581175A704758307E54824F650028034
:105A4C005C201259202905202A02805112C865E4D5
:105A5C00F516F517751000125AC2E510700312C82E
:0B5A6C005F125ADB302910E51B2517E4
:105A7700F517F51BE51C3516F516F51C125AE81235
:105A8700C85F0510C3E511951050D175A70002C86E
:105A97006BE55AF51124F6500375110A75A70475BD
:105AA7008306751000125AC2125ADB125AE8051003
:105AB700C3E511951050EE75A70022E510C4F582D5
:105AC700E0E0F564E0F565E0F566E0F567E0F568C8
:105AD700E0F5692275A701125ED4123ED775A704B7
:105AE70022E9F0E51CF0E51BF022E510C454F0F5BF
:105AF70082E0F512E5822406F582E0F511E0F51C57
:105B0700E0F51B22E512B426157F757E34740D125D
:105B1700D53620442575110012CF00025C397F6D00
:105B27007E3BE012D51BE5137E3512D51BE5127EB1
:105B37002F12D51B20440312CF0012CE6C025C3902
:105B4700202852E558B4FF012275A704758307E59D
:105B570059F51030330965586005204802051012C1
:105B67005AF1E0F513305E07204304E5376095E00E
:105B77007F797E3D12D4E9E5137E3912D4E9E51227
:105B87007E3512D4E930480B7F7F7E3512DE740EE6
:105B9700BE40F980392012012275A7047583068556
:105BA7005B10125AF1305E0A204307E53770030293
:025BB7005D5B34
:105BB900E512700B7E3A7F79745D12D51B800D75E5
:105BC900F06484E5F07E397F7A12D46BE537B4024C
:105BD90005128FDE8045B403028040E51C7006E59E
:105BE9001B24FB5036E511F964B4602F20062CE51F
:105BF90037600D200C0AC3E99570F9500324B4F9F4
:105C0900E912DCF9781D79547D1D90D845E53F20CE
:105C1900E00390D84C12DDF712D547751779751640
:105C29001930280375161DE51264266003125C7C81
:105C390075A7009006E3E511F0A3120E7BE5BC758C
:105C4900F01970040475F014A4951BFBE5F0951C7C
:105C5900FC922450031255F6ECF0A3EBF0C24FC2AC
:105C690063EC700EEB24E64002D24FEB24C84002ED
:105C7900D26322E51C24ED402BAE1CAF1B125E9EA5
:105C89007C007D3212547CC005EFAF17AE1612D4DA
:105C990024CE2405CE742C12D51B0E0ED0E023126F
:105CA900D41E801B125E95125CD6CE2405CE742CB0
:105CB90012D51BCE2402CEE875F0058412D501CE8B
:105CC9002404CE7422305D02748302D517EE243D7C
:0D5CD90050047EC37F4B7C017DF412547C8F
:105CE600C004C005EF6007AF17AE1612D424D00764
:105CF600D0067C007D3212547CA805EFAF17AE1695
:105D0600CE240ACE02D501125E95EE2450305D03F4
:105D1600EE24A150047EC37F4B7C017DF412547C9B
:105D2600C004C005EF6007AF177E2F12D471D007ED
:105D3600D0067C007D3212547CC005EFAF177E374B
:105D460012D4D67E3B742C12D4E97E3DD0E075F099
:105D5600058402D4D67F6D7E2F746312D51BE5129F
:105D660075F06484E5F07E3512D3B312CF0002CE0F
:105D76006C30480320740122E4FCF5A79006E3E0AA
:105D8600F9A3E0FE24FE40EFA3E0FF7D78E537604F
:105D960008304FE3200C2A800B120E67E5BD20E089
:105DA60010304F0DD206E57124FE5015125E8B8021
:105DB600107D3CE546600A7D141460057D0A14706A
:105DC600B6891112534F7D6F12546FBE00A9EF248E
:105DD600E240A4AD07E51112DCF9202404B2D5B2E5
:105DE600D1781F795612DDF7A806A907E511242DEB
:105DF60075F0B484E5F012DCF97407304F02740EC6
:105E0600FDFA12DDF7B2D5B2D112DDF7B2D5B2D1B5
:075E1600DDF0AD0212DDF723
:105E1D00850616850717B2D5B2D112DDF785061E98
:105E2D0085071F7A03304F027A06E511241675F0A7
:105E3D00B484E5F012DCF9A816A917AD0212DDF74E
:105E4D00DDFBE51124EA400224B412DCF9A81EA9F9
:105E5D001FAD0212DDF7DDFBE5377021304F1E90CF
:105E6D00A627305D0390A6237F3C7E331277351233
:105E7D000E67E5BD20E00612CAB812D7E622C3E9C7
:105E8D009570500224B4F922E51B2402FFE4351C61
:105E9D00FE305D1ABEC305BF4D028012AC06AB07C6
:105EAD007A1B1253717832125513AE04AF03227858
:105EBD007379641256E01257F6751CC3751B4B208F
:105ECD0032048B1C8A1B22125EBC30320122AC19AB
:105EDD00AE1AA91DAF1FB90005BC00028010C3E9A1
:105EED0013F9EF13FFC3EC13FCEE13FE80E8BF298B
:105EFD00005006BE2900500122C3EF13FFC3EE135D
:105F0D00FE80EB3E7FE3E3E3E3E3E3E3E3E3E37F01
:105F1D003E0C1C3C7C7C1C1C1C1C1C1C1C7F7F3EDA
:105F2D007FE3E3E3070E1C3870E0E3FFFF3E7FE302
:105F3D00E3030F0E0F03E3E3E37F3E070F1F3F77EE
:105F4D00E7E7FFFF0707070707FFFFE0E0E0FEFFBA
:105F5D00030303E3E37F3E1E3F73E0E0E0FEFFE358
:105F6D00E3E3E37F3EFFFFE3E30303070E1C383853
:105F7D003838383E7FE3E3E37F3E7FE3E3E3E37FBF
:105F8D003E3E7FE3E3E3E37F3F030303E77E3C0015
:105F9D000000181818FFFF18181800000000000066
:105FAD00000000FFFF0000000000003FF00000387F
:105FBD001C38F00180C1F020F0FC0038F03FE0000B
:105FCD000000007CC6C6C6C6C6C6C6C67C183878D4
:105FDD001818181818187E7CC6C60C183060C0C664
:105FED00FE7CC6C6061C0606C6C67C0C1C3C6CCCCC
:105FFD00FE0C0C0C0CFEC0C0C0FC0606C6C67C3CDC
:10600D0066C0C0C0FCC6C6C67CFEC6C6060C18302F
:10601D003030307CC6C6C67CC6C6C6C67C7CC6C6FD
:10602D00C67E060606CC78000018187E7E1818006D
:10603D0000000000007E7E00000000000000000057
:10604D000000000000C6E2E2D2D2CACAC6C6C20033
:10605D000000000000000000008080A0C0A0003003
:10606D004020C08080C0A0A0000060A0600000A003
:10607D0040A05098D090882050A850888850A850A3
:10608D002060806000000040E040000000000080C3
:10609D000000E000000000000040002040800040B3
:1060AD00A0A0A04040C04040E0C02020C0E0E020C3
:1060BD004020E02060A0E020E0C02020C06080E013
:1060CD00A0E0E020404040E0A0E0A0E0E0A0E02023
:1060DD00C0004000400000800080002060E0602093
:1060ED0000E000E00080C0E0C080E0E0E0E0E00023
:1060FD000000000040A0E0A0A0C0A0C0A0C040A033
:10610D0080A040C0A0A0A0C0E080C080E0E080C022
:10611D0080806080A0A060A0A0E0A0A0E0404040F2
:10612D00E0202020A040A0A0C0A0A080808080E022
:10613D00A0E0A0A0A0A0E0E0E0A040A0A0A040C0F2
:10614D00A0C0808040A0A0C060C0A0C0A0A0608002
:10615D004020C0E040404040A0A0A0A060A0A0A072
:10616D00A040A0A0A0E0A0A0A040A0A0A0A0404062
:10617D0040E0204080E02020A870202070A8202042
:0D618D0008F030D0100000F0A8A8000000BD
:10619A00E0000000902048708898984000E0E0E015
:1061AA0000A0E0E0E04060301030604040E0404055
:1061BA0060909090909060206020202020706090E5
:1061CA0010204080F06090102010906010305090A5
:1061DA00F01010F080E010109060609080E09090D5
:1061EA0060F0102020404040609090609090606085
:1061FA00909070109060C0E0F0F8F0E0C0000000ED
:10620A000000000000000000000000506050007014
:10621A007050000078807008F000F8888888F800CC
:10622A00C0C8102040981800C0B098B0C0006020C4
:10623A0040000000000090D8FCD8900000246CFCBC
:10624A006C24000020A870A82000002020F820203C
:10625A000000000000000080000000F000000000C4
:10626A0000000000606000081020408000708888EC
:10627A00888888702060202020207070880810206C
:10628A0040F8F810201008887010305090F810105C
:10629A00F880F008088870304080F0888870F80824
:1062AA00102040404070888870888870708888788C
:1062BA0008106000606000606000000080000080DC
:1062CA0000002040F84020000000F800F80000001C
:1062DA002010F8102000708808102000200000000C
:1062EA000000000070888888F88888F08888F0881C
:1062FA0088F070888080808870E09088888890E034
:10630A00F88080F08080F8F88080F0808080708843
:10631A0080B8888878888888F888888870202020BB
:10632A00202070381010101090608890A0C0A090A3
:10633A0088808080808080F888D8A8A88888888803
:10634A0088C8A898888870888888888870F088881B
:10635A00F080808070888888A89068F08888F0A08B
:10636A00908870888070088870F82020202020206B
:10637A00888888888888708888888888502088884B
:10638A0088A8A8A85088885020508888888888506B
:10639A00202020F80810204080F800CCAC9CACCC1F
:1063AA000000CCD4E4D4CC0004781828C800FC40FF
:1063BA00A04018202018000000000000F80000008B
:1063CA0000A040A05000788888986870884030887B
:1063DA0070200000F0A8A8A8A878484848487888FB
:1063EA0070888080887020A88898A8C8888880507B
:1063FA0048FC485080304C5C6060603C00E0F0082B
:10640A000808F88044485C484480F880808080808E
:10641A008078484848484888B8A8A8E8A8A8B8880A
:10642A0088888888F808500070888888708080F08A
:10643A0088888888F8888888888888F090909090DA
:10644A0090F0A8A8A8A8A8A8F8888888F808080832
:10645A0050008888888878A8A8A8A8A8F808000002
:10646A000000000000000000000000008888888802
:10647A00E8A8E8A8A8A870A8A8A80000000000003A
:10648A000000000000000000000000000000000002
:10649A000000000000000000006000606000600072
:1064AA0060006060205020000000005090B890D03A
:1064BA0090886050500070705000882020887000CA
:1064CA000080C0A090F8003048B4B448300030488A
:1064DA00B4B44830FC0098D02058C800F8E8D880F6
:0A64EA00D8E8F8404050F850404058
:0300000002005E9D
:03000B0002B62614
:0C000E00206E06859950D26E32D26F32FF
:0E00230010990AC298206DE385994FD26D3274
:10003800E4F537F534F52F12DE6AC229C22AC26800
:09004800C227C214C215022D9C4E
:03005B00022B2A4B
:10B619008530F0C5F065308530F060F722C0D0C0C4
:10B62900E0C0F0C0A775A700C083C08275D00875B7
:10B639008A00300503758A7A758CEA0532E532701D
:10B649000215320530E530640A6026201520E531FF
:10B65900B40C0BE530B4010612BAA112D91DE531BB
:10B66900B4180BE530B4060612BAA112D91D02B8F6
:10B6790040C2AFD2C075C07AD2AFF5300531E531DD
:10B6890064197040F531201529C225C22C7D0A7430
:10B699000412DF1BEF33EE339005CCF0EE24F540B6
:10B6A900112402400B24014005DDE4022B2AD22596
:10B6B900D22CE5A6600215A678B5E660011678B623
:10B6C900E6600116302E0BE5367007C22FC22E1226
:10B6D900B9CEE5367004C24B8002153678A9E6600A
:10B6E900011678D8E66001160535E535700215357D
:10B6F900E590307B0B30E008D278C27BC200801A1B
:10B70900307C0B30E108D279C27CC201800C307DDB
:10B719000930E206D27AC27DC202E59044F8F4709B
:10B7290003753500304A09E53324FA5003753305AA
:10B73900E5336005153302B7E5E590F45407700366
:0DB7490002B7E5A2E09200A2E19201A2E2A7
:10B75600920230100320143D75330820001B201080
:10B766000C2011098013E59030E10E8006E53724A0
:10B77600FC40F3E543541FF53320100375A6FF2064
:10B786002E5D301004E536705620100C201109E5A8
:10B796003524F55003753304D21BD2A5D2A612B9AF
:10B7A600CE75B44075B24078D8E6700205342027CD
:10B7B6002E20682B202928202A25A2107211501F1E
:10B7C600E52054076019E53424375004C24A800F37
:10B7D6002401400B200026200119D27D7534C82093
:10B7E6001558E531702412DEFB74E812DED4802A87
:10B7F60002B913E53724FC40E6D27C80DF3011DF46
:10B80600E53724FC40D9D27B80D275F00384E5F07D
:10B8160070DE12C55074E812DED4E531B4060512A6
:10B82600C6C88016B40C0512C6DE800EB412051208
:10B83600C6C88006B4180312C6DEE59030E10530AE
:10B84600E202800620100820110520103C807D2091
:10B8560027F82068F52029F2202AEFE53424304025
:10B86600E9240750E5600B205E088590F020F2027F
:10B87600740190B88893D2A5201002C2A512B9B956
:10B88600806FC8A08269554646202F12E536603C77
:10B8960024AA500AE53675F01984E5F06040D2A670
:10B8A600201002C2A6D2A5202F0C7418304B0274A9
:0EB8B6006412B9B9803BE53675F00C304803DA
:10B8C40075F00684A2E0744640E9743780E5E52B00
:10B8D4005403600C20100E301106E54A6402600522
:10B8E40012B9D4800312B92B101B08A25892A5A236
:10B8F4005992A675A700D082D083D0A7D0F0D0E00B
:10B90400D0D0201009C5A67003022B2AC5A632C2C6
:10B9140018B40202D21812C5EE30180874E412DE0C
:10B92400D402B82002B81B78A7E5B4600924E0402B
:10B9340005760002B9D4E534702920412220751F10
:10B94400300D1CE57924CE40167AFFE5B110E701ED
:10B954000A2325B3F5B3EA35B4F5B4C313F5B2E657
:10B9640060021622C2412075028075E579FF605895
:10B9740020120424FD5051206502C21CD265FF240C
:10B98400B050027F4FEF90BA519375C70375C6FC50
:10B9940075B90185BFF0A4E5F0F624F44002760CF5
:10B9A400301C2DE5BEC39FF5F0A4E5F024E0400370
:10B9B40075F020E5F0C21C79AA770375B300F5B4DD
:10B9C400C31375B100F5B222C26578A77680D2415F
:10B9D40079AA7703D21CE4F5B3F5B4F5B1F5B22234
:10B9E400C26579A1E57924CE500DE720E7E27628F7
:05B9F400301CDD74327F
:10B9F90080BE7680E720E7D3E5799740CE79AAE73C
:10BA0900FAE5792323B4C500400274C42437300E03
:10BA190031F42437300D15F7BA0302FA0AC39AF53F
:10BA2900B175B300EAF5B4C313F5B222101C07D2FD
:10BA39001C76C802B9BB763274FF200E02749B02D1
:10BA4900B9BBC313247E80CCFFF3E8DDD3C9C0B8EA
:10BA5900B0A9A29A948F8A85817D7975716E6B6878
:10BA690065625F5C595653504E4C4A4846444240C1
:10BA79003E3C3A383634333231302F2E2D2C2B2A96
:10BA89002928272625252424232322222121202071
:10BA99001F1F1E1E1D1D1C1CD2B5C28EAE8DAA8D68
:10BAA900AF8BAB8BE4F58DF58BD28E3014012278F8
:10BAB900B6BE0007EF24E24002800806E624EC50F7
:10BAC900027614206705E624F64005E4FEFAFFFB3A
:10BAD9007C007D0A12534F7C007D5E12546F8F519A
:10BAE900EE60037551FFEAFC7A33125363EBF5F00C
:10BAF900A4E5F0CB8CF0A425E0C5F035E0CB92D5D8
:10BB090025F050060BBB0002D2D530E7060BBB006F
:10BB190002D2D5ECF5F0A42BFBE5F03400FC30D5CE
:10BB2900010C78A6E6C39BFF18E608F6EB18F61891
:0EBB3900E69CFE18E608F6EC18F63014012221
:10BB47007A0050040A1255E67C007D6E12546F8FFE
:10BB5700F078A2E6A4FBACF0125585EBBA0002F42C
:10BB670004FAE4F8FFEA30E70118E5796006207582
:10BB7700031FF4042AF579EF38D27520E70860032C
:10BB87007579FF02C821C2750470F5E579F4046080
:10BB9700EFF57980EE120E5D78BBA6BC120E7BE541
:10BBA700BE78A2F624F65007E4F5BEF6124EE6126A
:10BBB7000D46E5BEF54824F65008E4F5BEF54812F3
:10BBC7004EE6E5BFF54324F3503924F34035120E12
:10BBD7007178A1A6BCE5BF789DF61424FB500874C4
:10BBE70003F6F5BF124EE678B7A6BE120E67E5BD9F
:10BBF700A2E39266A2E49267035403C253B401021C
:0EBC0700D25322740DF5BFF543124EE680C0F5
:10005E0078FFE4F6D8FDF4F5A6D2B4D2C075C07A16
:10006E0075D75075AE1375AF017581D87590F8754B
:10007E00EFBC75FDFFD2A412DE41C2A47450122B48
:10008E0042758951D28C75A882D2BC12BC1512DE73
:10009E00FB12C4C612BB9C12D9D0122A087F407E16
:1000AE0001909C73127702124D4A12DE4112DB222E
:1000BE0012DD5912DE6A7C1412DE4B300003022B65
:1000CE002ADCF512489F753A001248EDE53A701693
:1000DE0012DF2F7F437E0690A40B12770212DD599A
:1000EE003000FD022B2A75A6FF12489F12BB9C12F0
:1000FE002A0812DD5912DE3D12DE6A78B5761E121E
:10010E00D9D012C4BBC215C214122A08909CBA7F51
:10011E00781276F0205E0A7F767E12909CC712D5FA
:10012E00477F4012DDCF7F497E0978AEE612D3B30A
:10013E007E15743A12D51B7E1AE53E12D3B37E2677
:10014E00743A12D51B7E2BE53F20E00805A6E5A6E6
:10015E00700215A6E53F12D3B37F5312CA367F57EE
:10016E007E0B12D2E012D3687F6020730302020866
:10017E007E0BAC5DAB5C12D2E412D3687E3112778B
:10018E008D7F697E1212D86B3025087E1290DB8B24
:10019E0012D547E5A60303543FFDFE0D7F7312DE15
:1001AE00740F12DE741EDDF478B5E57124F640028C
:0801BE00761E307419E660564C
:1001C6007F727E16744012D4E97E17E612D4717ED1
:1001D6001F745312D4E912DD59100037100137107D
:1001E600023712483FD2AC75369612DBD1B4E00521
:1001F600124935800AE53670F112488D12DE3A0250
:10020600010D2074097E2BE52E540712D5087E17A2
:1002160002018C022B2A022D628072E53524C85019
:1002260049E59020E244D0E0D0E012027102735614
:10023600E53524D25034E59020E22FD0E0D0E0120C
:10024600DF2F8038E53524D25020E59020E21BD000
:10025600E0D0E012DF2F306B0B7F091276E7124FEA
:100266001E127BBD1202710206BE2212DF2F90A45F
:10027600C37F001276F012DD5902DE3A12DF2F90AC
:10028600A4C37F001276F012DD5912DE3DC215C2FC
:1002960014C227C26812DE6A753701909DA4121C2B
:1002A600FF9002AB730200F70217C2020B56021F41
:1002B60012021F0E0206BE0206FB0273560202C699
:1002C60012DE6A75370790A14F121CFF9002D67393
:1002D60002029302096B0209A50209D90202FA0277
:1002E60005AD0202C60202C60203180202FF024B55
:1002F600B30203261248F0805A7F517E00747212B0
:10030600D517121E5C40B9124E3512D9D012BB9CBD
:1003160080AE7F49A25E120D31925E120D5080A012
:100326007F64120E9E121E5C401DE5352480F47516
:0C033600F0198460157F727E1F12D5083C
:1003420012DD591001E810000280E30202C612BC5D
:10035200820202C6124EE612DE6A75370290A3329C
:10036200121CFF900369730202C6020EA8020F0D4F
:10037200020F61020FB6020FFA02100902035902BC
:10038200051302038980D0D21412DF2F7F147E0559
:1003920090A37C127702121E1912DD591248687559
:1003A200A6FFD2AC1000DE12DBD1204CF2B405EF76
:1003B200E4F511F514F5151204411204D51248683A
:1003C20075A6FFD2AC1000BD12DBD1204CF2B415E1
:1003D200051204C880E7B406E712047FE51424FC82
:1003E20050D5E4F56FF56EF56D12048B1204D5123B
:1003F200486875A6FFD2AC10004212DBD1204CF245
:10040200B415051204C880E7B406E71204B5E56F17
:1004120024F050D5124868743B12DC4D7A47909C08
:100422006A1224C9742A12DC41909C731224C97482
:100432002A12DC41DAF912DC6A12DE4B020359ACF1
:1004420014AB157A0412536375A704900400E4F008
:10045200ECF0EBF08514C78515C67F08120467DF40
:10046200FB75A7002275B901E5BCF0E5BDF0E5BE5C
:10047200F0E5BFF005C6E5C6700205C722E5152402
:1004820008F515E43514F5142275A704900400E567
:100492006F4410F0E56EF0E56DF0740312BC4E7F10
:0404A20020E4F5F766
:1004A600C2B2C2B2E5F7F0DFF4D2B275A700227489
:1004B60020256D54E0F56DE4356EF56EE4356FF587
:1004C6006F2205117F287E00E51112D42A8006903E
:1004D6000402E070177F287E15900400E012D42AEB
:1004E6007E2A900401E012D42A12DD59124868745B
:1004F6003A12DC8475A7009004007F23E0A312DC87
:1005060020DFF912DC5B3099FD2202035912DF2F3E
:100516007F0F90A6B61276F0121E1912DD59C2147C
:10052600C21512DE3A7510651000DFE53170F9E587
:10053600106465700D855E14857A15E4F512F51361
:10054600800C78A8E51326F513E43512F5127F1E04
:100556007E19E51012D3D0C3E57A9515F517E55E39
:100566009514F5167F287E0BAC16AB1712D2E41243
:10057600D36812DD5912DE4BD510ADAB17E516FC6C
:1005860030E7031255F67A0A79001253DCA912A84D
:1005960013125515EBF510243840037510C8120ECA
:1005A6005D8510BC02035612DF2F909CFE7F017EF4
:1005B60009127702909D077F0A7E091277027F1340
:1005C60012CA2E751700120E6CE5BC12068DE5BD1B
:1005D60012068DE5BE12068DE5BF12068D909D575B
:1005E6007F5F7E06127702121E9E12DD5975170076
:0605F60012066D10000862
:1005FC0010011510024880F20517E51724F7500377
:10060C0075170075100080E2E51764087015120E5E
:10061C006C75BC0175BD2375BE4575BF67124EE682
:10062C000205ADE51012069F12DD5912064D05109C
:10063C00531007E51724FE400353100380AC02024D
:10064C00C6A9BCAABDABBEACBFE5171304F8E64007
:10065C00085407C42510C4800454702510F6027D7C
:10066C00A17800E875F009A42417FF7E3B7D20E8F3
:10067C00651770027D89ED12D51B08B809E502DDFE
:10068C0059F8C4120693E812069F7E030517E51766
:10069C0002D508540775F009A4909D0F2582F582A8
:1006AC0050020583E51775F009A42417FF7E0C0290
:1006BC007702C26812DE6A753705909EE8121CFF3D
:1006CC009006D073020293027941027986027B1C58
:1006DC000206BE0206F4027A5E027AC402178B028C
:1006EC0006BE021771020C627F2E12168680C31290
:1006FC00DE6A753706909FC7121CFF90070B7302BA
:10070C0002930217C802182A0218A30219700219C0
:10071C00A2021A19020750020749021A62021B07A9
:10072C0002072F7F64120E67E5BDA2E7120D31128E
:10073C000E67E5BD92E7F5BD124EE680B27F491219
:10074C00168680AB12090C122B6912DF2F121DF3C7
:10075C00E55804607790A0971207F912871E12DDF6
:10076C005910000810011310021C80F50559C3E53F
:10077C0058955950D575590080D01559E55930E721
:10078C00C985585980C4E559B40F02802FB51F0292
:10079C00802A75F007A42408F51775162774B82558
:1007AC0059F987001207E712DD59100028100128AB
:1007BC0010020280F574B82559F9A700E53524FA22
:1007CC00508878C7A64812090312DF2F12DD591280
:1007DC00DE3D0206FB1880CC0880C9E875F005A444
:1007EC0085F01CF51BC000125C7CD000221287AF78
:1007FC00B4FF0122751000751FFF1287C6E5106447
:10080C000F6017120830401274B82510F8E675F016
:10081C0005A485F01CF51B125D0D0510C3E558955C
:10082C001050D7221211AEF8602E6404602AE8141E
:10083C00B51025F51F120E7BE5BC70060475F0147F
:10084C00800375F019A485F01CF51B125D0D7E223A
:10085C0090A657127735D322C322E558B4FF012254
:10086C00751000E510640F602EE51075F007A424D8
:10087C0009FF74B82510F8E61208ED75F00A84C06B
:10088C00F07E2012D4717E28742C12D4E9D0E07E34
:01089C002A31
:10089D0012D4D61208AD0510C3E558951050C322D9
:1008AD001211AEF8603964046035E8146510702FCC
:1008BD00120E7BE5BC1208EDF8C313923D7E1C129F
:1008CD00D4877E28742C12D4E9E4303D067405B823
:1008DD000001147E2A12D4D67E18742312D4E92274
:1008ED00305D1275F036A42432FBE435F0FC125560
:1008FD0085125585EB221209151276D5DFFB2212D2
:10090D000915127EB1DFFB2275C70375C6F078B8E5
:10091D007F042275C70375C6F375B901E5BFB548E8
:10092D0031E55924F1402BE55975F00484A9F024E3
:10093D00F0F5C675B901C5F0A9BC600CA9BD146070
:10094D0007A9BE146002A9BFE975F005A4F985F0E9
:10095D00CC22120E7BA9BD75CC0022124EE612DE02
:10096D006A75370390A1C0121CFF90097B730202B8
:10097D00C6020C7B02131F020C90020C9B0216E6A2
:10098D000213A6020D5C0213DA02142002173802BC
:10099D00138E021465124EE612DE6A75370490A2AC
:1009AD0088121CFF9009B5730202C6020CAA020C34
:1009BD00B50209A5020CCB020CD60210230209A523
:1009CD00020CE5020CC0020CFF124EE612DE6A7537
:1009DD00370B90A2D9121CFF9009E9730202C602CF
:0B09ED0010D10210D1020A6F020AAD07
:1009F800020A10020A330217CE02117602123E02D0
:100A080011E70212CF020D19120E67E5BF1470C16B
:100A18007F2E120E9E1F120E67E5BDA2E6120D3143
:100A2800120E67E5BD92E6F5BD80A37F37120E9ED4
:100A3800120E62A8BFE8120A6712DD5910000810EA
:100A4800010D10021280EE18B802EA780A80E60852
:100A5800B80BE2780380DE120E6288BF0209D67FE7
:100A6800367E2CE802D3B97F1C120E9E120E67A8A0
:100A7800BE120AA112DD5910000810010D1002144F
:100A880080EF18B800EB780B80E708E824F450E111
:100A9800780180DD88BE0209D67F1B7E35E875F0B7
:100AA80005A402D3B37F25120E9E120E67A8BF12AB
:100AB8000ADF12DD5910000810010D10021480EF32
:100AC80018B800EB780980E708E824F650E17801C7
:100AD80080DD88BF0209D67F247E3BE802D5081254
:100AE8000E5DE5BF75F03CA4ACF0FDE5BE75F00504
:100AF800A42DFDE5F03CFC120E67E5BF14603675C9
:100B0800F005A485BEF0A42DFFE5F03CFE7C007D39
:100B18003C12547CC005EF75F01884E5F07F2D7EFB
:100B28002412D3B37E30743A12D51B7E35D0E0122E
:070B3800D3B302DD597F2D4C
:100B3F007E0590A679127702120E67E5BDA2E67FB9
:100B4F002D12161502DD59D25712DF2F121DF31277
:100B5F000B640202937F177E02909E051277027F2D
:100B6F004C7E02909E1B127702AC5DAB5C7F577E72
:100B7F000412D360120E8A85BC6285BD63E56124C1
:100B8F00F84044909E267F371276F0AE61AF607CBE
:100B9F00017D5E12547CC3741F9FFAAC63AB62EC91
:100BAF0033921750031255F6125363AB047C003087
:100BBF0017031255F674F52BFB74033CFC125339D3
:100BCF007F377E1512D2D8909E337F697E0F1277B2
:100BDF0002E560240FFBE43561FCA25C923BD25C22
:100BEF007E1E12D2E4A23B925C7E30742012D51B83
:100BFF007E36742012D51BE5602562FBE5613563F7
:100C0F00FC7F227E0412D360E56245637016742E5A
:100C1F007E3A12D51B12DD5910000D10011510026E
:100C2F0026020B8C742080E81562E562B4FF0C1568
:100C3F006380080562E56270020563E53524F550AF
:100C4F0003753301020B8C120E8A8562BC8563BD5E
:100C5F00024EE67F637E00747212D517121E5C403F
:100C6F00087F631276E7124EED0206BE120E71E593
:100C7F00BCA2E77F0A120D34E5BC92E7F5BC02096E
:030C8F00687F1C5F
:100C9200A20D120D31920D80097F25A20E120D3187
:100CA200920E120D5002096B7F0AA20F120D3192A1
:100CB2000F802A7F13A208120D319208801F7F52E3
:100CC200A20C120D31920C80147F25A20B120D3151
:100CD200920B80097F2DA209120D319209120D503B
:100CE2000209A57F49120E67E5BDA2E3120D31127A
:100CF2000E67E5BD92E39266F5BD0209A27F5B1223
:100D02000E67E5BDA2E5120D31120E67E5BD92E553
:100D12009243F5BD0209A27F6D120E67E5BDA2E006
:100D2200120D31120E67E5BD92E0F5BD0209D61231
:100D32000D468F1F9217120E9EAF1F1F7E3912840F
:100D42000BA21722120E7685BC2B85BD2122120E14
:100D520076852BBC8521BD024EE6203714120E711A
:100D620085BE12120D89120E718512BE124EE680D8
:100D7200057F3F120D7B02096B7E0390A252127710
:100D82000212DD5902DE3A75A6FF12DF2F12B619E2
:100D9200740712DF1B8FF0740612DF1BEF2512C3DC
:100DA20095F0A2E7923D4010FD24CD50027D32AC79
:100DB20005C3743F9DFD800FF404FD24C850027DDD
:100DC20037AC0574402DFD7F4012CA2E7E1212DE12
:0F0DD200740EBE1EF91F303D020F0FEF6D70ED56
:100DE100E536700A753606EC2513F5148C13120ED0
:100DF1000712DD59100007100108300207221512F1
:100E01008002051280827F377E28742E12D51B7FC7
:100E1100347E21740A303D010412D536E514FC24D8
:100E21009C50027C637F347E2DEC12CE5A7F437E30
:100E31001E12D2E07E00E51212D4777F057E029069
:100E4100A25C1277027F6D7E0190A2671277357FD7
:100E5100747E0490A278127735021DF375C6F48072
:100E61003575C6F5803075C6F6802B75C6F78026B8
:100E710075C6F8802175C6F9801C75C6FA8017758C
:100E8100C6FB801275C6FC800D75C6FE800875C64E
:100E9100FF800375C6FD75C70375B9012274721F02
:100EA10012D5170F02DD597F0A120E9E7E2A1248B3
:100EB100F0120E7BA8BF120EDC10001210010510FB
:100EC100021580F508E824E750EC781880E818E866
:100ED10030E7E3780080DF88BF805F7F097E05907F
:100EE100A53AB80C0390A5341277027E27E53D2878
:100EF100240C75F01884E5F012D3B37E33743B12E1
:100F0100D51B7E35E53E12D3B302DD597F13120E98
:100F11009E120D46120F3E10000810010510021717
:100F210080F2105C07205D0BD25C80E8105DE5D299
:0D0F31005D80E1D25C80DD852BBC020356A3
:100F3E00205C10205D1890A58D7F127E2312770203
:100F4E0002DD5990A5A1205DF090A59480EB90A5AF
:100F5E009A80E67F1C120E9E120E76A8BF120F9874
:100F6E0010000810011110021A80F2E824F250034A
:100F7E001880EA780D80E6E824E740030880DE78E2
:100F8E001980DAE8F5BFF54380A37F1B7E26E412B5
:100F9E00D508E82323B464087E26740112D508E42C
:100FAE007E2E12D3B302DD597F25120E9E120E85B0
:100FBE00A8BCE8120FF112DD5910000810010D1037
:100FCE00021F80EEE824E050E9188006E824CF40A6
:100FDE00E108120E8588BC124EE6D21512D9D080C9
:100FEE00D180157F247E3724E202D4247F2EA20ADC
:100FFE00120D31920A120D500203597F37120E67ED
:10100E00E5BDA2E4120D31120E67E5BD92E49267C2
:10101E00F5BD0203567F367E00747212D5170F7E11
:10102E0016743F12D4E9120E71A8BD12109C12DD77
:10103E005910000810010510021080EFE8248750A7
:10104E0004240A800224E8F880E17F377E1674209B
:10105E0012D4E97E2C743F12D4E912109C12DD5981
:10106E0010000810011410022080EF18B80904783F
:10107E007880E7B878E478E780E008B87904780AF1
:10108E0080D8B8E8D5787980D188BD0209A2E82445
:10109E0087923DE8500224917F367E30C313923BF7
:1010AE0012D4247E3CE4303B02740512D5017E1A24
:1010BE0090A481303D0390A4851277027F3C7E3A46
:1010CE0002DE747F127E00747212D5170F7E2074AA
:1010DE003F12D4E9120E5D85BE1085BF1112115854
:1010EE0010000810011110021B80F21511E511B449
:1010FE00FFEB75111780E60511E51124E850DE753A
:10110E00110080D91211587F137E20742012D4E959
:10111E007E31743F12D4E912DD591000081001110E
:10112E0010021B80DF1510E510B4FFD875100B8070
:10113E00D30510E51024F450CB75100080C6120EA6
:10114E005D8511BF8510BE0209D67F127E24E51182
:10115E0012D3B37E30743A12D51B7E35E51075F07E
:10116E0005A412D3B302DD597F49120E9E1211AEA1
:10117E00F81211B410000810010D10021280F218AE
:10118E00B8FF02780480EA08B80502780080E212FF
:10119E000E5D88BD124EE6B800030209D902123E5A
:1011AE00120E5DE5BD227F487E0590A49B1277024C
:1011BE00E8601CB4040A7E0590A490127702800C9D
:1011CE0090A4A71277027E38E812D50802DD599056
:1011DE00A4A27E2912770280F31211AE601D640460
:0211EE00601986
:1011F0007F5B120E9E120D46121219120E7610000F
:101200000B10010810020C80EF0209D9105FE9D21F
:101210005F80E5852BBC0209D61211AE601F640405
:10122000601B7F5A7E0590A49B1277027E2390A4B8
:10123000AB305F0390A4B212770212DD5922121173
:10124000AE70030209D97F527E11120E9E120E7BE0
:10125000A8BC12127E120E7B1000081001081002AA
:101260000880EF1880EC0880E9120E7B88BC124ED3
:10127000E6120E85E875F005A4F5BD0209D6121137
:10128000AE604BE875F03270040475F028A4ADF040
:10129000FC305D11ACF0FB7A8A125371EB30E7053C
:1012A0000CBC00010DAE05AF047C007D6412547CC3
:1012B000C005EF7F517E1A12D3D07E2C742C12D52C
:1012C0001BD0E07E2F12D3B31241B712DD59227F1B
:1012D00064120E9E120E7BA8BD121300100008109F
:1012E000010F10021680F218E824CD50EC783280FD
:1012F000E808E824CD50E2780080DE88BD0209D6F7
:101300007F63E823C2E012CF8D75F06484C0F07E65
:101310002612D5087E2C742C12D51BD0E080A47F19
:1013200013120E9E120E71E5BCA2E7923DC2E7F8C1
:10133000E812135E12DD5910000810010D100212A0
:0313400080EE1824
:10134300B800EA783280E608B833E2780180DEE854
:10135300A23D92E7F5BC79A1F78079547F305C0117
:10136300237F127E2375F00A84C0F012D4247E2DCD
:10137300742C12D51BD0E07E2F12D5010F7E359031
:10138300A5A7305C0390A6030277357F64120E9EF7
:10139300120E7BE5BE7F637E2C128460F5BE79A2BC
:1013A300F780317F37120E9E120E76A8BC530003CE
:1013B3007F367E32E812D50812DD5910000810017D
:1013C3000710020780E718180880E2E5BC54FC48C0
:1013D300F5BCF52B0209687F49120E9E120E85A8F3
:1013E300BE12141112DD5910000810011110021A57
:1013F30080EFE8240AF8242450E778DB80E3E8242C
:10140300F6F8247F40DB788180D788BE80C6E8F475
:1014130024DC75F00A847F487E3B02D5087F521294
:101423000E9E120E85A8BF12145812DD5910000823
:1014330010011110021A80EFE82408F8245750E72E
:1014430078A880E3E824F8F824A040DB786080D70C
:1014530088BF0213D7E8F424A923C47F517E3B023B
:10146300D508122C74754A00D210C211D214D27549
:1014730075791475340012DF2F7F007E0290A2333A
:101483001277029041E07F087E2612D547E52B5460
:10149300030F7E3912D508121E0E12D1B1128ED14E
:1014A30012DD5910000810011A10022480C520759E
:1014B30004057980BE1579E579B4FF05C2757579A0
:1014C3000180B02075EB1579E57970A7D27580A3FB
:1014D300C210C21402096B120E76E5BE7F097E3A72
:1014E30002D508120E7BA8BF120EDC120D46120F96
:1014F3003EA8BF120F98120E85E5BC120FF17F2D87
:10150300A20A1216157F36A267121615120E5DE592
:10151300BC7F487E3202D42A120D467F1BA20D12D5
:1015230016157F24A20E121615120E71E5BC1213A6
:101533005E7F09E5BCA2E7121615A8BF121724E5C2
:101543002B54037F367E3212D508120E7BE5BE7F05
:10155300637E2C12D508120E85A8BE121411A8BFE3
:10156300121458120E67A8BC021769120D467F09A0
:10157300A20F1216157F12A208121615120E67E596
:10158300BDA2E37F48121615E5BDA2E57F5A1216E8
:10159300157F51A20C1216157F24A20B1216157F6C
:1015A3002DA209121615120E71A8BD02109C120E5F
:1015B3005D85BE1085BF11121158120E67A8BE12A9
:1015C3000AA1A8BF120ADF120AE7120E76E5BE7F50
:1015D3003F7E3A12D508120E62A8BF120A67120E96
:1015E3005DA8BD1211B4120E7BA8BC12127E120E9E
:0415F3007612121941
:1015F700120E7BA8BD121300120E67E5BDA2E07F95
:101607006C800B7F098040120D467F48A25E744EA6
:10161700400274597E3A02D51B127DAD7F73127A50
:101627000B127DFC7F6C127A1A7F2D801A120E67BF
:10163700E5BDA2E77F63121615120E76E5BE7F0998
:101647007E3A12D5087F4812166EB40104BF09010D
:10165700E4F51075F005A47E1E909F982582F5820B
:1016670050020583027702120E67E5BD035403C2D9
:1016770034C25330E103D2342230E002D253221273
:101687000E9E1F12164E12DD59E5101000121001A2
:101697000610020280ED22045403B4030AE4800713
:1016A700145403B403011423C5BD54F925BDF5BD76
:1016B700124EE680CE1275D1EBF516F5147F6C123B
:1016C7007A1A1275B57F647E23E51612D487C3E5AF
:1016D700169514F5167F73127A0B7F2D02164E7F1F
:1016E7002E120E9E120E71A8BFE824FA400330375F
:1016F70002780312172412DD5910000810010D108B
:10170700021280E518B800E1780580DD08B806D92F
:10171700780180D5799DE8F7F5BF0209687F2D7EAE
:101727002C7420B80502742E12D51B7E32E802D520
:0C173700087F5B120E9E120E67A8BCE833
:1017430012176912DD5910000810010D10021280E2
:10175300EE18B800EA780380E608B804E27801805E
:10176300DE88BC0209687F5A7E2CE802D508D2685D
:1017730075480A1248F0D214122B77127EE5123301
:10178300CFC26B12024A80F3D214751501127D6722
:1017930075B901E5BC20E71C127E9775A6FF127E82
:1017A300F1121E1912DD5912780B10000F50051299
:1017B300793380E70515E515242050D10206BE12C2
:1017C30017D40202931217D40206FB1217D402098C
:1017D300D91217E0120E768548BE024EE6122B6927
:1017E300122B83125A3612DF2F90A040D249128750
:1017F3004B128704121DC912DD5910001410010584
:1018030010021B80F50548E548640A7002F548801C
:10181300CF1548E54864FF700375480980C28548C1
:1018230049122B83E558221248F0122B6985484947
:10183300C250E558B40F02D250125A36803AD2271A
:1018430075480A122B77125A3612DF2F12866E90C2
:10185300A45220290390A45D121E8BC26A1233CFB7
:10186300106A0280E1C227127D3F854948121C3667
:10187300122B83D229125A3612DF2F909F551287CB
:101883004920500E121E7512DD591000101001AEC2
:1018930080F8121E1912DD5910000280FB0206FBAC
:1018A300122B69E55830E7137F1B90A43D7E051288
:1018B300770212DD5912DE3D0206FB122B83125A08
:0A18C3003685594912DF2F121E036B
:1018CD0090A45D12874912870E12DD591000081081
:1018DD00010A10020C80F512193B80DB12194880A9
:1018ED00D612DF2F121E0390A05012874912870EB9
:1018FD0012871212DD5910000810010A10020C8017
:10190D00F512195480DB12196280D6121BFC122BB2
:10191D0083125A3612DF2F90A3A2128749121E414D
:10192D0012DD5910000510028880F80206FB0559DA
:10193D00C3E55895595003755900221559E5596459
:10194D00FF7003855859220549D3E5491495584030
:10195D0003754900221549E54964FF70058558490D
:10196D00054922122B69E55830E7057F240218AD91
:10197D00122B83125A3612DF2F90A05B1287491259
:10198D001E8012DD5910000A10010280F8121CA5EC
:10199D0080DE0206FB122B69E55830E7057F2D022C
:1019AD0018ADC26B7559FF125A3612DF2F121DF387
:1019BD00E55930E703121E0E90A06C12874912876D
:1019CD001E12DD59E55820E7061000081001111010
:1019DD00021B80F00559C3955950CF7559FF80CA28
:1019ED001559E55964FE70C285585980BDE55920D9
:1019FD00E711D26B75A700758307C4F582E0B2E7D6
:101A0D00F080A7306B03121C530206FB122B69E505
:101A1D005830E7057F360218AD122B83125A361255
:101A2D00DF2F90A077128749121E5C4009121C9A75
:091A3D00121CCF121A460206FB2E
:101A4600120E7BE5BD75F00584F5BCF5BDF5BEF55A
:101A5600BF120915124EE605C6DFF922122B69E5FB
:101A66005820E7087F5190A0810218B012DF2F900E
:101A7600A468128749121E1912DD5912484FD2ACBA
:101A860010001FE55830E7F8306DF5121B9C7E20DC
:101A96007F00501390A4B912773512DD5912DE3D3E
:101AA60080CAC2AC0206FB1B8B13909F721277355D
:101AB60012DD59C26B7B007514B8121C8F127E663C
:101AC600127E185025A814E824384004A6010514EF
:101AD6000BC3E5139B50E678B8121CD1306B03128A
:101AE6007BBD122B83125A368082127DADE51660BD
:101AF600E6D26B127EC3C003127D7ED003A9158089
:101B0600C4122B69E55830E7057F5A0218AD122B2F
:101B160083125A3612DF2F90A08C128749121E3676
:101B260012DD5910003510010280F8754605121BAA
:101B36006450157F007E357407954612D48712DDF2
:101B46005912DE3DD546E7D390A473500390A4B94D
:101B560012874912DD5912DE3D80B30206FB124898
:101B66004F12DC73745212DC84745412DC41E55853
:101B76000475590012DC621277BA4016127D3F12C4
:101B86007E9712780B400B0559C3E558955950ECD2
:101B9600C322C2ACD32212484FD2AC12DBCC204CAB
:0D1BA600F1B440F712DBD1B4400312DBD1E3
:101BB300B452E2F53812DBD1B454DA12DBD1FA6055
:101BC300D424EF40D012DBD1E53870C912DBD11237
:101BD300DBD112779F7B007E031278965010205042
:101BE300B412DBD1204C03B440F7DEED80A7127EA4
:101BF300760B12779FDAE0C322121CE0E55924C862
:101C0300F88602E54924C8F9986013146010500F50
:101C130018E608F618E86970F7A702121CCF22E548
:101C230059640F60F91908E618F608E86970F7A710
:101C33000280E8121CE078C8C250E6B4FF028007B5
:101C430008B8D8F6D25022B8D702D250A615807C55
:101C530078B8121CE2E4F9F5A7758307E9C4F582A5
:101C6300E030E70AE924B8F82438400276FF09C3D4
:101C7300E5589950E7121C9A78B879C8E6B4FF0280
:101C83008002F70908E8243850F2804079B877FFDA
:101C930009E9243850F82279C877FF09E924285044
:101CA300F822121CE0C23D78D7B6FF04A900D23D4A
:101CB30018B8C7F5203D0279D81978C8B6FF0122B4
:051CC300C3E899500781
:101CC800C6C7C6081980F478C8121CF1127ED31250
:101CD8007ED3127ED3027ED378C8121CF1127EB155
:101CE800127EB1127EB1027EB175C703E54875F068
:101CF80004A42480F5C62212DF2FC23C1276F4E534
:101D080037605314604D14604514603D14603514F9
:101D1800602D14602514600E14600B14600D14609F
:101D28001414600C803012160E802B1216BC8026FC
:101D38001215B1802112160A801C1216348017124F
:101D48001620801212156E800D12151B80081214B1
:101D5800E680031214DA12DD5912DE41121DF31265
:101D6800B9DAA81F08E814C23BB51D02D23B75F0CA
:101D780007203C0375F009A4FF7E00303C0C74205A
:101D8800303B02743E12D4E9800A740B303B027473
:101D98000A12D501D8CF12DD59E51D10000810012F
:101DA8001010021880B9651F7003751DFF051D808E
:101DB800AE7005851F1D80A7151D80A375F003A4AF
:101DC800227F7B7E0090A3BA127735E54824F6403F
:101DD800087E0A90A42012773522127A377E05747D
:101DE8005B12D4E57E1D745C02D4E5121DE27E34DC
:101DF80090A3CB027735127A378003121DE27E3129
:0E1E080090A3CF027735121DE27E3190A4C464
:101E1600027735127A377E008005127A377E2D904A
:101E2600A4C4027735121E367E31909FAC027735F8
:101E3600121E197E1A909FB1027735121E1980C0A4
:101E4600121E197E18909F5F027735121E197E1A90
:101E560090A4C9027735121E197E1A90A4CE127765
:101E66003512DD59D3100006C310010280F6221286
:101E76001E197E1A90A04A027735121E197E1890F6
:101E8600A0650277357F007E2012773502DD591274
:101E96007A3790A4D3027733127A3790A4E4027784
:101EA6003312BE9C120E94E5BDF55EF56CE5BCF5ED
:101EB6005FF56B756A007561FF75A70490070012E0
:101EC600BE46B4FC23E582C313F561E56CF0E56B11
:101ED600F0E582600F12BDBDE56C655E70E1E56BF5
:101EE600655F70DB75A700223024EA0460E7240FE3
:101EF60040D380E1E560758307C333F582E0A3F53F
:101F06006CE0F56B756A0022D2248002C224D214DA
:101F1600C21F121EA7756000E561B4FF1612DF2FFF
:101F2600909E367F0A7E0512773512DD5912DE3A0B
:101F3600020293C210C21112DF2F121DF3301F0AC4
:101F46007F07909E4412773380647F007E01C3E54D
:101F56006012D4877E0E742812D4E5856048740713
:101F6600F51FFF7E00743E12D4E9E548121EFC12EE
:021F7600C83D64
:101F78001224D80548C3E5619548FD401CE51F2497
:101F880007F51F24C850E17F387E01ED0412D4877D
:101F98007E0E742912D4E5800DE51F2407FF7E010B
:101FA80090A4C3127735201F0312251B12DD591088
:101FB800001910012C10020280F5120236301F3D64
:101FC800020282101F02D21F021F39E56160F4E588
:101FD8006065617005201FF080E9201FE6056080BC
:101FE800E7E56160DEE56065617005201FD5800961
:101FF800201FD5E560700280CA156080CB121EA72D
:10200800121EFA12C83D12260F756A1012BE2F1240
:1020180026C6909E4ED23C1276F4121D649020295A
:1020280073021F3902330F022049022035121E5C49
:1020380040CB121EFA12BE46C2E2FF12BC6C021F4F
:102048001212DF2F7F6490A69C1276F07F7990A6FB
:10205800A91276F012DD5975160010000A10010950
:1020680010020280F505160516C253121EFA12C890
:102078003D75370A909E6B121CFF902086730220D4
:10208800050220AD02227C0222810220710220B4C6
:102098000220B90220710220F70220FB0220FF0271
:1020A800210602210A7F0A12168680BD124868801E
:1020B8000312485D780A1221D9740912DC3F1222F2
:1020C8001812DC5B12225312BE2F12BE5712BD7EAD
:1020D80012BF6E122362D5150C75150A12226612EC
:0C20E800248912DC5B100204E57F70DB31
:1020F400022005780A800678048002780112486874
:102104008009780A8002780112485D1221D9740985
:1021140012DC34122218E54812DC20E5165403447C
:102124003012DC41742A12DC4112DC4112DC5B12F5
:10213400225312BE2F12BE5712BD7E12BF6E12233F
:1021440062D51548854815122266E51C12DC20E587
:102154001B12DC20E51B2548F51BE4351CF51CE4AB
:10216400A27792E7A27492E0A27392E112DC20AD0E
:1021740075AC74AB73E57DC412219AAD78AC77ABC2
:1021840076E57D12219A1224A712DC5B100204E585
:102194007F709F022005540F2375F00584F8C3EB6C
:1021A40033FBEC33FCED33FDC3EB33FBEC33FCEDE1
:1021B40033FD20E713EB28FBE43CFCE43D12DC2078
:1021C400EC12DC20EB02DC20C3EB98FBEC9400FC6B
:1021D400ED940080E88848121E20E4F54AF549751C
:1021E4006A2075150112BE2F12BD7ED5150E8548C5
:1021F40015E5492401F549E4354AF54AE57F70E5DA
:10220400744012DC84747812DC41746312DC41740F
:0F2214002102DC34122464E56012DC20121EFA71
:1022230012C83DE53A12DC34E53B12DC34E53C12DE
:10223300DC34E53D12DC34E53E12DC34E53F12DCF0
:1022430034740112DC20E54A12DC20E54902DC206B
:10225300121EFA756A20E4F51CF51BF514F51375C7
:10226300150122753800E51412DC20E51312DC2079
:102273000513E513700205142212486880031248FF
:1022830052121E201223BC12DE45756A20751501F9
:1022930075A6FF754A0112BDD712BD7E12BF6E121D
:1022A3002362D5150975151E12238612DE4F1224DB
:1022B30089E57912DC20E412DC20E5711223471250
:1022C300DC20E57012DC20E57B24ACFFE55F3409FC
:1022D30012DC26EF12DC20E51520E033857D56E481
:1022E30012DC20E52EC412DC2612DC6A12DE4F104B
:1022F300021A30559B744012DC41744512DC417460
:102303004F12DC41744612DC4112DC6A022005E5FF
:1023130056122321C4FAE57D1223212A80C2FBC46D
:1023230012232E2323CB12232E2B22540FFC24F60D
:1023330050027C0090233DEC932200000101010236
:1023430002030303FA2440400A24804003EA3322B1
:10235300D2E72274FF2220E703C3132224C022E51D
:102363003F701F7F7B7E0078AEE612D471EE2404AB
:01237300FE6B
:10237400743A12D4E9EE2404FEE53E12D46B12DD65
:102384005922C015C016D21212A6F4C212D016D009
:102394001578AEE612DC34E53E12DC34E53F12DC9F
:1023A40034E54512DC20E55212DC20740A12DC20EC
:1023B40074C012DC2002DC6A744012DC41745412D2
:1023C400DC84744E12DC41743012DC41E516540393
:1023D400443012DC41122464742112DC34E53D12D1
:1023E400DC34E56012DC20121EFA12C83D78ABE63C
:1023F4000812DC34E60812DC34E60812DC34E61297
:10240400DC34E53E12DC341229EFE51212DC34E54B
:102414001112DC34740112DC2090A4F51224C97565
:102424006A1012BE2F057F057F787F12DC19787B36
:1024340012DC19787D12DC19787712DC19E4FEFFBE
:10244400780712DC1912DC19E57412DC20E5751228
:10245400DC20E412DC20E412DC2012DC1902DC6A49
:1024640075C70375C6FF75B901C217751D0085BC14
:102474001C85BD1B85BE1A85BF191252E9EE12DCFC
:1024840020EF02DC20E57512DC20E57412DC20E587
:102494007312DC20E57812DC20E57712DC20E57687
:1024A40012DC20E51664016011E55E12DC20E57A99
:1024B40012DC20E516640260012278BCE612DC20FE
:0A24C40008E602DC2075A700E4938F
:1024CE00700122A312DC411A80F4AF1F7E0478AD96
:1024DE00E612D46B7E0C742C12D4E97E0E18E61222
:1024EE00D46B7E1A78AEE612D46B7E22743B12D475
:1024FE00E97E24E53E12D46B7E2FE54012D4717E28
:10250E0037743B12D4E90E0EE54102D46B753200DE
:10251E00121EFA12C83D857946787A796412C85629
:10252E0074641256DE8E4712260F756A20D23D1243
:10253E00BE2F12BE57122646303D09307406C23DDC
:10254E008E1E8F1FE57F602BE54C24FFF54CE54D6D
:10255E0034FFF54D454C600512BD9380D2751D3C80
:10256E0012BE2F12BE5712BD7E122646E57F6003A5
:10257E00D51DED1226A79026BF12D547203D0DAED4
:10258E001EAF1F1226A79026B812D547E546FD703E
:10259E000B90A62B305D1190A627800C0470109026
:1025AE00A627305D0390A6237F381241B2804BE4FC
:1025BE00FFFC7E05305D047E027FB312546FAC06C5
:1025CE00AB071253397F38C23DE51C6007D23D7E02
:1025DE002C12D4D6E51B203D026007D23D7E301270
:1025EE00D4D6E51A203D026007D23D7E3412D4D6F1
:1025FE00E5197E3812D4D61241B7E53224C850FA06
:10260E0022E54075F03CA42541FFF54CE435F0FE83
:10261E00F54D7C007D1012547C0F8F4BAF4CAE4DA0
:10262E007C007D3C12534F7C00AD4B12547CEE4F20
:10263E0070010F8F4C8E4D2278647973C2D11226A1
:10264E005DFF78677976D2D112265DFE02DE74C305
:10265E00E796FB0809E796FC0809E796FDA2E792C4
:10266E001750031255FE75135A30D10E751320B242
:10267E0017AA47125383AB04AC05E546600B046002
:10268E000BAA4612539AEB03FBEB03FBEB543FFBF7
:10269E00E5132B2017029B9B22EE141430E701E466
:1026AE00FEEF141430E701E4FF2205057088A888B8
:1026BE007005052020F8202075320012DF2F7E1EB7
:1026CE007F1C12DE74DFFB12DE747E1E7F1C12DE98
:1026DE0074DEFB7E1D7F1D12DE74DEFB7F007E210D
:1026EE0078ADE612D46B7E29742E12D4E97E2D18A5
:1026FE00E612D46B7E35742E12D4E97E3918E612AA
:10270E00D46B7F077E21745412D4E97E25744F1248
:10271E00D4E97E2D78AEE612D46B7E35743A12D49F
:10272E00E97E39E53E12D46B78AE1229EF7F0E7E2C
:08273E0021744C12D4E97E2540
:10274600744112D4E97E2DE51212D46B7E35743AAB
:1027560012D4E97E39E51112D46B7F157E257444B7
:1027660012D4E97E2DE54012D4717E35743A12D426
:10277600E97E39E54112D46B7F217E0190A5F612E0
:1027860077357E0EAC77AB7612D31D7E2B85795FBF
:1027960085787B12D8C47F287E0190A5FA127735FA
:1027A600751D2B751E10E5741229A37E25742F1234
:1027B600D4E9751D2D751E2BE5751229A37F367E6E
:1027C6000290A5E6127735E5721228501228E81213
:1027D6001EFA756A209004E6E56CF09004E7E56B56
:1027E600F0AE4DAF4C7C007D4012547CBF00010F13
:1027F6000FAC07AD07E4FED23D12BE2F12BE571234
:102806002891E57F602CE54C24FFF54CE54D34FF1F
:10281600F54D454C600512BD9380DE751D3C0E12CC
:10282600BE2F12BE57122896E57F600612BD7ED5D2
:102836001DED1228667F7812CA407F767E007430BE
:1028460012D4E9E53224C850FA227E2112CF8D1225
:10285600D4877E2F90A5FE305D0390A603027735C0
:102866009004E6E0FD9004E7E0FCC3E56A9420FBF3
:10287600E56B9CFCE56C9DFD50032410FD12556E26
:0D2886009004E8EEF09004E9EFF022DD038D
:10289300AD040E7F78E55E20E72AE57A8549F0A44A
:1028A300A9F0E57A854AF0A429F9E435F0FAE55E62
:1028B3008549F0A429E435F02AFAE55E854AF0A4B7
:1028C3002ACF9FFF12DE74103D18C3EF9B50131BDA
:1028D300EF6B600E8F018B0712DE741FEF6970F8C8
:1028E300AF01AB072290A5AB305C0390A5C4754A3A
:1028F30040754900AF76E577FE20E76B7005EF245E
:10290300105064EF24A8EE34FD401190A5B0305C64
:102913000390A5C8754A1975499A8075EF2450EE3E
:1029230034FB401190A5B5305C0390A5CD754A0CDE
:102933007549CD805CEF24A0EE34F6401190A5B824
:10294300305C0390A5D2754A067549668043EF242F
:10295300F0EE34F1401390A5BB305C0390A5D7751E
:102963004A04754944802A8028EF2490EE34E840D5
:102973001190A5BE305C0390A5DC754A0275498FA2
:10298300800F90A5C1305C0390A5E1754A0175499C
:102993009A7F401277337F4612CA407F5F02CA4054
:1029A300AE1E75F064305C0375F03284C0F0F870CD
:1029B30004EE2404FEE51D12D4E9EE2404FEE860CF
:0129C300070C
:1029C40012D4D6EE2404FED0E075F00A305C037510
:1029D400F00584A8F012D4D6EE2404FE742C12D48C
:1029E400E90E0EE8305C012302D4D6E53E2541F51C
:1029F4001124C45003F511D3E63540F51224E850F0
:102A040002F5122212B9D4C21012DF2F7F057E09FB
:102A1400909C6A1277027F137E08902A3C12D54755
:102A24007F2B7E01902AA412D54720370A7F277E68
:102A340027902B1612D54722113007FE1FE001E123
:102A440001F80F00061B00F80C00180E007C1000A3
:102A54007006003C2000E006003E4001E004001E39
:102A64008003C004001F0003C004000F000780009F
:102A7400000F800780000017800F00000027C00FA0
:102A840000000043C00F00100083E00F002003018A
:102A9400F00700C00F01F80383007F87FE01FC00EC
:102AA4000E3E1800000300000000180000030000A0
:102AB40000003800000000000000300000000000AA
:102AC4000000FC761F0E1C6030ECFCBC3F172DF0A0
:102AD400F978613866264F619A706070C60E1EE3FD
:102AE40030E06060C60C1CC360C0E0618C0C18C789
:102AF400C0C0C0E18C1C39C611C0C4C19C993196B8
:102B04003180C8C1FF1E31E7E180F0C0EE1C31C343
:102B1400818006163091882892884924904927900C
:102B24009248A0E3C8BCC2AFD2C075C0107581D8AA
:102B340074FE122B42E4F5F9F5FBC2B480F7D2A679
:102B4400C2A512B9B912DE4102B9DA75C703E54864
:102B540075F004A42480F5C6C23C75B901E5BC0433
:102B64007002D23C22120E76E5BEF54824F65003DC
:102B7400754800753400753704C228D229D22A75E5
:102B8400C703E54824E75003754800E54875F00499
:102B9400A42480F5C6751607751700C23C122BC411
:102BA400122BC4122BC4122BC485175815587559EF
:102BB40000E548B40A09E5586005F46002055922A5
:102BC400203C1D75B90105C6AABCABBDACBEADBFEA
:102BD400EA122BE5EB122BE5EC122BE5ED122BE5BB
:102BE40022203C07F515B4FF03D23C22C0C7C0C65F
:062BF400127D6775A704C5
:102BFA00851683E517C4F8F58275B90105C6E5BCE3
:102C0A00F0C582F82406F92403C582E5BDF0E5BEC5
:102C1A00F0E5BFF075B90105C6E5BCF0E5BDF0E524
:102C2A00BFF08516838982E4F075B90105C685BCB3
:102C3A001385BD14E4F0F08882E5BEF0E5BFF075B7
:102C4A00B901E5BCF0E5BDF0E5BEF0E5BFF075837E
:102C5A0006E51723541E24B0F582E513F0E514F0B7
:102C6A0075A700D0C6D0C705172212BB9C78BEA68E
:102C7A004808E4F6F55908761808F6D23608760AAE
:102C8A0008F6060876BEC254C25512BEB1122B7798
:102C9A00C229C22AC207C227C268120E67E5BDA2AC
:102CAA00E59243C24AE4F52EF534F536F52F78B6A7
:102CBA00F678B5F678A9F6789EF678B8A65E08A6EC
:102CCA007A12D286C26BC233C238C240C223C2222F
:102CDA00122CF475460278C5A646C23AD221C21908
:102CEA00C226E4F542F541F54022E45407205E0984
:102CFA00B4040040027403801B120E6CC313A9BCF7
:102D0A00600C14A9BD600714A9BE6002A9BFE940FE
:102D1A0001C45407F53722122B69125A3612090CCC
:102D2A0012DF2F121E41E55804700A7F327E059089
:102D3A00A43D12770290A69312874B1208667F72FF
:102D4A0090A6881276F012DD591000051002048050
:102D5A00F8D322C3220200F7120E67E5BD20E70569
:102D6A00122D2140F0754E50122C7412852C754488
:102D7A00031248ED12AF19D54403022B2A201EF183
:102D8A00789F7680754A0012BCCDD210C211C21348
:102D9A00C21212483F75A60C12D9D012C4BBE5A6BE
:102DAA0024FA400612488D75A60C20250CE590548D
:102DBA00057009E53524E25003022E54E532241841
:102DCA00400D75F00C84E5F070D41233D280CFD266
:102DDA001ED2AC306DC87532F012DBD6B4E0BF1229
:102DEA004935E53124F39205201203123264122E7A
:102DFA001AC014128E17D014200A03122F3D123350
:102E0A00D212A6C31233D212852F1233D2022D9CAC
:102E1A0030122EE54024F0401C7A0AC3E53F954B58
:102E2A006013401E24E2400D305405C254757F01E0
:102E3A0012BCF3DAE679BCE7D2E7F57F09877EC2EE
:102E4A007722F40424E250ED80DE12DF2F7F2A7EFF
:0C2E5A000E90A4F912770275A6FFC210BA
:102E66001012137F367E08909F8F12770212DD595B
:102E760012DE3A0200F7D22112491112BCFD7F1E62
:102E86007E0B90A41612770212DD59122EA77F3EF2
:102E96007E0790A12D12770212DD5912DE34022B25
:102EA6002AD215D21412BE88120D4675B90575B907
:102EB6000212BE92D25512BDB77F0012BC6C12BE72
:102EC60092E56A600512BD7E80F7857A62120E94DD
:102ED60085BEBC85BFBD856BBE856CBF75B90575E6
:102EE600B90285BD6C85BC6B756A2012BE8812302E
:102EF600DE12BE92756A0012BE2FE57064FE703453
:102F06007570FC854077854178851F797818797AC0
:102F160012C85612BD2C12DE4F12BE92756A1012DE
:102F2600BE2F7F087810797212C85885627C855E3C
:102F36007D12BD2CC2152212486812308A745212B4
:102F4600DC41744D12DC41744312DC41123099129B
:102F5600DC7C7441207402745612DC41122FE61296
:102F6600303012DC7CE53C12DC34E53B12DC34E527
:102F76003A12DC3412306612DC7C744512DC4112E3
:102F860030CF12308A744712DC41744712DC417428
:102F96004112DC41123099122FE612DC7CE43074C7
:102FA600010412DC3F12DC7C9004C3E012DC341214
:102FB600DC7C9004E4E075F00A84AFF012DC341295
:102FC600DC80EF12DC3FAC5EAB7A1230ABAC5DABB3
:102FD6005C1230AB12DC7C12DC7C1230CF02483F34
:092FE6007875C23D122FF17878D4
:102FEF00D23D12DC7C128211303D05E51E12DC3F12
:102FFF00E51D12DC3F123073E51812DC3FE57D2032
:10300F003D01C4540F12DC3F12DC7C303D09744586
:10301F0030170274578007744E301702745302DC56
:10302F0041207408123066123066802775A704900D
:10303F0004BFE0FCE0FB7A1B125371783212551378
:10304F001253391230709004C1E0FCE0FB12533977
:10305F0012307075A7002212DC7CE4F51AF5198086
:10306F000D12DC7CE51C12DC3FE51B12DC3FE51A80
:10307F0012DC3F12DC80E51902DC3F742412DC41C4
:10308F00744712DC84745002DC4112DC7CE53D1283
:10309F00DC34E53E12DC34E53F02DC3412826D1283
:1030AF00DC7CE51D12DC41781CE612DC3F18B817FA
:1030BF00F812DC80E412DC3F12DC7C744D02DC4140
:1030CF00C038742A12DC41D03812DC5B02DE4F7834
:1030DF00107F0EE4F608DFFCF564F565F567F5681B
:1030EF007515FC751AC0751DC075664075694075FC
:1030FF004A0112BDD730550302319412BD7EE571DE
:10310F00B510004002F510E4F511E512207502E547
:10311F0013C395795006207545857913D3E57A95B4
:10312F0014E5156480FFE55E64809F400C857A147A
:0E313F00855E15857B16855F173074B3C2D18F
:10314D007864797312317278677976123172D2D1CF
:10315D0078187973123172781B79761231728091E9
:10316D0085791280B9D3E7960809E7960809E664D0
:10317D0080FFE764809F20D101B3400AE7F618195C
:10318D00E7F61819E7F622E51AB4C00E7873791828
:10319D0012C8567873796412C85678187964C2D1FA
:1031AD0012320574181256DE8E47AE1EAF1F781BF5
:1031BD007967D2D1123205C3E51F9FE51E9E5004DB
:1031CD008E1E8F1F7EFF7FFFAC1EAD1F12547C7AAB
:1031DD0004EF8AF0A4E5F0CE8AF0A42EFEE435F0DB
:1031ED00BEFF011E60051460057EFF8E1F22EE7E60
:1031FD000020E7F77EFE80F3C3E697FB0809E6970C
:10320D00FC0809E697FD1818191930E7031255FE49
:10321D00C3EB33FBEC33FCED33FDEB33EC33FBED68
:10322D0033FC30D105AA4712539A0BBB00010C7524
:05323D001E03751FFFD8
:10324200EC24FC40048C1E8B1FE627FB0809E637A2
:10325200FC0809E637A2E713F618EC13F618EB138D
:10326200F62210131978B5E624FA401AE57124F60D
:103272004008E57924F6400280360606803212DEE6
:103282004BE59030E2DF753612D22EE4F534F55A72
:1032920012BEE31232B5C219C257122CF412914671
:1032A200129173D212853F4B754C00205E02D228D8
:1032B200022CECD214123304E6F008DFFB857A62AA
:1032C2001232FA7570FE783A797112C85612BD2C14
:1032D2001232FA85627A855E7B120E8A85BC7E8501
:1032E200BD7F7570C012BD2C123304E0F608DFFBFF
:1032F20075A700D254C2142274FF7870F608B88001
:10330200FB2275A7049004F078707F1022121EFA37
:10331200122C7412DF2F12DD59C258C259754A019C
:10332200753901756A2012BDD71256DC8E47C2105C
:10333200D211D214D21212BEE3129146129173121A
:10334200D9D075A6FF753609753200E59020E206E0
:10335200E5352405400CE5905405701FE53524E25F
:103362005019C211C21212DF2F12DD59E4F535F5E0
:083372002F7E0612DE47C202A5
:10337A00022005C221E54AB40202D22112BDD712A7
:10338A00A6C330260F125A9812852F753606E536CF
:10339A0070FCC22612852C1233D2E54A20E021B4F1
:1033AA000209753900E53670F9808CE53960FAFD55
:1033BA0024E24002053912BDD72026C9DDF880E98A
:1033CA0075390080E475370410003A1001161002AE
:1033DA0016E52F5407600312B9CE20783D20790AEA
:1033EA00207A1F220235C802351CE53760091460AD
:1033FA00091460090236740235E7023645C27902B9
:10340A00369102354FE53724FC500FE537640760E3
:10341A000302370C0236D00234E62011FAE5902076
:10342A00E2028056753400201203D2132278A9E6EC
:10343A007017C226767DE5377005106B02D26BD203
:10344A0077753614D22E02BED8E537604314604031
:10345A00B40227200B24E6249B401F2414501C127C
:10346A00914690A3E67F207E0812770212DD5975F5
:10347A003608D22E78A9E624ECF622241940FB2439
:10348A001450F712914612917390A3F07F2980D7B6
:10349A002028E7E54824F640E1E5580460DC7F5D32
:1034AA007E10E6249B40D324145015C2330559C319
:1034BA00E55895595005855859D22690A3D480A924
:0434CA00241940B6CB
:1034CE00241450B2E55960021559102606E55960CC
:1034DE0002155990A3DD808D10780122753900E513
:1034EE003424384007754A0175340022700AE54AC3
:1034FE0030E0F2754A0280F0146008754A061291A7
:10350E00738006754A0412914675390180DA3029A6
:10351E0009C229D22A7559008005302A1BD22912D8
:10352E0086FA1286C8E53524AF400475340022753C
:10353E003700C229C22A80F3206841302703D26A9D
:10354E0022D2221238A812DD59107A0122E5342433
:10355E00384007122CF475340022700FAA37122C43
:10356E00F46A70F27401122CF580EB04122CF5241F
:10357E00FC50E3E537B40706D22880DA8036C2283D
:10358E00E53724FC2324BEF879C4E7F9A74809A738
:10359E005979C4E8F78648088607E537B4050575F6
:1035AE004818D236122B838F59E53764067002D233
:1035BE000702356412388402382EE537601B14601A
:1035CE007614600F146009E53724F9400902378636
:1035DE000236740236BF023753D223124096107948
:1035EE000122E534243840077546017534002278EF
:1035FE00D87020304A0BC24AE624F85004B24380F9
:03360E000AD24A93
:103611007614E54624FE40DDE54660D9154680D89E
:10362100B600D5B40500500C04F54624FA50C9750E
:10363100460580C424F95005127B5B80BB100FB88E
:10364100D20F80B4D223E53464C8600312409610CF
:10365100790122E534243750097011105B32D25BB5
:10366100802E100802D2081240968024100C21D21C
:103671000C801DD22312409610790122D24BE534E1
:1036810024374010C258C259201105D22E75360771
:103691007534002224FD401524037006D258C25906
:1036A10080EEC258D2591460E7D25880E3120E71ED
:1036B100E5BCB2E7F5BC79A1F7124EE680D278B845
:1036C100A65E08A67A2011C8753605D22E80C130B3
:1036D100122B128734055BE55B75F00B84E5F0F581
:1036E1005BE55A24F64009E55A955B5003755B008A
:1036F10012873812DD59E5346003D534D2753400B0
:1037010022D229D22A75480A0237F4C2401007F1A1
:103711003029030237F41286F612870A102A1BC2D7
:10372100330559C3E558955920E7025008755900EA
:10373100E548B41816E558B4FF0375590012871E01
:1037410012DD59E5346003D534C122D22A1286FA3A
:1037510080EE301223128734155BE55B30E70C7580
:023761005B0A01
:10376300E55A24F64003855A5B12873812DD59E582
:10377300346003D534DA75340022D229D22A75484D
:1037830017804CC2401007F22029441286F6128794
:103793000A102A22C2331559E55930E71C855859B6
:1037A300E558B4FF03755900E548B41802800AD2FE
:1037B3002A1286FA800E855859E558B4FF037559C5
:1037C3000012871E12DD59E5346003D534B522207B
:1037D300106220115F7F180548E54864187008F5EA
:1037E3004830270375480A122B4F303C2DDFE88001
:1037F3002620105A2011577F181548E54830E70551
:10380300754817800A640970063027037548171234
:103813002B4F303C05DFE275480A122B83125A36D0
:10382300E532244C50051286C8800312866E753427
:103833000002DD5912386B7F15E5486B70048A4826
:1038430080020548122B4F303CD0DFED80CC12387C
:103853006B7F15E5486A70048B4880021548122B6C
:103863004F303CB6DFED80B27A007B09E537B40414
:1038730001227A0A7B17B40601227418FAFBF54871
:103883002275A704758307E559C4F582E0E0F57353
:10389300E0F574E0F575E0F576E0F577E0F5787539
:1038A300A700025A36E59020E23EE534243750382B
:0638B3001238EC1238C9C6
:1038B900205E4F7F2C909D21123933909D2A806A7A
:1038C900E534243775F009A42435FF205E0624BEAB
:1038D90050027F3EEF249B50027F627E3274891230
:1038E900D51B2275A7049000317E087F3AE4F0DFEA
:1038F900FDE5822446F582E43583F583DEED75A77F
:1039090000227F2C120E6CE5BD12391CE5BE12395E
:103919001CE5BFF8C4123922E8540775F009A490D0
:103929009D0F2582F58250020583EF2409FF027657
:01393900F09D
:108529000285E312DF2FE53724FC40F4B4FE142062
:10853900110EE590F45407600122E532247450EFDE
:10854900028E2312DF2F12D6BE12D75012CF9B12E2
:10855900D2DC12D1257E197F3612D07912DC89122C
:10856900D08FC206E53760051460338053C23A12D2
:1085790086871241591242EE1245D41264F41265EB
:108589001C123E04E54864186009E54824F65003C6
:108599001246BF128DB912CE201241F48014D23A7C
:1085A9001286AD1239421241C312C9A6128DB912EF
:1085B900CDE1125D7712D797125848125B478012A6
:1085C90012869312C8E312D86712C975128DB912AF
:1085D900CDF830101112D02D800C12DF2FE5372481
:1085E900F9401E1286703022091238A8E53470024B
:1085F900C222302309124096E5347002C22302DDFB
:1086090059121DF375170012DA7A7F1212CA2E3029
:10861900124A75100075A704758306125AF1E51000
:1086290075F009A42415FFF5177E00E512602F7572
:10863900F06484E5F00F12D46B1F7E0EE51112CFA2
:10864900E3751623125CAD0510C3E55A9510400673
:10865900E51024F550BF3012031287388088745D05
:1086690012D51B80D5C249302905121DC9800312B4
:108679001DF3909F5512874B202A7602871E3012D0
:1086890023305E2030501D028A2F301217305E06CB
:03869900200B11A2
:10869C0002909012CA277F1712DDCF75172002DACD
:1086AC007A12D63512D5D630121120510512D69524
:1086BC00800612CD7B12CB5B1251AB22E4FEFFE5A0
:1086CC004824F6400D90A4201277357E16E548021A
:1086DC00D4D6B40E0690A42602773590A42D12772A
:1086EC00357E12E54824F702D4717D20800C7D3F45
:1086FC00302A077D633029027D3C7F0080247D2059
:10870C0080127D3E800E7D3CE54975F007A4240661
:10871C00800A7D3FE55975F007A42409FF640270B7
:10872C0001FF7E1CED02D4E97D2080027D3FE55BDC
:10873C0075F009A42416FF7E09ED02D4E9C2491292
:10874C0087AFB4FF01227510001287C67920E03084
:10875C00E702792F3049171211AEFAB40408E5106C
:10876C00700C79658008EA14651070027923E97E33
:10877C001812D4E97E20E51230E708909F8F12770B
:10878C00358016E51112883C125D0D201005201164
:10879C000280063012031287EE0510C3E5589510BF
:1087AC0050A7227E207F001277351286C87E007F6C
:1087BC000690886E12D547E5582275A70475830775
:1087CC00125AF1E51075F007A42409FFF5177E0085
:0B87DC00E51212D4E97805EE2404FE3B
:1087E700E012D4E9D8F6221288F612890CFD7C0033
:1087F700AE1CAF1B12546FBE003A8F00C3E57A95CB
:1088070013FFE55E9514FE402B7C007D2812547CF7
:10881700C3EF98401F75F0058404FB24F950027BD1
:10882700067E2CAF170F12DE740F12DE740F12DEE6
:10883700740EDBEF2264B4602464B475F03284C034
:10884700F012D4D6CE2404CED0E075F00584C0F063
:1088570012D4D6CE2404CED0E02302D4D690886A90
:108867000277352D2D2D000140FFFFFFE0FFFFFFB1
:10887700FFC25030123F20283CE558F460372048AB
:1088870003200931D250E559F51030330665586099
:108897000205101288C012891C75A7049006DCE532
:1088A70012F0E511F0E517F0E510F075A704900652
:1088B700E0ECF0EBF075A7002275A70475830712AB
:1088C7005AF17813E0F608B819FA9006D07811E64D
:1088D700F008B819FAE51CF516F0E51BF515F012C6
:1088E70088F69006DAE514F0E513F075A70022750F
:1088F700A704758306E51023541E24B0F582E0F51E
:1089070013E0F51422120E71E5BD2487E5BD923BF5
:0289170050020C
:1089190024912212890C75F005A485F012F511E451
:10892900F519FEF51CF51D12BE88C23DC2567F3CE5
:1089390012CAD1303D05751900807DDFF3E559650F
:1089490058700A301007EE24D35002D2568C1B8D72
:108959001AE519FD24E250DEAE1CAF1D7C0012544D
:108969006FEFF51924F650CEAC1BAD1A12CA1620BA
:10897900D1108E048F05E51975F0A7A4AEF0FF128A
:10898900546FAC12AB117AA012539AEB33FBEC3350
:10899900FC20D11AEF9BEE9C5014C3E51213FCE5A1
:1089A9001113FBC3EF9BEE9C4004AC06AB072048B8
:1089B90007203B048C128B119006E2E519F0128A0C
:1089C90004AC16AB157AC8125371A912A811125525
:1089D90015ED7005EC249E50057C807B0822C3E5CB
:1089E9007A305602E55C9513FFE55E305602E55D87
:1089F9009514FEC3EF9BFBEE9CFC22AE16AF157CD3
:108A090000E519FD24F6501A12546F7C007D0612F8
:108A1900534F7C007D0512546F8F10EEF51724E932
:098A290050037517FF2212CA2741
:108A3200128A4C128A8F12D28B128AB520480912DE
:108A42008BA3128BD3028C3680747F177E20204832
:108A52000E748A204D101258B5500E742F80077470
:108A62006A305F02746712D51B75A7049006D0782E
:108A720011E0F608B819FA7F177E00781275190509
:108A8200E60812D51BEE2406FED519F42275A704BA
:108A92009006D8E0F516E0F515E0F514E0F513E0E0
:108AA200F512E0F511E0F517E0F510E0FCE0FB75DA
:108AB200A700227F187E26AC14AB1302D31D9006AA
:108AC200E4E0F51CA3E0F51B7F2A304E13120E677B
:108AD200E5BF90A489B4010390A6821276F0804289
:108AE2000F7E00745312D4E99005CBE0F830E7050D
:108AF200E53F30E0091F7E00E8540F12D5019004D3
:108B0200EEE0FEF51EA3E0FFF51F128B4BE51E24DF
:108B1200E9500C7E06742B12D51B7E0C12D51B124B
:108B22008B7BC20375172A751627125C7C202415CD
:108B3200205F15D2037F2A7E1E908B69304E0390F0
:108B42008B7202D547205FEB227C007D3C12547C65
:108B5200A805EF7F2A7E0812D4247E12743B12D518
:108B6200177E14E802D41E0707384C9EBAF2643806
:0F8B72000707387CE6C2E67C38AC1CAB1B7A48A0
:108B8100305D027A27125371A91EA81F125515EDE7
:108B91004C60027BFF7F207E28EB12D42A7E3902B3
:108BA10091237F2B90A433127733E517F46022AE23
:108BB10017AF107C007D3C12547CA805EF7F2A7E04
:108BC1000C12D4247E16743B12D5177E18E812D4E9
:108BD1001E22AE12AF117C007D0A12547CA805EF53
:108BE1007F207E3012D4247E3A742C12D51B7E3C19
:108BF100E812D5010F7E29744502D4E974858007F6
:108C0100748720560274867E2912D51B301707748B
:108C11002D7E3A12D51B227C007D0A12547CA805B8
:108C2100EF7F2A7E3012D4247E3A742C12D51B7E1B
:108C31003CE802D501128D67E54824F65005128CF7
:108C41001880B9E559046558600D128C18128BFD16
:108C5100E559655860AA22A217923D8E1E8F18858C
:108C610015179006D0E0F51185581015101245B46E
:108C7100C3E51195105002F404F924A65005C374FC
:108C8100B399F9E975F00584F924EE500279119050
:108C91008DA7E993F5F0120920E5CC7004E930E7DE
:108CA10002747F23A4A9F0E51B2517FDE51C3516E9
:108CB100FEC3ED99F515EE9400F51675A7007583C1
:108CC10006E55823541E24B0F582E0A3F513E0F520
:108CD10014128D67203D2C201729120E71E5BD2439
:108CE10087E5BD5002249175F007A4FB9518E5F0C6
:108CF100951E400FEB9FE5F09E4008EF9518EE950D
:108D01001E500EA23D9217AE1EAF18128C18028B88
:108D1100FD306B10128D04E53F20E00774867E2242
:108D210012D51B2275A7009006E0E516F0A3E51504
:108D3100F0128C18128C0174857E2312D51B855874
:108D4100101288C0128A4C128A8F8C168B15128AC7
:108D5100B51289CA1288B212D28B9006E2E0F519D7
:108D6100128A04028BA3C3E57A305602E55C95139F
:108D7100FFE55E305602E55D9514FE921750031231
:108D810055E6AC16AB157AC8125371A906A807129D
:108D910055157E037FE7ED700CEB2418EC34FC4095
:108DA10004AE04AF032200172E43576C8092A4B681
:108DB100C5D3DFE6EDF3F8FD305E4F30504C75A7BB
:108DC100009006E0E0A3FCE0FBECA2E79217402054
:108DD10024FE50047F3B8022AE04AF037C007D144F
:108DE10012547C74542F2017029F9FFF7462800CD1
:108DF1001255F6EC24FE50E07F6D743D7E0012D4D6
:108E0100E97E017D197C03128E0C227F3D12DE74F6
:108E1100EF2DFFDCF822E537B40206E534243750A4
:108E2100292212DF2F12D6BE12CF9B128FA312C896
:108E31007112CE08128FFB125B477F207E2B12D05E
:108E41007912D75012DC891238A812D1B1128ED101
:108E510012514502DD5920041EE579FD24A050027E
:108E61007D5FED24CD401E744520750C2DFFF5125C
:108E7100128EA61FBF44F922C39DFFF512128EA6C2
:108E81000FBF46F92220750EED2413FFF512128E45
:108E9100A60FBF78F922C374779DFFF512128EA633
:108EA1001FBF12F922EF24BA40082433FCC37432E5
:108EB1009C1404FC24D750047C238009EC2375F016
:108EC10005842413FC7E0512DE740EECB506F8222F
:108ED100E59020E206E53424374003128E577F45A2
:108EE1007E047D1212DE740EDDFA7F437E0074640F
:108EF10012D4E97F4F7D12128F8C7F3B7D12128F2E
:108F01008C7F597D16128F8C7F317D16128F8C7F4D
:0F8F1100637D1A128F8C7F277D1A128F8C7F6DD4
:108F20007D1E128F8C7F1D7D1E128F8C7E057F19FA
:108F300012DE740FBF72F97804E57924CD500278FF
:108F400009E8305C0123F87F1B128F7B7F6B128F47
:108F50007B18305C01187F25128F7B7F61128F7B1D
:108F600018305C01187F2F128F7B7F57128F7B1870
:108F7000305C01187F39128F7B7F4D7E00E875F0E1
:108F80000A847004E802D4D6E802D471EF65126056
:108F90000C7E04EE20E00712DE740EDDF62212DEF7
:108FA000A480F790A5487F287E2C1277357E3B124F
:108FB000D334AC5EAB7A7F307E19C23D12D373904E
:108FC000A4377F5D7E2D12773578B9C3E57A961880
:108FD000FBE55E96FC7F507E19D23D02D373E5110E
:108FE00064B4700122E51112DCF97831790F7D0B40
:108FF00012DDF71F1E90908B02D547E5716012E5D8
:109000007012DCF97831790F7D0412DDF30DBD0AA1
:10901000F97F011290637F1D1290637E2312906D81
:109020007E3F12906D7E247F171290777E397F02EB
:109030001290777E247F071290817E397F1C1290D8
:10904000817E317F0212DE747F1C12DE747F0F7E00
:109050002412DE747E3E12DE747F0C7E2E90D83C8D
:1090600002D5477E2A12DE740EBE39F9227F08121D
:10907000DE740FBF17F9227D0612DE740E0FDDF9C4
:10908000227D0612DE740E1FDDF9220303E0A0E04C
:1090900012CA277F18909D611277337F217E017459
:1090A0004112D4E97F2A7E01745312D4E99005BE9F
:1090B000E0F51AA3E0F519A3E0F51EA3E0F51D8580
:1090C0001A1C85191B751720129140E519251DF5ED
:1090D0001BF51DE51A351EF51CF51E751729129195
:1090E000409005BA129130AC1AAB19751720129046
:1090F000FE9005BC129130AC1EAB1D751729EC70AB
:1091000006EB24CD4001227A48305D027A271253C3
:1091100071125515ED4C600122AF177E07EB12D38B
:10912000D07E1A0F90A60B305D0390A60E02773505
:10913000E0FEA3E0FD12BFDEC3EB9DF8EC9EF9223A
:10914000751627025CAD12BFDE75A7049005B478D2
:10915000737F06E6F008DFFBECF0EBF0E0E0E0FC0C
:10916000E0FDE0FEE0FFEF2DFFEE3C9005C0F0EFEC
:0B917000F0801275A7049005BAE0FB28
:10917B00E0CBF0EBF0E0E0E4F0F075A7002275A790
:10918B00049005B478647F06E0F608DFFB75A70052
:0E919B00125EBC9005BEE51CF0A3E51BF022A1
:10393A00D23C799E77008002C23C12BE88E4F51020
:10394A00F511F512F513F514F515F516F517C23D2F
:10395A00123C8A203D1F123C8A203D19E51F30E5A2
:10396A001130E40E1239B1303C08799EE724F55043
:10397A000122D510DBAE14AF157C00AD12125449EA
:10398A008F55AE16AF177C00AD1312546F125670D6
:10399A007E00E55530E7011E2DFFE43E30E7027F49
:1039AA0000740A2FF55622C235E51CAF1DBFFF056C
:1039BA000FD235F404FABF003F532CF8E518AF19BB
:1039CA00BFFF050FD262F404BF002D20E72A205B57
:1039DA000123FF24AA4021E51AAE1BBEFF050ED221
:1039EA0061F404BE00128547F0A4E5F020E709203F
:1039FA005B0123FE24AA5001227C807B8030516621
:103A0A00302163C006C0078AF0E545A4AEF0FFE5A1
:103A1A0056205B011375F009A4ACF0FD12546F74C3
:103A2A00FFBE0001EFFA24C050027A3FD007D00649
:103A3A00E55212DCF9303504B2D5B2D1EA8CF0A4E1
:103A4A0030E70205F0748025F020D10495F095F056
:0A3A5A00FCEA8BF0A430E70205F04F
:103A6400748025F030D50495F095F0FBC3EC2F203D
:103A74006203C39F9FFFEB2E306103C39E9EFE2013
:103A84003C64200C05123B1E4064123B00405F1254
:103A9400DE74E51EFD24FB50550E12DE74ED24F693
:103AA400504C1E1F12DE74ED24F150421E0F12DE24
:103AB40074ED24EC50380F12DE74ED24E7502F1F00
:103AC4001F0E0E12DE74ED24E250231E0F0F12DEC1
:103AD40074ED24DD50180E12DE74ED24D8500F1E40
:103AE4001E1F1F02DE74123B004003799E0722E969
:103AF400242AFFE82461FE123B1E401DEF2460408F
:103B040018243F5013EE2460400F243F500AEF2442
:103B1400D6FFEE249FFEC322D322532CF8432C0459
:103B2400EE10E706D2E7F404D261FE24D340EAEFB4
:103B340010E706D2E7F404C262FF24D340DBEFB5FA
:103B440006005003CED26070057480FE8062FF24AC
:0D3B5400FD5060903C0A938EF0A4AAF0335F
:103B6100CA33CA33CA33CA33CA33FA903C34938F47
:103B7100F0A433C5F033CA903C5593FB123BD29568
:103B810070500224B412DCF9EA8BF0A430E702058C
:103B9100F0C3748095F020D50425F025F0FEEA8C61
:103BA100F0A430E70205F0C3748095F030D104250C
:103BB100F025F0FFC3227A01EE6F70097B16BF0278
:103BC100BB7A0380B7BF01047B0080B07B0D0A8004
:103BD100ABE52C540723C3903BDC73800E800E8031
:103BE10024801E8010800A80108012EB22742D9B8D
:103BF10022742D2B22745A9B22745A2B2274879B78
:103C01002274872B2274B39B22FFFFCCAA9280716E
:103C1100665D554E4944403C383533302E2C2A28B8
:103C2100272524232221201F1E1D1C1B1A1A1918A7
:103C31001817178181818282838384858687898A87
:103C41008B8D8F90929496989B9D9FA2A4A7A9ACCF
:103C5100AFB1B4B400010203040405060708090A60
:103C61000A0B0C0D0D0E0F0F10111112131314145A
:103C7100151516161612BDC012BC4EE4F5F7C2B2E8
:103C8100C2B2E5F7D2B264C022203D07123C767081
:103C910003D23D22056D056D12BC4E7D008DF7C22C
:103CA100B2C2B285F71F8DF7C2B2C3E5F79573F5BE
:103CB100188DF7C2B2C2B2E5F79574F5198DF7C246
:103CC100B2C2B2E5F78DF7C2B2C3E5F79576F51A40
:023CD1008DF76D
:103CD300C2B2C2B2E5F79577F51B8DF7C2B2C2B295
:103CE300E5F78DF7C2B2C2B2E5F7F51E8DF7C2B2A2
:103CF300C3E5F7957AF51C8DF7C2B2C2B2E5F78D2D
:103D0300F7C2B2C2B2E5F7D2B2543F30E50244C0C3
:103D1300955EF51D156D156DE51024784001227E25
:103D230000AF55EF30E7011E0512E51FA2E592D55E
:103D3300400EE515951EF515E5149400F514800B5A
:103D4300E515251EF515E43514F5147800E51E6018
:103D53000620D50318F404C39FF5F0E89E30E7016D
:103D6300220513E5F0A42517F517E5F03516F5162A
:103D730022303D03D23D22123C7660F8123C76603D
:103D8300F3E546600A123C7660EA123C7660E5058C
:103D93006D056D056D12BC4E7D008DF7C2B2C3E596
:103DA300F79573F5188DF7C2B2C2B2E5F79574F5BE
:103DB300198DF7C2B2C2B2E5F78DF7C2B2C3E5F708
:103DC3009576F51A8DF7C2B2C2B2E5F79577F51B72
:103DD300D2B2156D156D156D2230742412BE88C2D2
:103DE3003D75101E123D74203D167902123E484067
:0A3DF3000CA806A907123AF34003DA
:103DFD0012DE74D510E422200F4030123D2006CF84
:103E0D00304806200C03204FC6E546790260147930
:103E1D000614600F791614600A79361460057976E8
:103E2D0014701712BE88C23D7896123D74203D0A5B
:103E3D00123E48400312DE74D8F022532CF8AB1812
:103E4D00E519FC339262123E9ABC002BEB89F053BC
:103E5D00F00784FF24DF401FAB1AE51BFC33926192
:103E6D00123E9AAA4712539ABC000CEB89F053F0FC
:103E7D000784FE24DF5002D32274562F2062029F46
:103E8D009FFF741F2E3061029E9EFEC322500312AF
:103E9D0055F6E920E40122C3EC13FCEB13FBE920FA
:103EAD00E50122C3EC13FCEB13FBE920E60122C371
:103EBD00EC13FCEB13FB2274542F2062029F9FFF27
:103ECD00741D2E3061029E9EFE2279B4203249204F
:103EDD001D46EFB506009260AC06AB074004AC077B
:103EED00AB06903F26EC2304938BF0A4A9F0EC23B2
:033EFD00938BF0B4
:103F0000A429F9903F8693C9904086E52C540793E5
:103F100013E95001F490408EF9E52C54079329756C
:103F2000F0B484A9F022FFFFFFFF7FFF55553FFF4C
:103F300033332AAA24921FFF1C711999174515556E
:103F400013B1124911110FFF0F0F0E380D790CCC60
:103F50000C300BA20B210AAA0A3D09D8097B0924BF
:103F600008D30888084207FF07C107870750071CC6
:103F700006EB06BC06900666063E061805F405D15B
:103F800005B005900572000000000001010101016B
:103F90000101010102020202020202020203030302
:103FA00003030303030304040404040404040405D6
:103FB00005050505050505050606060606060606A9
:103FC000060607070707070707070708080808087E
:103FD0000808080808090909090909090909090A55
:103FE0000A0A0A0A0A0A0A0A0A0B0B0B0B0B0B0B2A
:103FF0000B0B0B0C0C0C0C0C0C0C0C0C0C0C0D0D02
:104000000D0D0D0D0D0D0D0D0D0E0E0E0E0E0E0ED9
:104010000E0E0E0E0F0F0F0F0F0F0F0F0F0F0F0FB4
:10402000101010101010101010101010101111118D
:10403000111111111111111111111212121212126A
:104040001212121212121213131313131313131347
:104050001313131313131414141414141414141426
:104060001414141414151515151515151515151505
:1040700015151515151616161616161616161616E5
:1040800016161616161600FFFF00FF0000FF002E82
:10409000B5875B2D5A88E537607414603EB40258CA
:1040A0007F347E12E5342437400810644B90A40717
:1040B000801AF89041E012D547E824FD501179A10B
:1040C000E77E0590A23E20E70390A2480F803A24A5
:1040D000040F7E2312D508D26480627F357E02E50C
:1040E000342437401410641090A12430081B127738
:1040F000027E1A90A406801122700590A1368009D4
:10410000909D8C200C03909D9812770280C97F357A
:10411000E5342433402A2404501B7D0F600C7D1E9F
:104120001460077D3C1460027D78ED305D02C3139E
:104130007E2B12D3D07E0090A13712770202DD5978
:104140007E0524FE5005909F7C8009909D71200F74
:1041500003909D7C12770280E4E546604A14603C3F
:1041600014602E14602014601290A63F205D4190D0
:1041700041D97F367E3412D547803C90A63F305DD2
:104180000390A63B802A90A63B305D0390A6378023
:104190001F90A637305D0390A633801490A633306D
:1041A0005D0390A62F800990A62B305D0390A62773
:0241B0007F3658
:1041B2007E331277357E3C7422305D02748302D5E1
:1041C2001B305D0890A617305BE4800690A61F2086
:1041D2005BDC90A61B80D70508B28D8DB5BA09109D
:1041E20006000A10F248922492249224F2480A10FD
:1041F2000600305E5220434F20284CE55864FF6091
:1042020046E54824F640407F3FE55804F9C23D1296
:10421200424A1211AE601AB404047401D23D75F020
:1042220003A4243CB5070A7E3A303D027E36124290
:104232004C0F0F0FD9D7E55975F003A4243EFF1296
:10424200424A0F0F12424A227E3D12DE740EBE40D7
:10425200F922C248C249305E56202853E55864FF0D
:10426200604DE54824F640471211AE6042D249B48F
:104272000402803B1465597036D248304E31E559FC
:104282006558602B3074281242B7120E67E5BFB42E
:10429200011DE5BD20E618202416205F129006E4D9
:1042A200E0700CA3E024CE400624255002055922DA
:1042B200305FFC80E820113375A7009006E4E070BF
:1042C20028A3E0302402F404305F02F4042404F949
:1042D20024F74015E924FC4003D26C2270012230FD
:1042E2006C097536A7D22ED22FC26C22305E0830EE
:1042F2007405E558B4FF0122C244C24D780075A787
:0B4302000475830712463688188A1ED7
:10430D008E168F17C23EC23BE54824F6500302437A
:10431D00C7D23EE55860F7E8655970F22048EF12B4
:10432D00447C30D13BAE16AF17A818E54670551238
:10433D000920E5CC49604DD244E5CC7033E924CD5C
:10434D00402EE975F038A4ACF0FB12558512558559
:10435D00EBFDF5111243DD304D2CC206C23B8043FF
:10436D00E546705C120920E5CC7005E924CD50506E
:10437D00124F7C75A704758307A8181246368A1E3E
:10438D008E168F178037120E67E5BDA2E0B3923BF4
:10439D005011307428123AF34026A907A806D20608
:1043AD0012CAB81243F91243F0124439890788062C
:1043BD001E1F90463112D547800630D1031244118D
:1043CD00A81808C3E55898400302430075A70022BA
:1043DD0074562F2062029F9FF9741F2E3061029E2A
:1043ED009EF822E51865586001227D057A00EA12D3
:1043FD00DCF912DDF70A0AED24F240020A0AEA247A
:10440D004C50EB22AE16AF17123EC41E303E021EAC
:10441D001EE51E12D4E9EE2404FEE51212D4E93095
:08442D003E09EE2404FEE51334
:1044350012D4E922E5186558603CC001C000C012DD
:10444500C0138518101245B4D013D012D000D00176
:10445500E510303B07C39570500224B412DCF920F7
:104465003B07AE16AF171243DDE5112402FD7A06B0
:1044750012DDF71DDAFA221211AEB40457E87054B2
:10448500120E85E5BD604D78C6A61308A61208A6CE
:104495002C12C86575A704758307751001125AC2D9
:1044A50012C85F1510125AC21256DC8E628F631243
:1044B50057648B1C8A1B12C86B20320E1245642070
:1044C5003B08D24D1266FF1244DA78C68613088679
:1044D5001208862C22120E85AABD7C027BB31253CC
:1044E5009A8C128B13AA1DA91F1253DCA91CA81B99
:1044F5001255158C1D8B1FAC12AB13AA19A91A12D4
:1045050053DCA91CA81B1255158C198B1AE56E25B1
:104515001AF9E56D3519F8C3E56E951AFBE56D9544
:1045250019FAC3E554951FFDE56F951DFCE5542566
:104535001FFFE56F351DFEE52C23652C30E206ECEB
:10454500CEFCEDCFFD75A7049005C2E8F0E9F0ECCF
:07455500F0EDF0EAF0EBF0DD
:10455C00EEF0EFF075A70022D23BC3E5649573C56E
:10456C00659574F564E5669575600404600822E54C
:10457C006424E0500822E5642420400122C3E5674E
:10458C009576F567E5689577F566E5699578600940
:10459C0004600122E566F48002E5668562F0A4748D
:1045AC00E025F04002C23B2212C86575A704758352
:1045BC0007125AC212C85F0510125AC2C02C125AE6
:1045CC00DBD02C891002C86B30125120064E7800BB
:1045DC0075A70475830612463630D139123EC4E5F0
:1045EC004624FE500A0E0F90462C12D5478026EA20
:1045FC007007745D12D4E5801C75F06484ADF070A6
:10460C000FED75F00A847008E5F00E12D4D6800513
:10461C001EED12D46B08C3E55A9850B475A700224E
:10462C00030340A040030340E040D2D1E8C4F5822C
:10463C00E0FA797312468F30D146AF06532CF8ED61
:10464C00BFFF07F40460390FD262BF00331247C3B7
:10465C00402E797612468F30D126E5822403F582DE
:10466C00E0F512E0F513EEA2E713FEED13BEFF0723
:0A467C00F404600C0ED261BE0006CB
:104686001247E0400122C2D122C3E09709FDE0971C
:1046960009FEE097600904700AEE30E7068007EE2F
:1046A60030E703C2D122E546600E14600BF9EDCE69
:1046B600A2E713CE13D9F8FD227C007B44E54660C1
:1046C600207C007BCC1460197C017B981460127CE2
:1046D600037B3014600B7C067B601460047C0C7BCF
:1046E600C08C148B157AE9125371A8471255138C96
:1046F600168B1775C70075C6047510DF75B901E509
:10470600BC20E76FF51385BD1205C605C675B90150
:10471600532CF8C3E5BE9573FBE5BF9574FC05C63F
:1047260075B901E5BC9575FD5005D2621255FEC3FB
:10473600E5159BE5149CE49D40338C198B18C3E565
:10474600BD9576FBE5BE9577FCE5BF9578FD5005F2
:10475600D2611255FEC3E5179BE5169CE49D400DFC
:104766008C1B8B1A12478AE5322428401305C6E5AE
:10477600C68006E5C62404F5C6700205C7D5100135
:0F47860022024702AE19AD181246ACED1247C31E
:10479500AE1BAD1A1246ACEE13ED131247E0123EF6
:1047A500C4E54624FB50080E0F90463102D5471E3E
:1047B500E51312D4E9EE2404FEE51202D4E975F0FE
:1047C500067FFDA946B9000575F0027FFF84C5F097
:1047D5002F500205F0C5F0FF24DE228547F0A430F6
:1047E500E70205F0E5F0A946B9000280050475F079
:1047F5000384FE24E022E537B4020122E537700286
:10480500D23964027002C239E53724FC799EE7602B
:1048150005640B600C22D27E20081E401C107F1000
:1048250022D27F2008134011107E01227537012204
:104835007537002039037537022275F9FF75FB00BE
:10484500800E75F9FF75FBFF801C2053F512487D1E
:10485500759E85759D2D801412487D759E84759D68
:104865002D800912487D759E83759D09C2AC75988A
:1048750052C26DC26EC26F2212166EC253E4F5F9B2
:10488500F5FB30340215FB22D2A47F3212DE51C271
:10489500A412D9D012DD5912DE3AC214C21512483B
:1048A5003F74C012DC8474A312DC41748F12DC41A6
:1048B5001248D374C012DC8475A7049048DD7F10BC
:1048C500E49312DC41DFF91248D375A70022E538DD
:0548D50012DC4174CA71
:1048DA0002DC41A29494859C8080808080818380C0
:1048EA00819E8075A60A12489FD269D2ACE5A62499
:1048FA00FA500C306DF712DBD6B4E0F1124935C22A
:10490A00ACC26975A6FF22D21EC274C273E4FDF559
:10491A0071F570C22D12483FD2AC12DBD6C5F070C9
:10492A0005DDF7C2AC22C5F0B4E0EFF538E4F532A4
:10493A0012DBD1A2E19273A2E2927475A7049004E9
:10494A00B4F012DBD1C2D1124B1C20690330740BB4
:10495A008D758E748F73E514C4F57D124B9C124BC2
:10496A001C20690330740C8D788E778F76E51425B8
:10497A007DF57D124B9CD2D1124B1CEEF0F55DEF0A
:10498A00F0F55C207303E4FEFF79BCA70609A707CC
:10499A0012DBD17D0A124B898F71EE60037571FFAC
:1049AA007D14124B89C22DED24F150010F240A50B7
:1049BA0002D22DBFB4027F008F7012DBD1F05407F0
:1049CA00C52E54F8252EF52EE571700EE4F571F515
:1049DA0070C22D9004BFF0F0F0F012DBD1E5386020
:1049EA0009D21EC27412AF1D8005C21E12AF19125F
:1049FA00DBD1B4E1FA75A7049004C412DBD1F0123A
:104A0A00DBD1F0F53A12DBD1F0F53B12DBD1F0F550
:0B4A1A003C12DBD1F0F53D12DBD1F0C7
:104A2500F53E12DBD1F0F53F12DBD112DBD1B4E25A
:104A3500FA12DBD1F07E0C12DBD1FF12DBD112DBD7
:104A4500D112DBD112DBD120E1027F00EFF012DBC6
:104A5500D1DEE412DBD1B4E3FA12DBD1FF12DBD1F4
:104A6500CF60027F7F9004E4EFF0E4F012DC019068
:104A750004D8124B8912DBD1B4EAFAC2AC75A7048B
:104A85009004DAE561F0E560F0E55EF0E57AF0E5E1
:104A950079F0E52EF0E55FF0E57BF0E551F0207467
:104AA50012E4F571F5709004B4F09004BDF0F0F0E7
:104AB500F0F0F075A70078ABA63A08A63B08A63C2F
:104AC500120E7BE5BF253D240C75F0188478AEA643
:104AD500F0186005640260182216E670121816E6D2
:104AE5007004760C181678ACE6904B0F9308F622F6
:104AF5000618E608904B0F930466700D76011806AC
:104B0500E6640D70047601180622001F1D1F1E1F86
:104B15001E1F1F1E1F1E1F12DBD1FC12DBD1FD1233
:104B2500DBD1FE12DBD1FFECA2E692E7921713FC74
:084B3500ED92E713FDEE92E79B
:104B3D0013FEEF92E7301701F4F513ECA2E713FC27
:104B4D00ED92E713FDEE92E7301701F4F512ECA2AA
:104B5D00E713301701F4F510ED92E7301701F4F576
:104B6D00111255A620D10E8C1C8D1D8E1E8F1F125D
:104B7D00B3251255A630170312B2FF2212DBD1C393
:104B8D0013FEF012DBD192E7FFF07C0002547CACF7
:104B9D001CAD1DAE1EAF1F30170312B2FFECF0EDB2
:104BAD00F0EEF0EFF022124BBC0202C612BC8DC229
:104BBD00101248F07F5A7E0590A41612770212DD6E
:104BCD0059D214D215C255122CEC789F76800876E6
:104BDD000012BCCD1232FA7570FE853A71853B72AA
:104BED00853C73853D74853E75853F7612BD2C12CF
:104BFD0032FA7570C0757B03757A54E4F57FF57ED6
:104C0D0012BD2C751421751348755F01757B0075E8
:104C1D00750475745275780175776CE4F57DF551F1
:104C2D00757F0190DF5C85836E85826DC23D124C70
:104C3D009A851C1D75A6FF305505C221022EA7129F
:104C4D004C9AE572A2E59275A2E79277D274D2736F
:104C5D00E51275F008A4AEF0FF2075031255E612AB
:104C6D00C7B512C7FE124D1DE51C251D13F5718527
:054C7D001C1D12BCA586
:104C820012BCFD757F02E56A70B57F5A7E2FE54141
:104C920012D3D012DD5980A7856E83856D82C255ED
:104CA2007873124CFE7876124CFEE493F570B4B42D
:104CB20002D255A3E493F51CA3E493F512A3203D7D
:104CC2000FA97BE493F57BC399502A20E702055F85
:104CD200A385836E85826D103D16D23DE582240543
:104CE200F582E43583F583E493F52654F0F57222D8
:104CF200E526C480F630E7D8155F80D48601E493B8
:104D0200F6A308C399500A20E70606B60002080671
:104D12002230E70616B6FF0218162230750DE5138B
:104D22002579F513E43514F514800DC3E51395794F
:104D3200F513E5149400F514AE14AF137C007D0A4C
:104D420012547C8E5E8F7A22124DDF851617203D1B
:104D520001227F5A909C831276F07F64E5166404E8
:104D6200700C909C9B12773312DD5902DE34909CBA
:104D72008F1276F07F6E7E0890A607127702121EBF
:104D82000312DD597515B87514047F6E7E20C22496
:104D9200A815E82404F9C23DE7124E27203D06E695
:0A4DA20012D51B8008E6128460E8B9
:104DAC00A815F60515EE2406FED514DA851716128D
:104DBC001E5112DD5910000510018D80F878B812C3
:104DCC000E8F86BC0886BD0886BE0886BF124EE6CE
:104DDC0012DF2F120E8FC23D75160078B87F4B7EF6
:104DEC000890A6071277027E20E5BC12D51B124E46
:104DFC001E7E26E5BD12D51B124E1E7E2CE5BE1264
:104E0C00D51B124E1E7E32E5BF12D51B124E1E0252
:104E1C00DD59F608080808F618181824D05005248F
:104E2C00F64001220516D23D2275C70375C6FE1247
:104E3C00766E124EE675C6FC75BC2675BD6475BEE5
:104E4C00A975BF70124EE675C6FB12766E124EE651
:104E5C0075C6FA75BC1475BD1475BE0075BF0C1201
:104E6C004EE675C6F975BC4E75BDBF75BE0075BFF7
:104E7C0019124EE675C6F875BC0A75BD7E75BE0076
:104E8C0075BF01124EE675C6F775BC0175BD23756D
:104E9C00BE4575BF67124EE675C6F675BC0275BD8C
:104EAC00AB75BE0175BF01124EE675C6F512766E76
:104EBC0075BE0275BF0A124EE675C6F412766E7593
:104ECC00BCE1124EE675C6F312766A124EE615C6B2
:104EDC00124EE615C6124EE615C675B90575B90221
:104EEC0022751500127D6775B901E5BC64816003FC
:104EFC001276510515E515242050E975C70375C6C2
:104F0C008075B90505C6E5C6241C50F5124F1E0266
:034F1C007BBDE476
:104F1F00F5C7F5C6742612766F75BD4E124F38124F
:104F2F004F35E4124F3512766F124EE605C6227FCB
:104F3F00357E00E54B12D4877E10E54C12D4877E68
:104F4F0020E54D12D4877E30E54E12D487227F465E
:104F5F007E00E56C12D4877E10E56B12D4877E201D
:104F6F00E56A12D4877E30E57F12D4872220740140
:104F7F0022D24475A700758307E559C454F024075E
:104F8F00F582E0F51A244C40E7A3E0F512A3E0F513
:104F9F00131209208938120E67E5BDA2E0923BE596
:104FAF001A40069570500224B4F51A203B05D2061C
:104FBF0012CAB8E51A1250DFE5152437F51DE4358E
:104FCF0014F51CE5172437F51FE43516F51E85CCAF
:104FDF0012853813AC12AB137A0412536375380170
:104FEF0024FA401A05382402401405382401400ED3
:104FFF000538053824014006053805380538C3E55E
:10500F001A945A500224B4F51AC23BC23CC23D75E1
:10501F001B00A23B823C406D203B2CE51A75F0082B
:10502F00A4951BFBE5F0303D04940180029400FC35
:10503F005008EB24A0FBEC3405FC1250E6125095FF
:0A504F00923B40031250B8203C2CA5
:10505900E51A75F008A4251BF9E4303D010435F083
:10506900FAE994A0FBEA9405FC5004AB01AC0212E6
:1050790050E6125095923C40031250B8E51B253872
:10508900F51B5094203D04D23D808D22E51F251744
:10509900FEE51E35167016EE24914011E51D251505
:1050A900FFE51C35147006EF2491400122D3228EAE
:1050B900027C8A7B3B125371ED2402FE8F027C8AAB
:1050C9007B3B125371ED2439FF02DE741256CF80F7
:1050D900311256C2804675F008A4ACF0FB75190070
:1050E900C3EB9468F9EC9401FA40080519AC02ABDA
:1050F9000180ED8C108B11531903E51920E0CD12B5
:1051090056C212513AAF05E51924FE50031255E66D
:105119008E168F17E51920E0B81256CF12513AAF03
:1051290005E5191460061460031255E68E148F15EF
:1051390022AC06AB07AA12A9130253DC125227208C
:105149003D4974857F227E0812D51B7E0830173CA5
:10515900AC1EAB1FEB2418EC34FC402F125342E574
:105169001B60077F207E0812D5367F207E10E51A46
:0951790012D5367F237E17742E37
:1051820012D5177F207E1BE51B7011E519C2E012B4
:10519200D536227F207E0E740A02D536E51975F0C7
:1051A200058475F005A402D536125227203D5E749F
:1051B200857F227E3A12D51B301753AC1EAB1FEBF4
:1051C2002418EC34FC4046EC7033EB249C402E7ED9
:1051D2002D125219125585C0E07F2A7E2EEB12D570
:1051E200367E39D0E0C2E012D5367F347E3712DE09
:1051F200741E12DE741F12DE740E02DE747E301212
:105202005219125585EB7F2A7E3112CE5A227F2AFD
:105212007E39740A02D5367F2912DEA40FBF34F913
:105222000EBE40F322D23D301266120E71E5BDF57C
:105232001C75F00AA4F824E15002781EE4FCFBFE7F
:10524200FFC23D12BE88125293203D44D8F8751D0C
:10525200CEE51C146009751D9C146003751D6AC29D
:1052620017EC30E705D2171255F68C018B00E9488E
:105272007003D23D22EE7008EF251D4003D23D227D
:10528200AC06AB077A1C1253711255158C1E8B1F7C
:1052920022203D07123C767003D23D22056D12BCDE
:1052A2004EE4F5F7C2B2C2B2ADF7F5F7C2B2C2B27E
:0252B200E5F71E
:1052B400FAD2B230E4E3ED2FFFE43EFEE56D2408BC
:1052C400F56D12BC4EE4F5F7C2B2C2B2ADF7D2B27C
:1052D400EA30E508EB2DFBEC3400FC22C3EB9DFB2C
:0552E400EC9400FC2227
:0100030055A7
:10DF5C0069FC362E06FD69FC372F071169FD383038
:10DF6C0007FD69FD3931061169FE383107FD68FE80
:10DF7C003732091168FF373008FD68FF372D07115C
:10DF8C006800362909FE680036290C116801372B08
:10DF9C000CFF6801372F0A116802383009FF68023C
:10DFAC00372E08116803372C0AFE6803372E081128
:10DFBC006704373208FE67043633091167053535B7
:10DFCC0005FF6705353303116706362F02FF670619
:10DFDC00362B05116707362B07FF6707352F051101
:10DFEC006708353104FF6708332E0511670931289E
:10DFFC000700670931250A11670A35240B01670AE6
:10E00C003A240A11660A3C210801660B3D1E0B11CD
:10E01C00660B3D1E0C00660B3D200A11660C3B2165
:10E02C000CFF660C39220E11660C37231100660D9D
:10E03C0036240D11660D34260F01660E3226111191
:10E04C00660E32251401660F35251311660F37271E
:10E05C0016016610392918116610392B1502651135
:10E06C00392D11116511372E0C026512332F081141
:10E07C006512312F07026513302C0A1165132D29F7
:10E08C000E0265132A271011651429270E02651438
:10E09C002C290C1165153129080365153726071134
:10E0AC006515321F09036516411B09116516411CC4
:10E0BC0008036416461F081164164D2105046416E6
:10E0CC005922031164166425040563156A2407118B
:10E0DC0063156D23090663156C230D1163156C25EF
:10E0EC00130762146E2B151162146E2F1406621333
:10E0FC006E30161162136E30150761136F311211E9
:10E10C0061126F350F0761126F380D116011723A81
:10E11C000A086011763F0611601079420209600FFF
:10E12C007A3A0533600F7832040A5F0F742C01338E
:10E13C005F0E722B030A5F0E732E08115F0E743084
:10E14C00050C5F0D722C02135E0D6C2B010C5E0D19
:10E15C00622C05315E0D5F2B030D5D0D5E290833BE
:10E16C005D0D5F23030B5D0D5F1B01335D0D5A16B7
:10E17C00020A5D0D521B00115C0D4D26000C5C0E4D
:10E18C00462802335C0E3926040C5C0F2C2B08330A
:10E19C005C0F23320C0F5D0F172E0A335D0F0C2E04
:10E1AC0009105D0F043507335E0FB23C080F5F0F8B
:10E1BC00AB4209335F0EA43E070F5F0EA2430B3335
:10E1CC00600EA746120B600D9F490C73610C9C49A5
:10E1DC000F0C610B97460973610B8B440A0C610A97
:10E1EC008B420B336109843A080C6108823A043380
:10E1FC0061087934030C60086F2F063360086228BD
:10E20C00050C6008572505336008511F040D5F0885
:10E21C004E1B05335F08491B090D5F094120103760
:10E22C005F0938270D0D5F0A302F06335F0B2B3239
:10E23C00070F5F0B282F0A335F0B262E0E0E600C78
:10E24C0023361137600D1F3F160F600D18411277E2
:10E25C00610D0F320A13610D042B0633610D022E72
:10E26C00040E620D043A0231620E0343050D630D78
:10E27C00B1470113630DA94A000B640CA14D0511A4
:10E28C00640C9B44070E650B99490911650A944768
:10E29C00090D65098E49021365088848060D650845
:10E2AC0081400E336407793B130F6407722F187784
:10E2BC0064076D231A106407692911776407651CBC
:0DE2CC00080F63075D180B33630751190D30
:10E2D9000D630746220E336308402B110F6308387C
:10E2E900291837630932271B0D6309312B1477620B
:10E2F9000A372C0F0A620A3C280973620A441E0B6A
:10E309000C620A48150E33620B46190C0A620B4758
:10E31900260D33610B4C280C0B610B54251037610A
:10E329000B5E24170C600B63291A77600A66361492
:10E339000A600A68390B735F0A6C2C100A5F09724C
:10E349002015775F097422120A5F0873300F775F0F
:10E35900087639140A5F077D3816775F0785370F06
:10E36900095F068D3B0D735F058B4410075F048BB6
:10E37900490C735F048E3F0C075F03863604335FD5
:10E389000394280708600299300E1160029E400527
:10E39900076102A34A0C336101AA4810086201B15E
:10E3A90042127762020131150A6202062B13776362
:10E3B900020830110C63020B361277630310331114
:10E3C9000C6403182B147764032223110A640426AE
:10E3D90023107764042226110A64051C2715776423
:10E3E900051D251508640521271277640628270FBE
:10E3F9000764062F1D11776406350F140764063E5E
:10E409000A19776406401216086407431B117763DB
:10E41900074A22120663075228127763075A2713FD
:10E429000662075E2314776206612011076206649B
:10E439001E0E7362066A1E0E076206742110376289
:10E44900057828130661057A2F157761047A332038
:10E459000661047A301B7761037A281B0761037F01
:10E4690023187761028429160661028832177761B9
:10E47900018D371305610193340C7362009A2E09DB
:10E489000562009D2E043362009D370C0663FFA0D0
:10E4990040103763FFA844140564FFAF4612776440
:10E4A900FF014511056500043F12776500053E101F
:10E4B900076600073F117766000B430D07670110D8
:10E4C9003D117367011539120767021A321277670E
:10E4D900021A2C12076702192C107768031B2E0FDA
:10E4E9000668031F2C117768042729100468042E75
:10E4F9002A0F776705322F130467053330127767C0
:10E5090006362D140567063B291677670643231B34
:10E51900046706471E16776607491E150366074CEA
:10E529001B157766074C2217046607522214776574
:10E53900075B26150265066229157765066D291799
:10E549000165067529137765057D281A0265058217
:10E5590028187765047F1F160265048F2A117765CD
:10E5690003953211006602993D157766029C401C9D
:10E57900FF6602A13E1F776701A43F1CFF6701A741
:10E589004314776801AB4710FF6901B1490F7769F7
:10E5990001024911026A0207490D736A020B480C0C
:10E5A900056B030F480B336B03144A0D026B0419F7
:10E5B9004914376B051F491CFE6C06224824776CE9
:10E5C90006233F21FC6C07203023776C0721272184
:10E5D900FC6C07262420776C08292812FC6C082873
:10E5E9002C0F776C0927230CFF6C09251802316C55
:10E5F90009350F05FC6C094C1401116C09561D01F4
:10E60900FC6B095F2003136B086B2108FB6B087413
:10E619002509336B08772507FC6B0778210D336BC8
:10E62900077A1E0AFB6B077F220C336B06832E0ABF
:10E63900FA6B05853C09336B0489410EF96B048C2F
:0DE649003E10376B038D3C0FFA6B038D40C4
:10E6560013776B02904112FA6C01934110776C01AB
:10E66600984410F86C009B471A776D009F461EF879
:10E676006DFFA24519776EFFA14019F86EFFA640FF
:10E6860014776FFEAA4417FA6FFEAF4A127770FE30
:10E69600B34D18FA70FF024B1B7771FF054718FD43
:10E6A60071FF0942177772000E4012FD7200163D87
:10E6B6000C7372011B3510FA7201232E1577720244
:10E6C60029321AF872032C371D7772032F3014F88B
:10E6D600720336210F77710346190DF87103502026
:10E6E6000B33710353290EF87003572B143770033D
:10E6F600612712F870036F2911777002793017F7C6
:10E706007001803722777001843D1FF67000883FC4
:10E71600197770FF8D3F11F670FF933D0C7371FEF4
:10E72600973D0EF571FE9B3E0C3372FD9F4310F62E
:10E7360072FDA448127773FDAB4C13F573FDB14F10
:10E74600167774FD034F14F775FE074C127775FEA6
:10E756000A4510F975FE0E400F7776FF124111F843
:10E7660076001745167776001C4614F67601214288
:10E7760017777602263D17F3760229382177760336
:10E786002A3315F276032B3009737604302A07F004
:10E79600760439220A337604472110F07504512590
:10E7A60012777504552416F1750459210F777504EF
:10E7B6005F2111F0740463231477740468240EF245
:10E7C600740370230933740379270AEF74028030C7
:10E7D6000B33740185360DEF74018B3913377400D2
:10E7E600903D1BF075FF94441E7775FF984823EF04
:10E7F60075FE9B46207776FE9F4221F076FEA13F6E
:10E80600177777FDA44313EF77FDA747157778FDB4
:10E81600AA4915EF78FDAD4C157779FDB04D19EE87
:10E826007AFDB34D1C777AFD024E19F07BFD054F3C
:10E836001B777BFE094F24F37CFE0D531D777CFF6F
:10E84600114619F37CFF173F12777C001F3810EF33
:10E856007C00263613777C012B3115ED7C012F2B9E
:10E8660015777C02332513ED7C02392214777C025E
:10E87600402110EE7C0249210B737B02531F0FEBE4
:10E886007B02601E15777B026A2214EA7B017428DC
:10E8960019777B017B2D1AEA7B00833122777B0077
:10E8A6008A3320EB7BFF91371A777BFE953C1FEA74
:10E8B6007CFE983C26777CFEA74621EC7CFD9939A8
:10E8C60023777CFC9A3B1FEA7DFC9A3F1C777DFBF5
:10E8D6009A401EE87DFB9B3F20777EFA9B3F1FE612
:10E8E6007EFA9C431A777EF99E4717E57FF8A04A81
:10E8F6000E737FF8A34A0AEA80F8A548073380F822
:10E90600A94402EA81F8AE46041182F8B24C00E747
:10E9160082F80351021183F8085304EA83F90E4D75
:10E92600061183F914430CEC84FA1A400E1184FB89
:10E93600203F0AE884FC2540061384FC2B4008E6A9
:10E9460084FD3039073383FD36300EE483FE3C2BDD
:10E95600193783FE402A1EE783FE3D25187783FE7E
:10E96600371B16E783FF3114137783FF35170FE440
:10E9760083FF3E220D738200412C15E58200432C55
:10E986001A77820046251BE782004C201577810006
:10E99600552116E581005E2510778100682718E469
:10E9A60081FF72291E7780FF7A2E22E580FE7E3057
:10E9B600277780FE812B22E680FD85251C7780FD4A
:0DE9C600882618E281FC8A2F187781FC8DCD
:10E9D3003821E181FB903F287781FA924025E0813D
:10E9E300FA943D237782F9973C18E082F99A3F1510
:10E9F3007782F89E4412E083F8A347107783F8A741
:10EA03004A0CDF84F8AA4D133785F7AC5214E2851C
:10EA1300F7AF56107786F7B2580DE087F802560223
:10EA23003387F8055002E388F8094C051188F90C7F
:10EA33004E02E489F91052011189FA155004DF8955
:10EA4300FB1D45041389FB233304DE89FB292306BD
:10EA53003389FC2B1F05DE89FC2F23093389FD3302
:10EA6300280ADC89FD3B23103788FD471E0EDD880D
:10EA7300FD511E0E3388FD53200CDD88FD54210B00
:10EA83003387FD57200DDD87FD5C20093387FD5D4E
:10EA93002403DE87FD5B29013386FD592C04DE86C2
:10EAA300FD5D2C093385FD622F0CDC85FD652D0B87
:10EAB3003385FC672908DF85FC6722093385FC6BF6
:10EAC300210CDD84FC72280A3384FB783005DD8455
:10EAD300FA7C37073384FA7E390ADC84F9813B06F2
:10EAE3003384F8843F05DB84F8873F023384F78A55
:10EAF3003C04DB84F78D390A3384F6903908D985D1
:10EB0300F5923F113785F595430FD985F498440A5B
:10EB13007386F49B440AD986F39C440C3386F39C96
:10EB23004507DA87F29C47063387F19E4C0AD9885A
:10EB3300F1A251103788F1A65516D989F0A7571FAE
:10EB4300778AF0A9541BDA8AF0AA4D12778BF0ACBE
:10EB5300460DDB8BF0AC4906338CEFAB4D05DB8CFC
:10EB6300EFA95002318DEEA85209E28DEEA7530EA4
:10EB7300118EEEA75316E58EEDA44A20118FEDA05A
:10EB83004423E28FEC9C4821118FEB9A4A22E090B8
:10EB9300EB95411D1190EA8E391DDF90EA893621EC
:10EBA3001190E9873223E590E9852C2C118FE87DBC
:10EBB3002A26E08FE8762124118FE8662122E08F50
:10EBC300E856221F118EE947201DE08EE9392116F0
:10EBD300118EE9302518E28EEA2D2917118EEB30BC
:10EBE3003213E18EEB333711118EEC373C10E18E8B
:10EBF300ED393E07138DED3B4203DD8DEE3B3E09C0
:10EC0300338DEE3B310DDE8DEE392812378DEF3823
:10EC13002319DC8DEF382A18778DF0372A12DC8D13
:10EC2300F0382214778DF0361B0EDC8DF1361B0C79
:10EC3300338CF1371F0DDB8CF136250E378CF23414
:10EC4300270CDC8CF22A270D338DF31F2A0CDC8D65
:10EC5300F3173409338DF4143A08E48EF4123A0CA2
:10EC6300338EF4103D11EA8FF50E411A778FF50CB0
:10EC73004917EA90F50A50157790F5054F13E79178
:10EC8300F5B24F107792F5AD5408E492F4AB5A0104
:10EC93003393F4AB5C05E893F4A9500A3394F3A4DB
:10ECA300450CE094F3A041093394F29A3A05E295B6
:10ECB300F29734043395F1913208DC95F19E310DCE
:10ECC3003395F08A320CDA95F0872D0B3395EF806C
:10ECD300250EDE94EF73220C3394EF6C2412DD9433
:10ECE300EF6928157794EE6B2812DF93EE69280EEF
:10ECF3007393EE64270DDF93EE5C260B3392EE578E
:10ED0300270EDB92EE5828123792EE5E2610DB9226
:10ED1300EE64240D7391EE6C2108D991ED722304F6
:10ED23003391ED782904D991EC7C320A3391EB7F4E
:10ED33003A08D891EB833D093391EA883C0CD7918B
:0DED4300E98D3B103791E9903E12D792E820
:10ED50009143137792E794420ED792E7993E073397
:10ED600093E7A03901D993E7A63B0A1194E6A83F9F
:10ED70000CD794E6AB490E1195E6AE4F07D695E653
:10ED8000004D011396E6034601D996E6033E0811AD
:10ED900097E7043D0ED997E70740151198E70C4314
:10EDA00012DA98E812460F1198E918490CDA98E936
:10EDB0001D44081198EA243D05D898EB293A03111F
:10EDC00098EB2C3707D898EC2D38093398ED2E3D69
:10EDD0000ADC98ED2E3E0A3398EE2D3F0BDB98EFC0
:10EDE0002C420C3398F02B430ED998F02B3D113761
:10EDF00098F12D3710D898F130340D7398F23433E0
:10EE00000FD698F237330F7798F339331CD597F331
:10EE10003C32167797F43E2F11D797F440280973A8
:10EE200097F4422109D797F4461F0AB396F44B2171
:10EE300008D796F45325083396F45C2505D796F445
:10EE40006723023395F4722503D695F3782B0231AC
:10EE500095F37B3102D695F27E31063395F1832FFF
:10EE600004D695F18A2F023395F0913201D596F0B0
:10EE70009638061196EF9A3F02D497EF9D450213FC
:10EE800097EE9F4704D497EEA247073398EEA64427
:10EE900008D398EEAA430B3399EEAD440CD499EE07
:10EEA000B1400D339AEE013F11D39AEE054512772A
:10EEB0009BEE064A15D59BEE064712779CEF05425E
:10EEC00012D79CEF063E0F779DEF084111D39DEFBF
:10EED000094619779EF00B4718D39EF00D431C7717
:10EEE0009FF10F4015D69FF1114113779FF2134602
:10EEF0000ED9A0F2174A0B33A0F31C4A08D4A0F491
:10EF000023420333A0F42A3305D3A0F53127071198
:10EF1000A0F5382300D29FF53D2702339FF6442900
:10EF200003D39FF64F2808119EF55E2807D19EF562
:10EF30006C2D04119EF4752F01D09EF47C2D0433AA
:10EF40009EF3822B04D09EF3872E05119EF28B3503
:10EF500007D09EF2903D01119FF1954203D09FF0A2
:10EF600094400333A0F09F3F0BD0A0F0A13D0F379A
:10EF7000A0EFA33C0DD1A1EFA43C0C33A1EFA43C26
:10EF80000AD0A1EEA53D0533A2EEA63C00D1A2EE2B
:10EF9000A8390211A3EEAA3C04D0A3EEAD3F05119F
:10EFA000A4EEB24008D0A4EE03410C11A5EE064138
:10EFB0000AD2A5EE08450711A6EF094A05D2A6EF29
:10EFC000094C0111A7EF0A4807D3A7F00B420B1118
:10EFD000A8F00B420DD4A8F00D461311A9F111466B
:10EFE00014D9A9F1173F1B11A9F21E381ADAA9F397
:10EFF00021381811A9F31F3A17DFA9F41839151190
:10F00000AAF4163A1DDCAAF5183C1A11AAF51C3A06
:10F010001AD9AAF61F391A11ABF6203615D9ABF753
:10F0200021341711ABF8203B19D9ABF81E3F17114B
:10F03000ACF91D4011D9ACF91E3F0E11ACFA1F40BE
:10F040000CD6ACFB22410D11ACFC23450FD6ADFC18
:10F0500023490B11ADFD214A0DD6ADFE2047091104
:10F06000ADFE21450CD6ADFF22430E11AE00224568
:10F070000CD8AE01214B0A11AE0220500DD7AF03C0
:10F080001D4F0B11AF031A5109D9AF04174A0D11C7
:10F09000B00418470BDBB0051A500A11B0061C5516
:10F0A0000ED7B1071C560B11B10719470ED9B1087D
:10F0B000173C0C11B208183D0CDCB2091C490E11AA
:0DF0C000B20A1E4E0AD9B30B1D500B11B33E
:10F0CD000C1A5109D9B30C174F0711B40D17490B71
:10F0DD00DBB40D17480D11B50E19490ADCB50F1922
:10F0ED004F0B11B50F185605DBB61017550711B696
:10F0FD0011174C0ADBB61116430B11B711173F0D43
:10F10D00DDB71219430C11B7131A480BDCB8131ADB
:10F11D00450F11B81419410DDCB81418400B11B975
:10F12D001518430DDBB91618470F11B91618490DEF
:10F13D00DBBA1718470A11BA1717450CDBBB1814A1
:10F14D00460F11BB18134C0EDBBC1912510A11BC22
:10F15D001A125007DBBC1A12470B11BD1A10400DC5
:10F16D00DCBD1B10400A11BE1B124509DCBE1C156F
:10F17D00490B11BE1D184A0ADBBF1D1B4A0811BFE2
:10F18D001E1B480CDBBF1F1A470E11BF1F1A490B60
:10F19D00DBC0201B4B0D11C0211C4910DBC0211DF4
:10F1AD00470F11C1221D4711DBC1231C4B0F11C18C
:10F1BD00231B4B0EDBC22419441111C224193D0F20
:10F1CD00DBC2251B3B1011C2261D3F0DDAC2261EC8
:10F1DD00411011C3271D3F12DAC3271C3D0F11C368
:10F1ED00281B3D10DBC4291C401111C4291C450FDF
:10F1FD00DCC42A1C460E11C42A1B4510DCC52B1974
:10F20D00431111C52C184511DDC62C164A1011C617
:10F21D002D174A11DEC62D18491211C72E19471088
:10F22D00DEC72F1A460E11C72F1C4410DFC7301F23
:10F23D00471111C731214B0CDBC832224D0E11C8BD
:10F24D0032224A10DAC83321471111C83420460F33
:10F25D00D9C83520461111C93521430CDBC93623D8
:10F26D003F0F11C937253D11DBC93725400E11C997
:10F27D0038254211DCC93925431311C939254312EB
:10F28D00DCC93A25431111CA3B24400DDCCA3C248C
:10F29D00411011CA3C23400EDCCA3D22401111CA57
:10F2AD003E20420FDECB3E20451011CB3F204714B0
:10F2BD00DECB4021441211CB40213F10DFCB412248
:10F2CD003C0D11CB42234011DFCC42233E1111CC1A
:10F2DD0043202F0EE0CC4319221211CC43122011E2
:10F2ED00E3CC4311250E11CD43132B10E3CD441266
:10F2FD002D1111CD440F2B0FE3CD44092B1211CE3F
:10F30D004404320FE2CE4401360E11CF44B3370D13
:10F31D00E0CF44B3330E11D04401370EE0D0440595
:10F32D003D0D11D0450A3B0CE3D14512330D11D1E2
:10F33D00451A2D0EE3D1461E2B0F11D1461D2E0F52
:10F34D00E4D1471D300F11D1471E320EE3D24821B3
:10F35D00330F11D248233510E2D24923350F11D284
:10F36D004A20360EE3D24A1D360E11D24B1B3410F5
:10F37D00E3D34B1B320F11D34B1B300EE4D34C1B7D
:10F38D00340D11D34C1B3A0DE5D44D1A3B0E11D44F
:10F39D004D1B360AE6D44E1D340E11D44E1E360DBD
:10F3AD00E5D44F1F360C11D5501F350EE5D5501F26
:10F3BD00340D11D5511E340EE5D5511E370C11D516
:10F3CD00521E390EE5D652203B0F11D653223C0F5B
:10F3DD00E4D65423391111D654243710E3D65524CD
:10F3ED00360F11D655253310E3D65626330D11D6CB
:10F3FD005627350BE2D657273A0C11D658273C0F16
:10F40D00E2D75827391011D75927370FE2D75A2786
:10F41D00381011D75A283B0FE2D75B293C1111D771
:10F42D005C2B3C12E2D75C2D391111D75D2C3910B4
:0DF43D00E3D75E2B3C0F11D75E293B0EE399
:10F44A00D75F27371011D75F26360EE3D760273CE0
:10F45A000E11D761284310E3D76229451111D762EB
:10F46A00293F0FE4D763283A1011D763293A11E4E8
:10F47A00D7642A3E1011D7652C4211E4D7662E4272
:10F48A001011D7662D3F11E4D7672F3A1011D768AC
:10F49A002D3B0CE4D7682E3D0711D7692E4204E4B0
:10F4AA00D76A2E470111D76B2E4702E4D76B2D403E
:10F4BA000513D76C2B3503E4D76C2A2B0711D76DAC
:10F4CA002B2909E5D76D2B300611D76E2A3A04E4A9
:10F4DA00D76F28400611D76F283E08E4D77027381F
:10F4EA000C11D87026320DE6D871252F0911D87162
:10F4FA0024310AE9D87221340811D8721B3A08EA71
:10F50A00D9730D420A11D973104909EADA730C4505
:10F51A000811DA730A3B06E8DB74093D0211DB7451
:10F52A000A4003E9DB740B3C0213DC75103406EA6B
:10F53A00DC7517350333DC761A3F06EADD771C469D
:10F54A000433DD771F4001E8DD7824360731DD78A2
:10F55A002C3206E7DC7933320413DC79373409E7D5
:10F56A00DC7A3A340C33DC7A3C3508E7DC7B3D370D
:10F57A000233DB7C3C3A05E7DB7C3C3D0333DB7D35
:10F58A003B3A04E7DB7D3B320331DA7D3E2D09EA63
:10F59A00DA7E43270D11DA7E4D230AE9DA7E5726F1
:10F5AA000B11D97D5E2C0BE9D97D61300C11D97D07
:10F5BA00632F08EAD87D662F0511D87C683005EAE2
:10F5CA00D87C6D330611D77B733608E9D77B7C3834
:10F5DA000511D77A853A04E8D8798B3B0711D8798F
:10F5EA008E3809E9D8788F371011D878903B0BE814
:10F5FA00D87791420D11D976954A08E7D976984974
:10F60A000411D9759D4008E8DA75A23A0B33DA7508
:10F61A00A53C0AE8DB75A8430031DB74AA4603E976
:10F62A00DC74AF460213DC74004A02EADD75054C4D
:10F63A000333DD75084D00EDDE75084B0533DF76C3
:10F64A00064902EDDF76044A0131E076044902EA0E
:10F65A00E076044C0513E176045006EAE176014DA2
:10F66A000D33E276B1450FEAE276AD3F1077E375E6
:10F67A00AB3F0DEAE375AC430A33E475AE4604EAE0
:10F68A00E475B0400131E575B23908EAE575013C27
:10F69A000611E675054607ECE6760A4B0311E7768E
:10F6AA000F4604EEE777163B0611E778203405EC9F
:10F6BA00E77827350611E7792D3409ECE7793234F2
:10F6CA000B11E77A3B260AECE67A45250B11E67A16
:10F6DA004D230BEAE67A56250711E67A5F270AEAEE
:10F6EA00E579672A0C11E579731F0AEBE578792E1B
:10F6FA000811E578843302EAE5778D3B0313E67651
:10F70A00954104EAE676993F0733E6759A3801EAA5
:10F71A00E67595310531E6748F3202EAE6748E3564
:10F72A000111E773923301EAE77398310413E77220
:0AF73A009D3304EBE872B4370911A7
:00000001FF
